:020000040800F2
:1000000000200020D1B5000819B6000819B6000874
:1000100019B6000819B6000819B60008000000005B
:1000200000000000000000000000000019B60008F9
:1000300019B600080000000019B600087F970008F4
:1000400019B6000819B6000819B6000819B6000854
:1000500019B6000819B600086D98000873980008D2
:10006000799800087F9800088598000819B600085C
:1000700019B6000819B6000819B6000819B6000824
:1000800019B6000819B6000819B6000800000000EB
:100090000000000000000000000000008B98000835
:1000A000D591000839910008E99100085D91000898
:1000B00071910008859100089991000819B600080F
:1000C00019B60008000000000000000019B6000882
:1000D00019B6000871A6000889A60008A5A60008A0
:1000E000A198000819B6000819B600080000000021
:1000F0000000000000000000000000000000000000
:1001000000000000000000000000000000000000EF
:100110000000000000000000AD910008C19100083F
:1001200000000000000000000000000000000000CF
:1001300000000000000000000000000000000000BF
:1001400000000000000000000000000000000000AF
:10015000000000000000000000000000000000009F
:10016000000000000000000000000000000000008F
:10017000000000000000000000000000000000007F
:10018000000000000000000000000000000000006F
:10019000000000000000000000000000000000005F
:1001A000000000000000000000000000000000004F
:1001B000000000000000000000000000000000003F
:1001C0000000000000000000000000005FF808F1DF
:1001D00010F8012B11F8013B012A28BF9A42F7D0F1
:1001E000D01A7047034613F8012B002AFBD1181AC6
:1001F0000138704781F0004102E000BF83F0004306
:1002000030B54FEA41044FEA430594EA050F08BFB1
:1002100090EA020F1FBF54EA000C55EA020C7FEA75
:10022000645C7FEA655C00F0E2804FEA5454D4EBF2
:100230005555B8BF6D420CDD2C4480EA020281EABC
:10024000030382EA000083EA010180EA020281EAF4
:100250000303362D88BF30BD11F0004F4FEA013146
:100260004FF4801C4CEA113102D0404261EB410155
:1002700013F0004F4FEA03334CEA133302D05242DB
:1002800063EB430394EA050F00F0A780A4F1010497
:10029000D5F1200E0DDB02FA0EFC22FA05F28018D1
:1002A00041F1000103FA0EF2801843FA05F35941B7
:1002B0000EE0A5F120050EF1200E012A03FA0EFC36
:1002C00028BF4CF0020C43FA05F3C01851EBE37160
:1002D00001F0004507D54FF0000EDCF1000C7EEB7D
:1002E00000006EEB0101B1F5801F1BD3B1F5001FBB
:1002F0000CD349085FEA30004FEA3C0C04F10104DA
:100300004FEA445212F5800F80F09A80BCF1004F02
:1003100008BF5FEA500C50F1000041EB045141EA84
:10032000050130BD5FEA4C0C404141EB0101013C4D
:1003300028BFB1F5801FE9D291F0000F04BF01463C
:100340000020B1FA81F308BF2033A3F10B03B3F10E
:1003500020020CDA0C3208DD02F1140CC2F10C029E
:1003600001FA0CF021FA02F10CE002F11402D8BFFC
:10037000C2F1200C01FA02F120FA0CFCDCBF41EAC8
:100380000C019040E41AA2BF01EB0451294330BD97
:100390006FEA04041F3C1CDA0C340EDC04F1140474
:1003A000C4F1200220FA04F001FA02F340EA03004B
:1003B00021FA04F345EA030130BDC4F10C04C4F191
:1003C000200220FA02F001FA04F340EA0300294671
:1003D00030BD21FA04F0294630BD94F0000F83F4BB
:1003E000801306BF81F480110134013D4EE77FEA9E
:1003F000645C18BF7FEA655C29D094EA050F08BFEA
:1004000090EA020F05D054EA000C04BF19461046CA
:1004100030BD91EA030F1EBF0021002030BD5FEA0E
:10042000545C05D14000494128BF41F0004130BD36
:1004300014F580043CBF01F5801130BD01F000458A
:1004400045F0FE4141F470014FF0000030BD7FEAFD
:10045000645C1ABF194610467FEA655C1CBF0B46F8
:10046000024650EA013406BF52EA033591EA030F0F
:1004700041F4002130BD00BF90F0000F04BF002107
:10048000704730B54FF4806404F132044FF000053A
:100490004FF0000150E700BF90F0000F04BF0021B3
:1004A000704730B54FF4806404F1320410F0004519
:1004B00048BF40424FF000013EE700BF42004FEA14
:1004C000E2014FEA31014FEA02701FBF12F07F4391
:1004D00093F07F4F81F06051704732F07F4208BF48
:1004E000704793F07F4F04BF41F40021704730B54F
:1004F0004FF4607401F0004521F000411CE700BF9B
:1005000050EA010208BF704730B54FF000050AE01D
:1005100050EA010208BF704730B511F0004502D51E
:10052000404261EB41014FF4806404F132045FEA20
:10053000915C3FF4D8AE4FF003025FEADC0C18BFC9
:1005400003325FEADC0C18BF033202EBDC02C2F1BB
:10055000200300FA03FC20FA02F001FA03FE40EA4D
:100560000E0021FA02F11444BDE600BF70B54FF051
:10057000FF0C4CF4E06C1CEA11541DBF1CEA13552F
:1005800094EA0C0F95EA0C0F00F0DEF82C4481EA97
:10059000030621EA4C5123EA4C5350EA013518BFB7
:1005A00052EA033541F4801143F4801338D0A0FBA4
:1005B00002CE4FF00005E1FB02E506F00042E0FB51
:1005C00003E54FF00006E1FB03569CF0000F18BF57
:1005D0004EF0010EA4F1FF04B6F5007F64F54074FF
:1005E00004D25FEA4E0E6D4146EB060642EAC62192
:1005F00041EA55514FEAC52040EA5E504FEACE2EFF
:10060000B4F1FD0C88BFBCF5E06F1ED8BEF1004F01
:1006100008BF5FEA500E50F1000041EB045170BD7D
:1006200006F0004646EA010140EA020081EA0301C1
:10063000B4EB5C04C2BFD4EB0C0541EA045170BDBD
:1006400041F480114FF0000E013C00F3AB8014F137
:10065000360FDEBF002001F0004170BDC4F1000480
:10066000203C35DA0C341BDC04F11404C4F1200501
:1006700000FA05F320FA04F001FA05F240EA02005C
:1006800001F0004221F0004110EBD37021FA04F692
:1006900042EB06015EEA430E08BF20EAD37070BD4C
:1006A000C4F10C04C4F1200500FA04F320FA05F0AB
:1006B00001FA04F240EA020001F0004110EBD370AD
:1006C00041F100015EEA430E08BF20EAD37070BD1D
:1006D000C4F1200500FA05F24EEA020E20FA04F3F6
:1006E00001FA05F243EA020321FA04F001F00041A5
:1006F00021FA04F220EA020000EBD3705EEA430E16
:1007000008BF20EAD37070BD94F0000F0FD101F044
:100710000046400041EB010111F4801F08BF013C7D
:10072000F7D041EA060195F0000F18BF704703F0BB
:100730000046520043EB030313F4801F08BF013D42
:10074000F7D043EA0603704794EA0C0F0CEA1355FE
:1007500018BF95EA0C0F0CD050EA410618BF52EAB8
:100760004306D1D181EA030101F000414FF00000BE
:1007700070BD50EA410606BF1046194652EA4306CC
:1007800019D094EA0C0F02D150EA013613D195EA40
:100790000C0F05D152EA03361CBF104619460AD188
:1007A00081EA030101F0004141F0FE4141F4700192
:1007B0004FF0000070BD41F0FE4141F4780170BD82
:1007C00070B54FF0FF0C4CF4E06C1CEA11541DBFE7
:1007D0001CEA135594EA0C0F95EA0C0F00F0A7F8E9
:1007E000A4EB050481EA030E52EA03354FEA013116
:1007F00000F088804FEA03334FF0805545EA131329
:1008000043EA12634FEA022245EA111545EA1065F0
:100810004FEA00260EF000419D4208BF964244F187
:10082000FD0404F5407402D25B084FEA3202B61AA6
:1008300065EB03055B084FEA32024FF480104FF47A
:10084000002CB6EB020E75EB030E22BFB61A7546EE
:1008500040EA0C005B084FEA3202B6EB020E75EB81
:10086000030E22BFB61A754640EA5C005B084FEAE9
:100870003202B6EB020E75EB030E22BFB61A7546B6
:1008800040EA9C005B084FEA3202B6EB020E75EBC1
:10089000030E22BFB61A754640EADC0055EA060E82
:1008A00018D04FEA051545EA16754FEA06164FEAC5
:1008B000C30343EA52734FEAC2025FEA1C1CC0D171
:1008C00011F4801F0BD141EA00014FF000004FF0FE
:1008D000004CB6E711F4801F04BF01430020B4F1BF
:1008E000FD0C88BFBCF5E06F3FF6AFAEB5EB030C77
:1008F00004BFB6EB020C5FEA500C50F1000041EB74
:10090000045170BD0EF0004E4EEA113114EB5C0440
:10091000C2BFD4EB0C0541EA045170BD41F4801113
:100920004FF0000E013C90E645EA060E8DE60CEA1B
:10093000135594EA0C0F08BF95EA0C0F3FF43BAF38
:1009400094EA0C0F0AD150EA01347FF434AF95EAEF
:100950000C0F7FF425AF104619462CE795EA0C0FD3
:1009600006D152EA03353FF4FDAE1046194622E7A0
:1009700050EA410618BF52EA43067FF4C5AE50EA7A
:1009800041047FF40DAF52EA43057FF4EBAE12E76A
:100990004FF0FF3C06E000BF4FF0010C02E000BF4B
:1009A0004FF0010C4DF804CD4FEA410C7FEA6C5C2E
:1009B0004FEA430C18BF7FEA6C5C1BD001B050EAD1
:1009C000410C0CBF52EA430C91EA030F02BF90EABC
:1009D000020F0020704710F1000F91EA030F58BF7B
:1009E000994208BF90422CBFD8176FEAE37040F0DD
:1009F000010070474FEA410C7FEA6C5C02D150EA7B
:100A0000013C07D14FEA430C7FEA6C5CD6D152EA35
:100A1000033CD3D05DF8040B704700BF84461046FA
:100A200062468C461946634600E000BF01B5FFF7F9
:100A3000B7FF002848BF10F1000F01BD4DF808EDC9
:100A4000FFF7F4FF0CBF012000205DF808FB00BF9A
:100A50004DF808EDFFF7EAFF34BF012000205DF8F4
:100A600008FB00BF4DF808EDFFF7E0FF94BF012041
:100A700000205DF808FB00BF4DF808EDFFF7CEFF42
:100A800094BF012000205DF808FB00BF4DF808ED81
:100A9000FFF7C4FF34BF012000205DF808FB00BF52
:100AA0004FEA410C7FEA6C5C02D150EA013C0AD16A
:100AB0004FEA430C7FEA6C5C02D152EA033C02D15C
:100AC0004FF0000070474FF0010070474FEA4102BD
:100AD00012F5001215D211D56FF47873B3EB625290
:100AE00012D94FEAC12343F0004343EA505311F0B7
:100AF000004F23FA02F018BF404270474FF0000049
:100B0000704750EA013005D111F0004008BF6FF086
:100B1000004070474FF00000704700BF4A0011D2FC
:100B200012F5001211D20DD56FF47873B3EB625247
:100B30000ED44FEAC12343F0004343EA505323FA53
:100B400002F070474FF00000704750EA013002D1C8
:100B50004FF0FF3070474FF0000070474FEA4102FE
:100B6000B2F1E04324BFB3F5001CDCF1FE5C0DD90B
:100B700001F0004C4FEAC0024CEA5070B2F1004F55
:100B800040EB830008BF20F00100704711F0804F58
:100B900021D113F13872BCBF01F00040704741F41D
:100BA00080114FEA5252C2F11802C2F1200C10FA21
:100BB0000CF320FA02F018BF40F001004FEAC12305
:100BC0004FEAD32303FA0CFC40EA0C0023FA02F3A9
:100BD0004FEA4303CCE77FEA625307D150EA01337F
:100BE0001EBF4FF0FE4040F44000704701F000404F
:100BF00040F0FE4040F40000704700BF80F000402D
:100C000002E000BF81F0004142001FBF5FEA4103E4
:100C100092EA030F7FEA226C7FEA236C6AD04FEAE4
:100C20001262D2EB1363C1BFD21841404840414029
:100C3000B8BF5B42192B88BF704710F0004F40F4DB
:100C4000000020F07F4018BF404211F0004F41F4F7
:100C5000000121F07F4118BF494292EA030F3FD0C3
:100C6000A2F1010241FA03FC10EB0C00C3F12003D6
:100C700001FA03F100F0004302D5494260EB400065
:100C8000B0F5000F13D3B0F1807F06D340084FEAD0
:100C9000310102F10102FE2A51D2B1F1004F40EBC5
:100CA000C25008BF20F0010040EA0300704749002D
:100CB00040EB0000013A28BFB0F5000FEDD2B0FACA
:100CC00080FCACF1080CB2EB0C0200FA0CF0AABFED
:100CD00000EBC25052421843BCBFD040184370478B
:100CE00092F0000F81F4000106BF80F40000013291
:100CF000013BB5E74FEA41037FEA226C18BF7FEA68
:100D0000236C21D092EA030F04D092F0000F08BFA9
:100D10000846704790EA010F1CBF0020704712F090
:100D20007F4F04D1400028BF40F00040704712F1CF
:100D300000723CBF00F50000704700F0004343F034
:100D4000FE4040F4000070477FEA226216BF08466A
:100D50007FEA23630146420206BF5FEA412390EA2D
:100D6000010F40F4800070474FF0000304E000BF23
:100D700010F0004348BF40425FEA000C08BF7047D4
:100D800043F0964301464FF000001CE050EA010298
:100D900008BF70474FF000030AE000BF50EA0102AD
:100DA00008BF704711F0004302D5404261EB41019A
:100DB0005FEA010C02BF84460146002043F0B643BF
:100DC00008BFA3F18053A3F50003BCFA8CF2083AE4
:100DD000A3EBC25310DB01FA02FC634400FA02FCED
:100DE000C2F12002BCF1004F20FA02F243EB0200F4
:100DF00008BF20F00100704702F1200201FA02FC56
:100E0000C2F1200250EA4C0021FA02F243EB020048
:100E100008BF20EADC7070474FF0FF0C1CEAD0528C
:100E20001EBF1CEAD15392EA0C0F93EA0C0F6FD04D
:100E30001A4480EA010C400218BF5FEA41211ED02B
:100E40004FF0006343EA501043EA5111A0FB013117
:100E50000CF00040B1F5000F3EBF490041EAD371EC
:100E60005B0040EA010062F17F02FD2A1DD8B3F168
:100E7000004F40EBC25008BF20F00100704790F0D7
:100E8000000F0CF0004C08BF49024CEA502040EA29
:100E900051207F3AC2BFD2F1FF0340EAC2507047EF
:100EA00040F400004FF00003013A5DDC12F1190F2D
:100EB000DCBF00F000407047C2F10002410021FA9F
:100EC00002F1C2F1200200FA02FC5FEA310040F1B7
:100ED000000053EA4C0308BF20EADC70704792F030
:100EE000000F00F0004C02BF400010F4000F013A68
:100EF000F9D040EA0C0093F0000F01F0004C02BF63
:100F0000490011F4000F013BF9D041EA0C018FE7D1
:100F10000CEAD15392EA0C0F18BF93EA0C0F0AD0D7
:100F200030F0004C18BF31F0004CD8D180EA0100FD
:100F300000F00040704790F0000F17BF90F0004F96
:100F4000084691F0000F91F0004F14D092EA0C0F78
:100F500001D142020FD193EA0C0F03D14B0218BF0B
:100F6000084608D180EA010000F0004040F0FE4051
:100F700040F40000704740F0FE4040F440007047ED
:100F80004FF0FF0C1CEAD0521EBF1CEAD15392EA6C
:100F90000C0F93EA0C0F69D0A2EB030280EA010C5C
:100FA00049024FEA402037D04FF0805343EA1111F5
:100FB00043EA10130CF000408B4238BF5B0042F153
:100FC0007D024FF4000C8B4224BF5B1A40EA0C00F8
:100FD000B3EB510F24BFA3EB510340EA5C00B3EB2A
:100FE000910F24BFA3EB910340EA9C00B3EBD10F18
:100FF00024BFA3EBD10340EADC001B0118BF5FEA6A
:101000001C1CE0D1FD2A3FF650AF8B4240EBC25092
:1010100008BF20F0010070470CF0004C4CEA502053
:101020007F32C2BFD2F1FF0340EAC250704740F4A2
:1010300000004FF00003013A37E792F0000F00F094
:10104000004C02BF400010F4000F013AF9D040EA12
:101050000C0093F0000F01F0004C02BF490011F4A6
:10106000000F013BF9D041EA0C0195E70CEAD1539E
:1010700092EA0C0F08D142027FF47DAF93EA0C0F85
:101080007FF470AF084676E793EA0C0F04D14B0269
:101090003FF44CAF08466EE730F0004C18BF31F01B
:1010A000004CCAD130F000427FF45CAF31F0004315
:1010B0007FF43CAF5FE700BF4FF0FF3C06E000BFAE
:1010C0004FF0010C02E000BF4FF0010C4DF804CDD1
:1010D0004FEA40024FEA41037FEA226C18BF7FEAE1
:1010E000236C11D001B052EA530C18BF90EA010FE3
:1010F00058BFB2EB030088BFC81738BF6FEAE17072
:1011000018BF40F0010070477FEA226C02D15FEA0D
:10111000402C05D17FEA236CE4D15FEA412CE1D079
:101120005DF8040B704700BF844608466146FFE740
:101130000FB5FFF7C9FF002848BF10F1000F0FBD22
:101140004DF808EDFFF7F4FF0CBF012000205DF81B
:1011500008FB00BF4DF808EDFFF7EAFF34BF0120A0
:1011600000205DF808FB00BF4DF808EDFFF7E0FF39
:1011700094BF012000205DF808FB00BF4DF808ED8A
:10118000FFF7D2FF94BF012000205DF808FB00BFED
:101190004DF808EDFFF7C8FF34BF012000205DF8CF
:1011A00008FB00BF4FEA40024FEA41037FEA226C8E
:1011B00002D15FEA402C08D17FEA236C02D15FEABA
:1011C000412C02D14FF0000070474FF001007047F2
:1011D0004FEA4002B2F1FE4F0FD34FF09E03B3EB44
:1011E00012620DD94FEA002343F0004310F0004F84
:1011F00023FA02F018BF404270474FF000007047DA
:1012000012F1610F01D1420205D110F0004008BF78
:101210006FF0004070474FF00000704742000ED260
:10122000B2F1FE4F0BD34FF09E03B3EB126209D421
:101230004FEA002343F0004323FA02F070474FF0D7
:101240000000704712F1610F01D1420202D14FF04C
:10125000FF3070474FF00000704700BF10B5054CDD
:10126000237833B9044B13B10448AFF30080012352
:10127000237010BD0803002000000000C4CB00084C
:1012800008B5034B1BB103490348AFF3008008BD09
:10129000000000000C030020C4CB00080C22C0009A
:1012A00090FBF2F302FB130202B101330B22103068
:1012B00002FB03031846002BB8BFD81DC0105B0704
:1012C00018BF0130704700002DE9F047CB1D23F017
:1012D000070300AFADEB030DCD0006460C4691466B
:1012E00068460A4600210AF02FFD1E4AE8460123FF
:1012F0001146ADB232F8020FA8420ED3013B31F8CD
:1013000013C000210A46954209D82246414630467C
:101310000AF0B2FDBD46BDE8F0870133EAE7B1FB54
:10132000F5FA05FB1A1AB9F1000F19D1D646924603
:101330004FEADA03F35C0AF0070A43FA0AF34FEACA
:10134000DE0003F001030EF0070E03FA0EF318F8A7
:1013500000E0013243EA0E0308F800306144D2E7AE
:101360009646E5E700000020F0B54FF495460025CD
:101370000127C9008D4200DBF0BD4FEAE50C10F8F3
:101380000CE005F007044EFA04F386EA560202F078
:10139000010203F001035340A34007FA04F42EEACC
:1013A000040E43EA0E03920300F80C3042EA56069C
:1013B0000135DFE7B0F5006F0FDA70475B100342CD
:1013C000FCD01A46002BB8BF03F2FF72D2124A4378
:1013D0005040B0F5006FF2D270474FF4800340F6F2
:1013E0007541ECE72DE9F74F064610469246FFF7A8
:1013F00055FF42F22443002426F8023B5246804621
:1014000030468B46A1460AF037FD254623460C217F
:1014100006EB0A074FEACA02934239DBBAF1000F22
:10142000B8BF0022374B5A43374BB3EBB20F14D23D
:101430004FEA69000003FFF7BDFF0A220B3540FAAF
:1014400002F303F001032343AC1A14F0070414BFA2
:101450005C0007F8013B013AF1D215F0070308D010
:101460006D4205F0070558BF6B42C3F107039C406E
:101470003C70A8F10204002221463046FFF724FF09
:1014800030462146FFF770FF404603B0BDE8F08FBD
:101490006FEA030CD8101BF800000CF0070C40FAA0
:1014A0000CF0013300F0010049EA0000B3FBF1F950
:1014B00001FB1939B9F1000F02D04FEA4009ABE73F
:1014C000C002CDE90032FFF775FFDDE900324FF0D1
:1014D000010E0C21CEF10B0C40FA0CFC0CF0010CAF
:1014E0004CEA040C05EB0E0414F007040EF1010E97
:1014F00014BF4FEA4C0407F801CBBEF10C0FE9D141
:101500000B3589E7ABAAAAAA5555551538B54B1E18
:101510005C420D465C41072864D8DFE800F00426F1
:1015200036393C3F4D5B214616200AF0BFF9214673
:10153000C3200AF0BBF9214621200AF0B7F9214661
:1015400022200AF0B3F9214613200AF0AFF9214610
:1015500014200AF0ABF9214615200AF0A7F921461C
:101560001C200AF0A3F921460AE0214616200AF0C1
:101570009DF921461C200AF099F9691E18BF012126
:10158000BDE83840C2200AF091B92146C320EEE7F9
:1015900021462120EBE721462220E8E721461320BF
:1015A0000AF084F9691E18BF01211C200AF07EF997
:1015B0002146C2200AF07AF9214614200AF076F971
:1015C000691E18BF01211C200AF070F92146C220B3
:1015D0000AF06CF9214615200AF068F9691E18BF57
:1015E0000121BDE738BD006804F0A8BE04F06EBE5E
:1015F0002DE9F043A1B0E9460546884600244F4650
:1016000008EB0406B6B23046FFF7F0FF68B904F104
:1016100080030DEB030404F8800C3946284609F0DA
:1016200037FD284621B0BDE8F0833046FFF7DEFFE6
:10163000013409F8010BE3E7F7B507460E4600242D
:101640002146304609F008FE01783D19ADB229B9AE
:1016500001A80195FFF7C7FF03B0F0BD2146304652
:1016600009F0FAFD017801A801950134FFF7BBFFED
:10167000E6E738B50546FFF7B9FF0446681CFFF7F3
:10168000B5FF04EB0024A81CFFF7B0FF04EB0044F7
:10169000E81CFFF7ABFF04EB006038BD37B50D4623
:1016A00004460190C9B201A8FFF79DFF631CC5F372
:1016B000072101A80193FFF796FFA31CC5F307417B
:1016C00001A801930334FFF78EFF290E01A80194AE
:1016D000FFF789FF03B030BD38B50546FFF786FF39
:1016E0000446681CFFF782FF44EA002038BD70B54D
:1016F000CEB204460D46FFF779FF864203D031464D
:10170000204604F01BFE01342046FFF76FFFC5F3AF
:101710000725854205D029462046BDE8704004F0E3
:101720000DBE70BD2DE9F047054600274FF00008BB
:10173000DFF8A8904146284609F08EFD037846461A
:101740002E2B08F1010818D03146284609F084FDF7
:10175000037893B149463846FFF75EFB31460446AD
:10176000284609F079FD007800F00F00FFF700FB34
:101770002146FFF749FA0746DCE700240026DFF898
:101780005C9008EB060A5146284609F065FD03788F
:101790004BB9124DDEB921463846FFF735FAFEF750
:1017A0008DFEBDE8F08749462046FFF735FB5146E0
:1017B0000446284609F050FD0078013600F00F007D
:1017C000FFF7D6FA2146FFF71FFA0446D9E720466D
:1017D0002946FFF7D5FB013E0446DBE70000204128
:1017E00070B505460C460B4E002120200AF05EF82D
:1017F00045F080010022304604F0A6FB2146304629
:10180000002204F0A1FBBDE87040012120200AF075
:101810004DB800BFD00A002008B500210620FFF710
:10182000DFFF01210720FFF7DBFF7F210920FFF702
:10183000D7FF05210A20FFF7D3FFF4210B20FFF784
:10184000CFFFEF210C20FFF7CBFF00210D20FFF78A
:10185000C7FF00210E20FFF7C3FF80210F20FFF7F5
:10186000BFFF00211020FFF7BBFF20211220FFF750
:10187000B7FF00211320FFF7B3FF20217020FFF7EF
:10188000AFFF1D211C20FFF7ABFF40211D20FFF7FC
:10189000A7FFA1212020FFF7A3FF20212120FFF790
:1018A0009FFF4E212220FFF79BFFA5212320FFF75A
:1018B00097FF00212420FFF793FF0A212520FFF73F
:1018C0008FFF00212C20FFF78BFF00212D20FFF739
:1018D00087FF00212E20FFF783FF27216E20FFF7CF
:1018E0007FFF52216F20FFF77BFF8C213020FFF715
:1018F00077FFFF213220FFF773FF42213320FFF7EC
:101900006FFF40213420FFF76BFF20213520FFF7C8
:1019100067FF2D213620FFF763FFD4213720FFF723
:101920005FFF73213A20FFF75BFF6F213B20FFF73A
:1019300057FF6E213C20FFF753FF67213D20FFF743
:101940004FFF334B3E201978FFF74AFF73213F20AA
:10195000FFF746FF6F214020FFF742FF6E21412035
:10196000FFF73EFF67214220FFF73AFFFF214320A8
:10197000FFF736FFFF214420FFF732FFFF2145200C
:10198000FFF72EFFFF214620FFF72AFF01215620F7
:10199000FFF726FF07216D20FFF722FF00217920A6
:1019A000FFF71EFF00217A20FFF71AFF082172209F
:1019B000FFF716FF00217320FFF712FF00217420AC
:1019C000FFF70EFF21217520FFF70AFF182176206F
:1019D000FFF706FF0A217720FFF702FF7F215A2039
:1019E000FFF7FEFE40215920FFF7FAFE8021582024
:1019F000FFF7F6FE0B216A20FFF7F2FE04216820B4
:101A0000FFF7EEFEBDE8084003211F20FFF7E8BE08
:101A1000A00100204B210720FFF7E2BE4321072051
:101A2000FFF7DEBE40210720FFF7DABE002171205C
:101A3000FFF7D6BE38B504460B4D0021202009F033
:101A400035FF04F07F010022284604F07DFA0022D1
:101A50002846114604F078FA04460121202009F0B6
:101A600025FF204638BD00BFD00A0020000000003E
:101A70002DE9F047FEF722FD31A3D3E90023064606
:101A80000F46FEF773FD0022314B04460D46FEF76C
:101A9000F3FFB0F1000A18BF4FF0010A2D4B0022EE
:101AA00020462946FEF78CFEFFF738F85FFA8AF8E1
:101AB0004FFA8AFABAF1000F14BF6FF01703002330
:101AC00008F10109C4B2183C48461C44FEF7E4FC86
:101AD0001DA3D3E90023FEF749FD02460B4630461D
:101AE0003946FEF76DFE94FBF9F40646E0B20F4668
:101AF000FEF7D2FC02460B4630463946FEF77EFB27
:101B00000022154BFEF77AFB0022144BFEF72EFD48
:101B1000FFF704F804F01F0141EA481185B241F0D3
:101B200040017520FFF75CFE290A7620FFF758FE7A
:101B3000E9B27720BDE8F047FFF752BEAFF300806F
:101B4000622776622776F23F555555555555214007
:101B500000007E4000002440000038400040EF407C
:101B600000F007016D20FFF73BBE01467320FFF731
:101B700037BE03280DD8DFE800F00204080AFFF79B
:101B800055BF11217120FFF72BBE1221FAE7222148
:101B9000F8E70021F6E7000008B5A0B10B4B186884
:101BA0000130C0B2FFF7E1FF094B0A4A1B680A493E
:101BB000B3FBF2F3094A4868126853434A68121AA1
:101BC0009342FBDC08BD0120ECE700BF10020020BF
:101BD0009802002040420F00001000E01C0200208C
:101BE00038B50E4B0E4C18680130C0B2FFF7BDFF80
:101BF0000C4B65681868FFF7BBF80B4B1968FFF7CB
:101C00000BF9FFF7E5FA094B094A1B68B3FBF2F33E
:101C1000584363685B1B9842FBDC38BD1002002010
:101C2000001000E01C020020140200209802002096
:101C300040420F0070B505460020FFF7ADFF0024BD
:101C4000074E3368A34203DCBDE87040FFF7C8BF0E
:101C500045FA04F000F00100FFF79EFF0134F0E7C1
:101C60001802002010B504460120FFF795FF6420FC
:101C700009F05CFE013C14F8010F00B910BDFFF73C
:101C8000D9FFF8E7022808B516D0032816D0012896
:101C900014BF01200220FFF768FF094B094A1B68A7
:101CA0000949B3FBF2F3094A4868126853434A688A
:101CB000121A9342FBDC08BD0320ECE70420EAE79C
:101CC0009802002040420F00001000E03003002086
:101CD0000020FFF7D7BF38B504460425A009FFF759
:101CE000D1FFA400013DE4B2F8D1012038BD38B5E0
:101CF00005460024A54200DC38BD1B20FFF7EBFFA2
:101D00000134F7E770B5044600254618B44201D106
:101D1000284670BD14F8010BFFF7DDFF0544F5E719
:101D2000082341F2210280EA012000F40041400032
:101D300001B15040013BF8D1704738B50446451811
:101D40004FF6FF70AC4200D138BD14F8011BFFF70D
:101D5000E7FFF7E7024630B5014441F221054FF6AF
:101D6000FF708A4200D130BD082412F8013B80EA9E
:101D7000032003B2002BB4BF85EA4303430098B2AB
:101D8000631E13F0FF04F4D1EBE700000F4B10B516
:101D90001B78C5200E4C83B109F076FCFEF7E4FFFA
:101DA0000C49FFF7EDF80C49FFF736F80146FEF74E
:101DB0002BFF2168FFF730F810BD09F065FCFEF736
:101DC000D3FF4FF06A51FFF727F8ECE7450B0020EF
:101DD0009C01002000F07F45000040400000000012
:101DE00008B5C92009F050FC314B1B78002B3FD0BF
:101DF000FEF752FB22A3D3E90023FEF7B7FBFEF761
:101E0000ADFEFEF75BFB02460B4600202949FEF7BC
:101E1000D7FC0022284BFEF7F1F91BA3D3E90023DE
:101E2000FEF7A4FBFEF79AFE01462448FFF7A8F848
:101E30000AF0F2FBFEF742FB15A3D3E90023FEF7FD
:101E400095FB15A3D3E90023FEF7DAF902460B460A
:101E500000201949FEF7B4FCFEF780FEFEF72EFBCA
:101E60000FA3D3E90023FEF7C9F9FEF777FE08BDFB
:101E7000FEF712FB0CA3D3E90023BEE7AFF300800B
:101E8000188001188001483F000000000050C44045
:101E90007DB968C570842E3F83DBB5DCE1796B3F8B
:101EA0006666666666127140061860800106683FC5
:101EB000450B0020000008400000F03F0080224653
:101EC00010B51120FFF7B6FD044680210F20FFF763
:101ED00087FC60104038C0B210BD00210F2009F00F
:101EE000E5BC01210F2009F0E1BC000008B51E4B44
:101EF0001860032837D8DFE800F0021C2E340121D7
:101F00001C2009F0D3FC0121C22009F0CFFC174BA3
:101F10001B782BB10021BDE80840002009F0C6BCA9
:101F2000134B1B78FBB10121BDE808400C20FFF7E3
:101F300057BC01211C2009F0B9FC0021C22009F086
:101F4000B5FC0A4B1B780BB10121E4E7084B1B7869
:101F50004BB10021E8E700211C2009F0A7FC01217A
:101F6000ECE70021E6E708BD9C070020450B0020B8
:101F700070020020000000002DE9F84F0121064604
:101F8000FFF7C4FAFA2009F0D1FC09F0CDFC0446B1
:101F9000DFF8CC80334DD8F808309A072DD4314F74
:101FA000D8F8085015F0020537D009F0BDFC47F20B
:101FB000305705464FF00009DFF8A8A0D8F80830E0
:101FC0009B0734D4D8F8083013F0020B39D0013F06
:101FD000F4D109F0A9FC044639463046FFF796FAD9
:101FE000601B61EB0101FEF78BFA1BA3D3E9002311
:101FF000FEF7E6FBFEF7B2FD0DE009F095FC0023CD
:10200000001B62EB020285429341C4D2304600219C
:10201000FFF77CFA1448BDE8F88F09F085FC001B37
:1020200063EB0303874275EB0303B9D2EEE709F0D4
:102030007BFC001B63EB0303824579EB0303BDD2FA
:10204000E4E709F071FC074A001B63EB03038242DB
:102050007BEB0303B6D2D9E700000000004CDD4063
:102060000008014080841E00000080BF10B5FFF70B
:1020700083FF00210446FFF78BF820B12146034877
:10208000FEF77EFF10BD0020FCE700BF002474496E
:1020900070B50120FFF7EAFF002104460846FFF76C
:1020A00035FA0220FFF7E2FF002106460846FFF757
:1020B0002DFA2046FEF702FA00220C4BFEF756FAE4
:1020C000044630460D46FEF7F9F90022084BFEF7AC
:1020D0004DFA02460B4620462946FEF791F80022AB
:1020E000044BFEF743FAFEF739FD70BD00708740E0
:1020F00000908F400000E03F7A4B2DE9F0471B78BD
:10210000002B00F0ED800020FFF7F0FEFFF7C0FF8E
:10211000754D764F28600420FFF7A8FF744B00210F
:1021200018600446FFF720F800286AD001233B70AE
:1021300000210846FFF7EAF90320FFF797FF6D4BF0
:10214000002118600446FFF70FF86B4EDFF8AC81F2
:1021500000286AD00123337000210846FFF7D6F922
:102160000520FFF783FF664B01461860654BD8F8E2
:1021700000A01D682846FEF745FD634B044619681C
:102180002846FEF73FFD01462046FEF7F9FEFEF722
:1021900095F900225D4BFEF7E9F9FEF797FCFEF793
:1021A0007BF9044650460D46FEF788F90022584B4D
:1021B000FEF706FB02460B4600200021FEF71EF844
:1021C00002460B4620462946FEF71AF8FEF77EFC2B
:1021D000504904465046FEF7BDFF4F4D002838D108
:1021E0002C602B68692B73DD65232B603B7803B96A
:1021F00033780021BDE8F047484A08461370FFF7DE
:1022000085B9214638702868FEF7BAFE444B454927
:102210001860FEF7F7FC4449FEF7B2FE434B19681D
:10222000FEF7F2FC424B186082E7214630702868C6
:10223000FEF7A6FE3F4B3B491860FEF7E3FC3A4928
:10224000FEF79EFE3C4B1968FEF7DEFCC8F8000066
:1022500082E751462F48FEF7D5FCFEF72FF9002202
:10226000364BFEF7ADFA0022354BFDF7C9FF80462D
:1022700020468946FEF710F902460B46404649467D
:10228000FEF774F9FEF722FC2E4904465046FEF78D
:1022900061FF0028A4D051462A48FEF7B3FCFEF7A0
:1022A0000DF90022284BFEF78BFA0022244BFDF794
:1022B000A7FF804620468946FEF7EEF802460B4609
:1022C00040464946FEF752F9FEF700FC286088E7D1
:1022D000642B01DD642388E7002B87DA002384E781
:1022E000BDE8F087DC010020A8070020A707002038
:1022F000D4070020C8070020A6070020C007002040
:10230000BC070020B8070020B40700200000594097
:1023100000001A400000A0C1B0070020A50700205F
:10232000D007002000007A4466667640D80100207D
:10233000CC070020C4070020D401002000806640A4
:102340000000F03F000020C200806B40F8B509F0AB
:10235000E9FA104F104E3B68104DC01AFEF78CF88A
:1023600000220F4BFEF72CFAFEF7F8FB0021044683
:10237000FEF70EFF40B129683068FEF743FC2146A6
:10238000FEF7FEFD074B186009F0CCFA33683860A1
:102390002B60F8BD9401002024080020FC070020D9
:1023A00000408F40F807002038B5214C0A217320E7
:1023B000FFF716FA1F4A23681F4DB3FBF2F3C4223E
:1023C000534369686A68521A9342FBDC0021732008
:1023D000FFF706FA174A23686968B3FBF2F3C422D1
:1023E0005343154D6A68521A9342FBDC0A2173204D
:1023F000FFF7F6F90F4A23686968B3FBF2F3C422CA
:1024000053430D4D6A68521A9342FBDC002173203E
:10241000FFF7E6F9074A23686968B3FBF2F3C422C1
:10242000534305484268521A9342FBDC38BD00BF53
:102430009802002040420F00001000E038B5124D15
:102440000A217320FFF7CCF9104A2B68104CB3FB1C
:10245000F2F34FF4C372534361686268521A9342B5
:10246000FBDC00217320FFF7BBF9084A2B68616889
:10247000B3FBF2F34FF4C372534305484268521A58
:102480009342FBDC38BD00BF9802002040420F00A1
:10249000001000E008B1FFF7D1BFFFF785BF0000D3
:1024A000064B1A88504040F3000020F4F74020F01B
:1024B000770080EA52001880704700BF8C0100202E
:1024C0002DE9F843044688460827164D164E04F0B9
:1024D00001094846FFF7E4FF2878B9F1000F18D04A
:1024E000FFF7D8FF33780133DBB23370B8F1000F58
:1024F00009D0052B07D1287880F001002870FFF75C
:10250000C9FF00233370013F4FEA5404DFD1BDE817
:10251000F88380F001002870FFF7BCFF86F8009078
:10252000F1E700BF9B070020D8050020074B10B53E
:102530001C880121E043C0B2FFF7C2FF6FEA1420FC
:10254000BDE810400121C0B2FFF7BABF8C010020E6
:1025500070B53C48FDF746FE00250446394EAC42B6
:1025600043DC062C09D00025C4F1060401214020DB
:102570000135FFF7A5FFA542F8D10025324E012114
:102580006020FFF79DFF347AAC4238DC052C4BD934
:102590002E4B0121187800253030400000F0FE005D
:1025A000FFF78EFF2A48FDF71DFE0446284EAC4279
:1025B0003EDC0025C4F10604012140200135FFF76F
:1025C0007FFFAC42F8D1234B0121187840006130E5
:1025D000C0B2FFF775FF01210320FFF771FFBDE8CF
:1025E00070400121F020FFF76BBF16F8010B0121AD
:1025F000400000F0FE00FFF763FF0135AFE729461A
:10260000304608F029FE00780121400000F0FE006D
:10261000FFF756FF0135B7E701214020FFF750FFD4
:102620000135AC42F8DCB3E70025C4F10604F8E755
:1026300016F8010B0121400000F0FE00FFF740FFFB
:102640000135B4E7350200208C0800203C02002050
:102650002F0200202E02002070B506460D460024F1
:10266000AC4200DB70BD305D0121FFF729FF013472
:10267000F6E7000010B504461349144809F0F4FBCE
:10268000012C0CD11248FDF7ADFD01461048FFF7B3
:10269000E3FF1048FDF7A6FD01460E4806E0022CB8
:1026A00008D10D48FDF79EFD01460B48BDE81040DE
:1026B000FFF7D2BF032C05D10848FDF793FD014673
:1026C0000648E4E710BD00BF30CC0008350200200A
:1026D00069070020A1060020D905002082070020FC
:1026E00038B505460024A54200DC38BD00217E2017
:1026F000FFF7E6FE0134F6E738B500250021044671
:102700007220FFF76DF80B4B64201D70FFF7E8FF98
:102710004FF6FF72084B1A80084B1D70FFF718FF29
:102720002046FFF7A7FFFFF701FFBDE83840032071
:10273000FFF7D6BF9B0700208C010020D8050020A2
:10274000F0B50028114CD8BF4042B0FBF4F6104F52
:102750000E8007FB06004FF03C0606FB00F090FBE6
:10276000F4F4E4B2147004EB8402C4EBC20442F249
:10277000107290FBF2F0D4BF0025012500EB84001D
:10278000187015B90B885B420B80F0BD40420F00FA
:10279000C0BDF0FF2DE9F04F0D4691B07A49099286
:1027A0000D90FEF739FBFEF713FD0DF13A030EAA6B
:1027B0000FA9FFF7C5FF74492846FEF72DFBFEF76A
:1027C00007FD0DF13B030DF139020DF13E01FFF75D
:1027D000B7FF0A22BDF93C309DF83860002BB8BF26
:1027E0005B429BB2B3FBF2F102FB11335FFA83FA57
:1027F000B6FBF2F35FFA81F902FB136603F13001D5
:102800009DF83A30C9B20A91B3FBF2F102FB1133E1
:102810005FFA83FB0BF13003DBB20893BDF93E3066
:102820005A4A002BB8BF5B421268DCB29DF83B30BD
:1028300010465FFA81F856490B930792FEF7A0FB0A
:10284000FEF7ECFCC0B21428079A8CBF1C306C3029
:10285000C3B210460793FEF7BBFC0A2290FBF2F1CD
:1028600001FB120000EB800040002030C3B209F1F0
:1028700050090AF1500A00210D989DF83970F6B2FE
:102880000C935FFA89F95FFA8AFAFEF781FC002857
:1028900064D13036A4F10A02592AF6B264D908F19B
:1028A0005008002128465FFA88F8FEF771FC0028DE
:1028B00065D10BF15002D3B2632C089350D96D2C23
:1028C00094BF0834483C334B092F186894BF5837DD
:1028D0001C37FEF77DFC42F2590300F51C551035FC
:1028E000B5FBF3FB03FB1B55089B4A46CDE902836E
:1028F0000A9B2949009301965346284809F0EAF9B2
:10290000274BE4B21B78FFB20593264B22461B7877
:10291000254904931C2303930C9B09980293079B5E
:1029200001930B9B1C33DBB200933B4609F0D2F9B9
:102930005B21B5FBF1F201FB12552132D2B20092BC
:102940002135099A0BF12103EDB210461749019583
:10295000DBB209F0BFF911B0BDE8F08F503699E74E
:10296000092C0ED91C34AEE708F1300800212846A6
:102970005FFA88F8FEF70CFC0028F3D199E7632C86
:102980009DD876349FE700BF0024744920080020BA
:1029900000002041240800203CCC00083502002023
:1029A0002C0200202D02002037CC000849CC000862
:1029B00070B506468AB00C462B491546FEF72CFA30
:1029C000FEF706FC0DF1090302AA03A9FFF7B8FE02
:1029D00000213046FEF7D2FB002814BF4E235323BC
:1029E000BDF90C200193002A9DF80930B8BF52426E
:1029F00092B200931D499DF8083004A809F06AF9C5
:102A000019492046FEF708FAFEF7E2FB0DF10B0329
:102A10000DF10A020DF10E01FFF792FE0021204692
:102A2000FEF7ACFB002814BF45235723BDF90E2049
:102A30000193002A9DF80B30B8BF524207AC0093B7
:102A400020469DF80A300A4992B209F043F9094B31
:102A500028461B780849CDE90043084B04AA1B7897
:102A600009F038F90AB070BD0024744953CC00084D
:102A700063CC00082D02002073CC00082C0200203B
:102A800008B50021182008F011FFBDE80840012119
:102A9000172008F00BBF08B5FFF7F2FFFEF7C2FFE3
:102AA00040F6B83008F042FFBDE8084001210C2094
:102AB00008F0FCBE10B5FFF769F9174B1C682146FA
:102AC000FEF748FB40B100212046FEF739FB18B95C
:102AD000FEF7A8FFFFF7DFFF104B1868421C19D064
:102AE0000F4B1C68FEF744F90E4B1968FEF732FBDA
:102AF00040B1631C0ED00C4BE0B21C60BDE810402E
:102B0000FFF72EB8013405D0084B1868064B186043
:102B1000C0B2F3E710BD00BF64080020FC01002034
:102B20006002002024080020000800206402002029
:102B300008B50121182008F0B9FEBDE808400021C1
:102B4000172008F0B3BE08B50021182008F0AEFE2B
:102B5000BDE808400021172008F0A8BE08B50121F3
:102B6000182008F0A3FEBDE808400121172008F056
:102B70009DBE00002DE9F84F00234FF0010BDFF858
:102B80002091DFF82081484C484E494D494F89F843
:102B9000003088F80030237033702B7087F800B055
:102BA000FFF7F4F8444B824601461868FEF7F0FA46
:102BB00060B389F800B0414B1A68414B1B689A42D8
:102BC00003DA404B1B685BBB23703F4B3F4A1978CD
:102BD0003F4B18783F4B28B329B3012111700021D6
:102BE000197099F8001009B912781AB301233370DB
:102BF00000232C783B705CBBC823374A1360374BEB
:102C00001B7863BBBDE8F84FFFF7A8BF344B5146B4
:102C10001868FEF7BDFA0028CDD088F800B0CAE7E2
:102C20000123D1E721B10021197001211170D8E7EA
:102C30001970FBE798F8002032B9227822B91B7886
:102C400013B9284B1B7833B101232B7000233B7041
:102C500000246423D1E701242B703C70CDE7224B84
:102C60001868FEF785F8214B1968FEF773FAB0FA79
:102C700080F01F4B4009187080B133781BB1BDE85C
:102C8000F84FFFF7FDBE2B781BB1BDE8F84FFFF7FB
:102C90005ABF1CB1BDE8F84FFFF74ABFBDE8F88F37
:102CA0000C0800200B0800200A0800200E08002055
:102CB0000D08002098010020680800201808002056
:102CC000F8010020E4010020A607002008080020E9
:102CD000A707002009080020100800200402002097
:102CE0006C080020A4070020000200202408002017
:102CF0005008002010B50424FFF725FF7D2008F0C0
:102D000015FEFFF72BFF7D2008F010FE013CF3D1EC
:102D1000FFF7B6FE21460F2008F0C8FD40F6B83098
:102D200008F004FE01210F2008F0C0FDFFF700FFAE
:102D3000322008F0FBFDFFF711FF322008F0F6FD0E
:102D4000FFF701FF024A13680133136010BD00BF93
:102D5000DC07002008B50B4B1B788BB108F0E2FDB7
:102D6000094B98420CD9BFF34F8F0849084BCA68EA
:102D700002F4E0621343CB60BFF34F8F00BFFDE767
:102D800008BD00BFA8010020FF07194800ED00E0C2
:102D90000400FA0510B5FFF793F80446FFF720F892
:102DA000FEF716FA782C0ADC80EAE073A3EBE073F6
:102DB000782BCFBF2046001900EBD070401010BD1B
:102DC000F0B50446A9B0854907A808F061F9834920
:102DD000204608F05DF9824A804913680AA8013349
:102DE000136008F055F97F4B7F4A1B687F490093B9
:102DF0007F4B12681B6803A808F06CFF002706468B
:102E000003ADB742C0F2D6807A4B052219680DA8EF
:102E100008F0C4F9784B0522196810A808F0BEF92B
:102E2000764B1B7823B9764B1B78002B40F0C9807A
:102E3000FFF7B0FF0246734905A808F04BFF67494A
:102E4000064613A808F024F9002705ADB742C0F2E2
:102E5000BD806D4B1868FEF7E1F96C49064616A86F
:102E600008F055F916A919A808F051F9684919A8E8
:102E700008F0DEF905465A4B0A2219681CA808F02A
:102E80007BF91CA9284608F0C7F9614908F0D0F978
:102E90000AA908F0C1F95E4908F0CAF90DA908F0BD
:102EA000BBF95B4908F0C4F910A908F0B5F9584915
:102EB00008F0BEF905460A2231461FA808F04AF973
:102EC0001FA9284608F0A8F9514908F0B1F90546AC
:102ED000504B0A22196822A808F03CF922A928467A
:102EE00008F09AF94A4908F0A3F90546FEF74EFFA3
:102EF0000222014625A808F051F925A9284608F024
:102F00008BF9434908F094F913A908F085F90146B3
:102F100007A808F0EDF825A808F078F822A808F02E
:102F200075F81FA808F072F81CA808F06FF819A827
:102F300008F06CF816A808F069F809990798FEF7E8
:102F400009FF354A034605211FA808F08FFE3349C3
:102F500022A808F09DF807A922A808F05DF93049D9
:102F600008F066F905461FA925A808F091F825A9DB
:102F7000284608F051F92B4908F05AF90146204635
:102F800008F0B6F825A808F041F822A808F03EF8A5
:102F900013A808F03BF810A808F038F80DA808F0BE
:102FA00035F80AA808F032F807A808F02FF82046EC
:102FB00029B0F0BD15F8011B0AA808F020F9013767
:102FC0001FE7194B1868FEF703F933E715F8011BE3
:102FD00013A808F014F9013738E700BF68D50008D6
:102FE000E007002028080020300800207DCC0008E1
:102FF0002C080020600800205C0800200908002040
:10300000DC0100208CCC000824080020740800207B
:103010008FCC00081808002091CC000896CC00083E
:103020009BCC000867D50008CC0700201FB5144BC7
:103030001B7813B3134B1B78FBB1134C01A8FFF79C
:10304000BFFE01A9204608F06CF801A807F0DEFFDA
:103050002468FEF7EBFC0D4B1868FEF709FD08F03D
:1030600061FC0B4B1860FEF7D5FC2046FEF7FAFD1D
:1030700004B0BDE81040FEF7D5BC04B010BD00BFE1
:10308000240200205D0200204408002020020020CD
:10309000F007002030B53E4A8BB013680446013378
:1030A0001360ADF80A303B4B3B4A1B6812688DF841
:1030B0000C303A4BADF808201B680AAD8DF80D3086
:1030C000374B1B688DF80E30364B1B68CDF80F3030
:1030D000354B1B68CDF81330344B1868FEF79EF85B
:1030E000334BADF817001868FEF798F88DF8190003
:1030F000FEF74CFE2F49FDF78FFEFEF769F8FF2320
:10310000009300234FF4FA72194607F075FF2A4B1B
:103110008DF81C001B688DF81A30FFF73BFE274B1B
:1031200024498DF81B001868FDF776FEFEF750F86D
:10313000234B2449ADF81D001868FDF76DFEFEF71E
:1031400047F8214B1F491B68ADF81F008DF821304F
:103150001E4B1868FDF760FEFEF760F81C4BADF8DB
:1031600022001B681E2102A8ADF82430FEF7E5FD01
:103170002346ADF8260002AA144603CCAC421860E0
:103180005960224603F10803F6D120200BB030BD70
:1031900004080020300800204C0200202C080020E9
:1031A00028080020600800205C0800202408002077
:1031B0001C0800200000C84218080020F807002062
:1031C000CC07002000002041B0070020AC07002001
:1031D00010080020000000001D4B10B51B788BB3B9
:1031E0001C4B1B7873B31C48FFF754FF1A49024667
:1031F0001A48FEF7F7F80446FEF718FC184B186853
:10320000FDF75CF910A3D3E90023FCF7F9FFFDF704
:10321000A5FCFEF72DFC08F085FB124B1860FEF7AD
:10322000F9FBFEF755FD40F2EE2008F07FFB082089
:10323000FEF75DFD21460948FEF764FDBDE810403C
:10324000FEF7F0BB10BD00BF2D431CEBE2364A3F3A
:10325000540200205D020020B4030020340300204B
:1032600050020020F00700202DE9F041264B86B0E7
:103270001E680546FEF78AFD244B07461B7813B9E6
:10328000234B1B7863BBFFF785FD224B0446D3F825
:103290000080214B30461B783BB3FDF70FF918A394
:1032A000D3E90023FDF762F9FDF710FC1B49064640
:1032B0003846CDF81080FDF7AFFDFDF789FFCDE969
:1032C0000240174BC8211B6828460193154B164A2C
:1032D0001B680093334608F0C9FC06B0BDE8F081D6
:1032E000124B1868FDF774FFCFE7FDF771FFC82197
:1032F00003460F4A2846CDF8008008F0B7FCECE7FB
:10330000E544BB0A293F0A402408002009080020A0
:10331000DC010020800800209808002000007A448A
:1033200018080020D40500209DCC0008CC07002000
:10333000BCCC00082DE9F04F064695B00C464A4932
:103340001546FDF769FDFDF743FF0DF131030CAAAA
:103350000DA9FFF7F5F900213046FDF70FFF002812
:1033600014BF4E23532301939DF83130BDF934200F
:103370003E4900930EA89DF8303008F0ABFC3A4966
:103380002046FDF749FDFDF723FF0DF133030DF155
:1033900032020DF13601FFF7D3F900212046FDF787
:1033A000EDFE002814BF4523572301939DF83330C9
:1033B0000DF14409BDF936202D49009348469DF88A
:1033C000323008F087FC2B4BDFF8ACB0D3F800A00C
:1033D0005046FDF773F80022284BFDF7C7F800228E
:1033E000274BFDF7EDF90022264BFCF709FFFDF70F
:1033F0006DFBDBF800400646632C32DC002C08BF76
:103400000124214B21491868FDF706FDFDF7E0FE78
:103410000746FFF7BFFCDBF800B08046FEF7B6FCBE
:103420001B4B1C491B680B93FDF7F6FCFDF7D0FE08
:10343000CDE909B05046CDF82080FDF7C9FE002344
:10344000CDE90670CDE90233CDE90093C8212846C5
:10345000CDE90464104A0EAB08F008FC15B0BDE8D5
:10346000F08F0024CDE700BF0024744953CC00083E
:1034700063CC0008CC070020B007002000002240E9
:103480000000144000004040AC0700200000204134
:103490008008002000007A44C8CC0008000000002A
:1034A00038B5314B1B78002B56D0304B1B78002B96
:1034B00052D00220FEF75DFB2D4B2E4D1868FCF715
:1034C000FDFF27A3D3E90023FCF798FEFDF746FB99
:1034D000FEF7CEFA08F026FA274B284918602B6829
:1034E0002748032B29D1274A09680068FFF752F9BA
:1034F000254A8024136801331360FEF78BFAFEF728
:103500009DFF013CFBD12878FFF7F6F8FEF78AFA19
:103510001E4B1B7803B3FEF77DFA41F28834FEF7A9
:1035200043FF013CFBD141F28834FEF787FF013CA9
:10353000FBD1BDE83840FEF775BA022B0068096878
:1035400003D1134AFFF7F6FED2E7124AFFF730FA2B
:103550001148FFF789FECBE738BD00BFAFF300800D
:10356000FA7E6ABC7493583F450200205D02002039
:103570004002002028020020F00700205C08002004
:103580006008002082070020D40500205808002091
:10359000D905002069070020A10600202DE9F04F81
:1035A000DFF83CC19FB00DF1280E16461F460546B8
:1035B000BCE80F00AEE80F00BCE80F00AEE80F005B
:1035C0009CE803000CF1080C8EE80300BCE80F0037
:1035D0000DF1500EAEE80F002A9CBCE80F00AEE8DB
:1035E0000F009CE8030000228EE80300DDE92801BB
:1035F0003C4BFCF705FE3C4BCDE900010022304678
:103600003946FCF7FDFD631E0A2B28BF062406463B
:1036100063100F460024DFF8D4A009930DF1280BA6
:10362000099B9C420AD100233049284601F81430F6
:1036300007F02EFD28461FB0BDE8F08FFBE80223FF
:10364000DDE90001CDE90223FDF7BAF814AB03EB85
:10365000C403D3E900238046894630463946CDE984
:103660000423FDF7ADF8E307CDE906012AD50022D2
:103670001F4B40464946FCF7C3FDFDF74FFA0022B9
:103680001B4B5FFA80F8DDE90601FCF7B9FDFDF799
:1036900045FADDE90223C0B28AF801008AF8008009
:1036A000DDE9000108F08CFFDDE90423CDE900012C
:1036B0003046394608F084FF013406460F460AF1C9
:1036C000020AADE740464946FDF700FA00F141081D
:1036D000DDE90601FDF7FAF95FFA88F84130D8E72D
:1036E000E0CB0008008066400080564024030020A4
:1036F000000048402DE9F0472C4990B0044607F0FF
:10370000C7FC2B4BDFF8ACA01868FDF787FD2A49F2
:10371000064607A807F0BCFC284904A807F0F7FCF8
:1037200004A907A807F078FD514607F081FD244B56
:1037300005460A271868FCF7C1FE224B029780460F
:1037400018688946FCF7BAFE4B464246CDE90001AF
:103750000AA8FFF723FF0AA9284607F05DFD514696
:1037600007F066FD184907F063FD05463A46314605
:103770000DA807F0EFFC0DA9284607F04DFD1349F1
:1037800007F056FD0146204607F0B2FC0DA807F0F1
:103790003DFC0AA807F03AFC04A807F037FC07A88C
:1037A00007F034FC204610B0BDE8F08768D500086B
:1037B0002408002019CD000818CD00087408002046
:1037C000600800205C0800201BCD000820CD000808
:1037D0001FB50021084602F0B1FD514B514C18684D
:1037E000FCF76CFE4CA3D3E90023FCF7BFFEFDF70A
:1037F00095F901460620FDF751FF4B4B1868FCF781
:103800005DFE45A3D3E90023FCF7B0FEFDF786F982
:1038100001460220FDF742FF444B1868FCF74EFEBC
:103820003DA3D3E90023FCF7A1FEFDF777F901469C
:103830000A20FDF733FF3E4B1868FCF73FFE36A326
:10384000D3E90023FCF792FEFDF768F901461B203F
:10385000FDF724FF374B0E20197802F06FFD364B31
:1038600036491868FDF7D8FAFDF7D8FCC1B20F2029
:1038700002F064FD324B10201968FDF738FF314B20
:103880001220197802F05AFD2F4B13201968FDF70A
:103890002EFF2E4B15201968FDF729FF2C4B172002
:1038A000197802F04BFD2B4B1820197802F046FDD9
:1038B000294B1920197802F041FD284B1F20197857
:1038C00002F03CFD0721302002F038FD3C21202091
:1038D000FDF70DFF4FF416512C20FDF7DFFE2146BA
:1038E00001A807F0D5FB01A93220FDF7A5FE01A82C
:1038F00007F08CFB214601A807F0CAFB01A93C2078
:10390000FDF79AFE01A807F081FB0021502004B0CA
:10391000BDE8104002F012BD0000000080842E417E
:103920005002002023CD0008400200202002002089
:103930000C02002018020020140200200000204188
:103940001C020020100200204C020020480200202F
:103950003C0200202D0200202C0200200802002042
:103960001FB50620FDF785FE013001D1FFF730FFBE
:103970000620FDF77EFEFDF7F7F96149FDF700FB34
:10398000604B614C18600A20FDF773FEFDF7ECF9FF
:103990005B49FDF7F5FA5D4B18600220FDF769FE03
:1039A000FDF7E2F95649FDF7EBFA594B18601B2079
:1039B000FDF75FFEFDF7D8F95149FDF7E1FA554BE8
:1039C00018601320FDF788FE534B18601520FDF793
:1039D00083FE524B18600E2002F078FC504B1860AA
:1039E0000F2002F073FCFCF757FD00224D4BFCF753
:1039F000E7FEFDF7B3F84C4B18601020FDF76CFEA6
:103A00004A4B1860122002F061FC494B18601720E5
:103A100002F05CFC474B1870182002F057FC464B34
:103A20001870192002F052FC444B18701A2002F052
:103A30004DFC20601F2002F049FC414B1860202003
:103A4000FDF74AFE4FF47A7358433E4BA0F5DA5027
:103A500018381860302002F039FC3B4B1860002009
:103A600002F034FC394B00F001021870384B10F0B2
:103A7000100F1A70374BC0F340021A70364BC0F368
:103A800080021A70354BC0F3C0021A700CBF0123BC
:103A900002232360324BC0F340121A70314BC0F343
:103AA00080121A70304BC009187008B103232360CC
:103AB00001A83221FDF79CFD01A92C4807F031FB3C
:103AC00001A807F0A3FA01A83C21FDF791FD01A987
:103AD000274807F026FB01A807F098FA01A8502113
:103AE000FDF786FD01A9234807F01BFB01A807F09D
:103AF0008DFA2C20FDF7BDFD1F4B186004B010BDE2
:103B000000247449500200202802002020020020D6
:103B1000400200200C0200204C020020480200203D
:103B20001802002000002440140200201C02002083
:103B3000100200203C0200202D0200202C02002058
:103B400008020020580200206802002034040020EF
:103B500054020020240200204502002071080020A9
:103B60007008002098080020440200208C080020E3
:103B700074080020800800208801002037B5252423
:103B80001D4802F0E1FB00941D231E221F211B484B
:103B900002F036F91A4D2346009409220A211948E9
:103BA00006F0E8FE23461A2200941B21164C174803
:103BB00006F0E0FE2946164807F06AFA2146154845
:103BC00007F066FA2946144807F062FA134B2146BB
:103BD0001A78134B13481A7007F05AFA2146124804
:103BE00007F056FA114B1A68114B1A60114B1A68FC
:103BF000114B1A6003B030BD480B0020D00A0020E2
:103C000023CD0008B809002068D50008A0080020CE
:103C10008C08002080080020740800200402002086
:103C200050080020440800203808002064020020CA
:103C3000000800209C080020D005002008B5084896
:103C400007F0E4F9074807F0E1F9074807F0DEF963
:103C5000064807F0DBF9BDE80840054807F0D6B98B
:103C60003808002044080020740800208008002044
:103C70008C080020000000002DE9FF410024884E40
:103C8000FD2C23D0304606F06EFD0028FADD844876
:103C900007F006F8834DC1B20A2929557CD0804827
:103CA00007F039F82B5D082B08BF023C2B5D0D2B6C
:103CB00072D1002364202B5507F038FE784806F0B7
:103CC00052FD002802DD764806F0EAFF7549764885
:103CD00000220C46064611F8013B202B06D03D2B56
:103CE00004D01BB10D2B01D0182A57D10021B1549B
:103CF000002B62D16D496C4808F02EF800287DD168
:103D00006B4901A807F0C4F901A8FDF70BFDFCF70A
:103D100025FF684C206001A807F078F925686649FE
:103D20002846FDF735FA20B128466449FDF728F901
:103D30002060256861492846FDF72AFA20B1284607
:103D40005E49FDF71DF9206025685D492846FDF7AD
:103D50001FFA002849D028465A49FDF7FBF90028E8
:103D600043D059494E4806F0F5FF58494C4806F0F3
:103D7000CEFF2068FCF7A2FB47A3D3E90023FCF7A2
:103D8000F5FBFCF7CBFE01460620FDF787FC04B0EF
:103D9000BDE8F041FFF7E4BD013471E7A3F161052F
:103DA000192D9CBF03F05F0301F8013C11F8013CA1
:103DB000013200F8013B8EE70132A15CA3182029F3
:103DC000FAD03D29F8D03A481A460446002312F8A2
:103DD000011B19B10D2901D0132B02D10022E2548D
:103DE00088E700F8011B0133F1E739492C4806F058
:103DF000B1FF36492A4806F08AFFC8E735492A4804
:103E000007F0AAFF002869D1294901A807F040F965
:103E100001A8FDF787FCFCF7A1FE2F4C206001A84C
:103E200007F0F4F8256824492846FDF7B1F920B1D8
:103E300028462249FDF7A4F8206025681F49284636
:103E4000FDF7A6F920B128461C49FDF799F8206036
:103E500025681B492846FDF79BF90028C5D0284650
:103E60001849FDF777F90028BFD017490C4806F02C
:103E700071FF16490A4806F04AFF2068FCF71EFB4E
:103E800005A3D3E90023FCF771FBFCF747FE0146CD
:103E900002207AE7AFF300800000000080842E410A
:103EA000A0080020CE0400203504002044CD0008E6
:103EB0004E040020500200200024744900007A447F
:103EC0000000D7430000DC434DCD000851CD000871
:103ED00053CD00086BCD0008400200209E499F484A
:103EE00007F03AFF002847D19D4901A807F0D0F814
:103EF00001A8FDF717FCFCF731FE9A4C206001A8E1
:103F000007F084F8256898492846FDF741F920B163
:103F100028469649FDF734F82060256893492846DD
:103F2000FDF736F920B128469049FDF729F82060C1
:103F300025688F492846FDF72BF900283FF455AF37
:103F400028468C49FDF706F900283FF44EAF8A4910
:103F50008A4806F0FFFE8A49884806F0D8FE2068A5
:103F6000FCF7ACFA7AA3D3E90023FCF7FFFAFCF7DD
:103F7000D5FD01460A2008E78249784807F0ECFEA3
:103F8000002847D1764901A807F082F801A8FDF77B
:103F9000C9FBFCF7E3FD7C4C206001A807F036F874
:103FA000256871492846FDF7F3F820B128466F4986
:103FB000FCF7E6FF206025686C492846FDF7E8F825
:103FC00020B128466949FCF7DBFF20602568684975
:103FD0002846FDF7DDF800283FF407AF284665497D
:103FE000FDF7B8F800283FF400AF6349634806F0D6
:103FF000B1FE6349614806F08AFE2068FCF75EFA6C
:1040000053A3D3E90023FCF7B1FAFCF787FD01467F
:104010001B20BAE65D49514807F09EFE60BB504840
:1040200007F0A7FCB0F5966F17D0B0F5166F14D057
:10403000B0F5965F11D0B0F5165F0ED0B0F5964F83
:104040000BD0B0F5164F08D0B0F5614F05D0B0F5E4
:10405000963F02D0B0F5E13F0CD14D4C4D49206068
:10406000464806F077FE4649444806F050FE2C20AC
:1040700021688AE64849B9E64849384807F06CFEA5
:1040800088B9374807F071FC454C3B4920603B48F4
:1040900006F060FE3A49394806F039FE1F202178C3
:1040A00002F04CF973E63F492C4807F055FE98B9E9
:1040B0002B4807F05AFC3C4C072820600AD82E49B0
:1040C0002E4806F047FE2E492C4806F020FE3020F0
:1040D0002178E5E7354989E63549204807F03CFE77
:1040E000C0B91F4807F041FC4FF6E653314C206041
:1040F000013898420CD82049204806F02BFE204970
:104100001E4806F004FE13202188FDF7F0FA3EE673
:1041100029496BE62949114807F01EFE002853D1B2
:104120000F4807F022FC40F22E23254C206029384E
:1041300098420AD81049114806F00CFE10490F4861
:1041400006F0E5FD15202188DFE71E494EE600BF99
:104150000000000080842E4173CD0008350400204B
:104160004E040020200200200024744900007A44FC
:104170000000D7430000DC434DCD0008A00800201C
:1041800051CD00087BCD00080C02002084CD000832
:10419000880100208CCD0008AACD0008C9CD0008F8
:1041A00008020020D4CD000868020020DDCD000800
:1041B000EBCD00084C020020F3CD000812CE000821
:1041C000480200201BCE00089449954807F0C4FD22
:1041D000F8B9944807F0C9FB934B944C93FBF0F368
:1041E0009048236007F0C1FB282810DD8D4807F0B8
:1041F000BCFBB0F5167F0ADA8D498E4806F0AAFDA1
:104200008D498C4806F083FD102021887DE78B497D
:10421000ECE58B49824807F09FFDA0B9814807F083
:10422000A4FB884C2060013803280AD880498148C3
:1042300006F090FD80497F4806F069FD1220217844
:104240002EE78149D2E58149754807F085FDA0B97F
:10425000744807F08AFB7E4C2060073801280AD892
:104260007349744806F076FD7349724806F04FFDB5
:104270000E20217814E77749B8E57749684807F0B8
:104280006BFD002833D1674901A806F001FF01A8A2
:10429000FDF748FAFCF762FC704C206001A806F0BC
:1042A000B5FE25684FF07E512846FCF749FF58B906
:1042B0004FF080412846FCF743FF28B94FF07F516B
:1042C0002846FCF73DFF80B159495A4806F042FDA7
:1042D0005949584806F01BFD61492068FCF79CFDD0
:1042E000FCF79CFFC1B20F20DAE65E497EE55E492D
:1042F0004B4807F031FDA0B94A4807F036FB5B4C4C
:10430000C0B20F2820700AD849494A4806F022FD59
:104310004949484806F0FBFC17202178C0E654497B
:1043200064E554493E4807F017FD70B93D4B524CC7
:104330001B783F493F48237006F00CFD3E493D483D
:1043400006F0E5FC18202178AAE64C49344807F02D
:1043500003FD70B9334B4A4C1B78354935482370FF
:1043600006F0F8FC3449334806F0D1FC19202178D6
:1043700096E644492A4807F0EFFCB8B9294807F007
:10438000F8FA84B20F2C2A492A4838BF0F2406F0C5
:10439000E1FC2949274806F0BAFC4FF47A72E31F82
:1043A0005343394A214620201360AEE637491C4862
:1043B00007F0D2FC044600286ED11A4D2B7853B377
:1043C000DFF8CC8015F8016B04F132075EB9314695
:1043D00001A80197FDF707F921462D4806F03CFF9B
:1043E0000670134902E5A6F16103192B98BF06F088
:1043F0005F06214698BF05F8016C404615F8016C30
:1044000006F02AFF067015F8011C01A80197013477
:10441000FDF7E9F8D6E71F49E8E400BF38CE000809
:10442000350400204E04002040420F001C020020F2
:104430004DCD0008A008002051CD000840CE000856
:104440005CCE00081002002066CE000885CE000871
:10445000180200208ECE0008A0CE00081402002012
:1044600000002041A9CE0008C4CE00083C02002074
:10447000CDCE0008DFCE00082D020020EACE0008D5
:104480002C020020F4CE000858020020FCCE0008C8
:104490008C08002005CF00089A499B4807F05CFC77
:1044A000044660BB994B1B78002BB4D0974E984FB5
:1044B00016F8015B04F13C0355B9294601A80193A4
:1044C000FDF791F82146924806F0C6FE057088E790
:1044D000A5F16102192A9CBF05F05F0506F8015C91
:1044E00016F8011C01A80193FDF77DF82146384616
:1044F00016F8015C06F0B0FE01340570D8E7854976
:10450000814807F029FCE0B9804C2378BBB12146F3
:10451000814806F00EFE8149814806F01BFC814966
:104520007F4806F0F4FB214601A806F0B1FD5020BB
:1045300001A9FDF781F801A806F068FD27E47A4992
:1045400054E47A49704807F007FC0546E0B96F4823
:1045500007F00BFA0128044614D87049704806F099
:10456000F9FB70496E4806F0D2FB714B04F0010272
:104570001A70704A137803F07E03E118C9B2117003
:1045800028468DE56C4931E46C495F4807F0E4FB4F
:104590000546D0B95D4807F0E8F901280446F1D88E
:1045A0005E495F4806F0D6FB5E495D4806F0AFFB0A
:1045B000634B04F001021A705E4B197801F07D0123
:1045C00001EB4401C9B21970DAE75E494E4807F0C1
:1045D000C3FB0546C0B94D4807F0C7F9012804469A
:1045E000D0D84E494E4806F0B5FB4E494C4806F02F
:1045F0008EFB554B04F001021A704E4B197801F0F6
:104600007B0101EB8401DDE750493F4807F0A4FB43
:104610000546C0B93D4807F0A8F901280446B1D8BD
:104620003E493F4806F096FB3E493D4806F06FFB89
:10463000474B04F001021A703E4B197801F07701E4
:1046400001EBC401BEE743492F4807F085FB05464F
:10465000B8B92E4807F089F90128044692D82F49A5
:104660002F4806F077FB2F492D4806F050FB3A4BB8
:10467000621C1A602F4B197801F06F0101EB0411D5
:10468000A0E73649204807F067FB0546C8B91F4830
:1046900007F06BF9012804463FF674AF1F49204824
:1046A00006F058FB1F491E4806F031FB2C4B04F066
:1046B00001021A701F4B197801F05F0101EB4411E0
:1046C00080E72849104807F047FB054600284DD1F0
:1046D0000E4807F04AF9012804463FF653AF0F4948
:1046E0000F4806F037FB0F490D4806F010FB1E4B34
:1046F00004F001021A700F4B197801F03F0101EB31
:1047000084115FE71ACF0008350400204E04002012
:104710007408002023CF0008800800204DCD000839
:10472000A008002051CD00082BCF00083FCF000883
:1047300054020020340400204BCF000852CF000860
:10474000240200205DCF00084502002068CF000849
:104750007108002074CF0008280200207DCF0008D7
:104760007008002087CF0008980800205449554859
:1047700007F0F2FA0546C8B9534807F0F6F80128E1
:1047800004463FF6FFAE5149514806F0E3FA51495D
:104790004F4806F0BCFA504B04F001021A704F4B20
:1047A000197801F07F0101EBC4110BE74C49454832
:1047B00007F0D2FA28B133783F2B02D0482B40F0D3
:1047C000CF804849424806F0C5FA4749404806F0BC
:1047D000C1FA46493E4806F0BDFA45493C4806F054
:1047E000B9FA44493A4806F0B5FA4349384806F060
:1047F000B1FA4249364806F0ADFA4149344806F06C
:10480000A9FA4049324806F0A5FA3F49304806F077
:10481000A1FA3E492E4806F09DFA3D492C4806F083
:1048200099FA3C492A4806F095FA3B49284806F08F
:1048300091FA3A49264806F08DFA3949244806F09B
:1048400089FA3849224806F085FA3749204806F0A7
:1048500081FA36491E4806F07DFA35491C4806F0B3
:1048600079FA34491A4806F075FA3349184806F0BF
:1048700071FA3249164806F06DFA3149144806F0CB
:1048800069FA3049124806F065FA2F49104806F0D7
:1048900061FA2E490E4806F05DFA2D490C4806F0E3
:1048A00059FA2C490A4806F055FA2B49084806F0EF
:1048B00051FA2A49064806F04DFAFFF768BA00BFD8
:1048C0008FCF0008350400204E0400204DCD000895
:1048D000A008002051CD000844020020340400202C
:1048E00098CF00089DCF0008B0CF0008F1CF000896
:1048F00007D000082DD000083ED000084FD0000897
:1049000061D0000885D00008A8D00008CAD00008EF
:10491000ECD000080FD100083BD1000856D10008A8
:1049200072D1000889D10008A5D10008BFD10008C4
:10493000D3D10008ECD100080CD2000821D2000825
:1049400047D200086DD2000889D20008A1D2000821
:10495000BAD20008CDD20008EDD20008FED200087D
:10496000A449A54807F0F8F9002840F0D381A349ED
:10497000A34806F0EFF9A349A14806F0C8F9A24BF5
:10498000A24DA34C19789E4800290CBF2946214608
:1049900006F0E0F99F499A4806F0B9F99E4998480F
:1049A00006F0CEF99D49964806F0B1F99C4B0322DA
:1049B0001968934806F0D2FA9A49914806F0CAF964
:1049C00099498F4806F0A3F998498D4806F0B8F93F
:1049D00097498B4806F09BF9964B0A22197888482C
:1049E00006F003FA9449864806F091F9934B8448FF
:1049F000197806F0B1F99249814806F088F9914B8F
:104A00007F48197806F0A8F98F497D4806F07FF9AC
:104A10008E4B8F4A19688F4B7948022914BF114673
:104A2000194606F097F98C49754806F070F98B4BDA
:104A30007348197800290CBF2946214606F08AF9E7
:104A400087496F4806F063F9864B6D48197800294D
:104A50000CBF2946214606F07DF98349684806F0D7
:104A600056F9824B6648197800290CBF2946214621
:104A700006F070F97E49624806F049F97D496048C0
:104A800006F05EF97C495E4806F041F97B4B032253
:104A900019685B4806F062FA6249594806F05AF90B
:104AA0007749574806F033F9764B0A22196854487B
:104AB00006F09BF97449524806F029F9734B01221C
:104AC00019684F4806F04FFA71494D4806F01FF932
:104AD000704B71491B680A2291FBF3F1484806F0BC
:104AE00084F96E49464806F012F96D4B0A2219689E
:104AF000434806F07AF96B49414806F008F96A4BD9
:104B00003F48197800290CBF2946214606F022F9B2
:104B100066493B4806F0FBF8654B0A22196838489D
:104B200006F078F96349364806F0F1F8624B032243
:104B30001968334806F012FA3A49314806F00AF982
:104B40005E492F4806F0E3F85D4B0A2219682C48AD
:104B500006F04BF95B492A4806F0D9F85A4B284829
:104B6000197800290CBF2946214606F0F3F8574969
:104B7000234806F0CCF8564B03221968204806F06B
:104B8000EDF928491E4806F0E5F852491C4806F0A0
:104B9000BEF8514B0A221968194806F026F94F4908
:104BA000174806F0B4F84E4B4E4A19784E4B14484D
:104BB00000290CBF1146194606F0CCF84B491048A5
:104BC00006F0A5F84A4B0A2219680D4806F00DF9BF
:104BD00048490B4806F09BF84FF47A71464B0A227D
:104BE0001B68074803F5DA53183393FBF1F106F01D
:104BF000FCF883E03DD300083504002042D30008D0
:104C0000A008002051D3000845020020F8CE00087B
:104C10002ACD000858D300088C08002064D300086F
:104C20004002002075D300087AD3000880080020D5
:104C300089D300083C02002095D300082D020020F3
:104C4000A3D300082C020020B7D3000828020020BC
:104C500030CD00082DCD0008C3D3000898080020EF
:104C6000CED3000844020020DBD300082402002039
:104C7000E2D3000874080020EED3000820020020D0
:104C8000FFD30008180200200BD4000814020020F3
:104C90001CD400081C02002040420F002CD4000845
:104CA0001002002039D400085402002041D400082A
:104CB0004C0200204CD40008500200205ED40008B2
:104CC000480200206FD400087108002077D4000843
:104CD0000C02002089D400080802002097D40008A4
:104CE000700800203CCD000837CD0008A4D400088F
:104CF00068020020B2D40008580200200749084882
:104D000006F005F8074B0A221968054806F08CF8EA
:104D1000FFF73DB80449FFF76DB800BFBDD40008E8
:104D2000A008002088010020CDD4000810B50F484D
:104D300005F019FD002801DDFEF79EFFC62006F0F4
:104D4000A3FC0446C52006F09FFC323484420CD9F3
:104D5000C52006F099FC502807D9054B1B68002B8D
:104D600003DDBDE81040FDF796BE10BDA008002091
:104D7000A401002038B5684805F0F5FC002801DDE5
:104D8000FEF77AFFC62006F07FFC0446C52006F039
:104D90007BFC3234844250D9C52006F075FC502883
:104DA0004BD95E4B1B68002B47D0012B03D1BDE8CC
:104DB0003840FDF770BE022B3FD1594C2368032BBE
:104DC00007DD2368013B032B35D8DFE803F01E37EE
:104DD0005DA2C62006F058FC0546C52006F054FC2E
:104DE00032358542EDD9FDF7A3FE4FF4C87006F0C9
:104DF0009DFDFDF745FE4FF4C87006F097FDFDF7E9
:104E0000ADFE236801332360D8E7464B1B7893B18E
:104E1000454B1B68032B0EDC444B1B685BB1444BBA
:104E20001A7842B901221A70FDF72AFEC82006F04E
:104E30007DFDFDF793FE0023236038BD3D4A00232E
:104E4000157885B11D46137023689D42F3DAFDF78E
:104E500017FE322006F06AFDFDF780FE322006F0D4
:104E600065FD0135F0E70123137023689D42E2DA06
:104E7000FDF75EFE322006F059FDFDF76FFE322091
:104E800006F054FD0135F0E72B4B1B68013330D1A0
:104E90002A4B18682A4B1A6882422A4A14D0186092
:104EA0001060C0B2FCF75CFE002523689D42C2DAA8
:104EB000FDF73EFE322006F039FDFDF74FFE3220B1
:104EC00006F034FD0135F0E7002528461D60156029
:104ED000FCF746FE23689D42ADDAFDF7D1FD322096
:104EE00006F024FDFDF73AFE322006F01FFD0135E5
:104EF000F0E70021182006F0D9FC4FF4C87006F046
:104F000015FD0121182006F0D1FC642006F00EFDED
:104F100091E7FDF7C0FD8EE7A0080020A401002066
:104F200054080020E901002018080020E4010020B6
:104F3000DA0700205D0200206002002068020020E5
:104F400064020020000800202DE9F0410C461C4EB0
:104F50001C4F451E15F8013F0BB9BDE8F0812E2B03
:104F6000DFF864801AD1FCF755FD3B687168B3FB2C
:104F7000F8F3634312484268521A9342FBDCFCF791
:104F800051FD3B68104A7168B3FBF2F363437268EA
:104F9000521A9342FBDCFFF7EDFEDBE72D2BF0D13D
:104FA000FCF738FD3B6804EB4402B3FBF8F35343D2
:104FB000716803484268521A9342FBDCDFE700BF86
:104FC000001000E09802002040420F00F8B5214F89
:104FD000214D97FBF1F7214E441E14F8013F03B910
:104FE000F8BDA3F14102D1B2192912D839461C4BA0
:104FF00053F82200FFF7A8FF2B681A4A7168B3FB29
:10500000F2F37B4303EB43037268521A9342FBDCD7
:10501000E3E7A3F13002092A05D8114A163B3946C5
:1050200052F82300E6E7212B04D10D4B3946D3F883
:105030009400DFE7202BDFD12B680A4A0749B3FB36
:10504000F2F37B434868C3EBC3034A68121A9342E6
:10505000FBDCD1E780841E0098020020001000E0F5
:105060009C00002040420F001FB51F4B1B78002BF7
:1050700031D01E4B1B7873B31D4B01A81B783BB37B
:10508000FDF79EFE01A91B4806F04BF801A805F0AC
:10509000BDFF184B1C68FCF7C9FC174B1868FBF7E1
:1050A0000DFA0FA3D3E90023FBF7AAF8FBF756FD8F
:1050B000FCF7DEFC06F036FC104B1860104B204667
:1050C0001968FFF783FF04B0BDE81040FCF7AABCE5
:1050D000FEF710FBD6E704B010BD00BFAFF30080B1
:1050E0002D431CEBE2364A3F710800205D02002090
:1050F00070080020380800200C020020F007002073
:1051000008020020264B10B518600446254805F01B
:105110002AFB002801DDFEF7AFFD8CB90021C72076
:1051200006F0C8FA0021192006F0C4FA0021C720B1
:1051300006F0BCFB0021BDE81040192006F0B6BB0C
:10514000631EFE2B0DD80021C72006F0B3FA002104
:10515000C72006F0ABFB2146BDE81040192006F041
:10516000A9BAA4F58073F32B0AD8C720A4F1FF01D4
:1051700006F0A0FAFF21192006F09CFA0121DAE7D7
:10518000B4F5FA7FCAD1FF21C72006F093FAFF21B8
:10519000192006F08FFA0121C72006F087FBEDE702
:1051A000A0070020A00800202DE9F843664B0C461C
:1051B0001B78154633B128B1FCF712FEFCF708F84E
:1051C00014283EDD0020FCF791FE604B1B78002B7D
:1051D00000F0AA80002D00F0A580002C00F0A48033
:1051E0005B4B1B78002B40F09F805A4B00211C68C2
:1051F0002046FBF7AFFF002800F09680564B1B6857
:10520000552B40F39180554B554F1868FBF7B0FD77
:105210002146FBF7F9FC534B1968FBF7F3FC5249A5
:1052200005463E68FBF7B4FFD8B1F41D4F4B1B6831
:105230009C42A8BF1C4620463C60BDE8F843FFF7EF
:1052400061BFA0F11303012B01D80120BBE7A0F13E
:105250001003022B01D80220B5E70A28B2DC032094
:10526000B1E74FF081412846FBF792FF08B1741D6A
:10527000DCE72846FBF722F92DA3D3E9002380467B
:105280008946FBF703FC08B1F41CCFE740462AA38C
:10529000D3E900234946FBF7F9FB08B1B41CC5E785
:1052A0004FF07F512846FBF773FF08B1741CBDE730
:1052B0002F4B4FF0414128461C68FBF74BFF20B1B4
:1052C000083EB442B8BF3446B5E728462949FBF743
:1052D00041FF08B1043EF4E7404619A3D3E9002397
:1052E0004946FBF7B5FB08B1023EEAE728462249EA
:1052F000FBF730FF08B1013EE3E7B4429BDC1B4BF8
:105300001C68B442A8BF344695E7124B00211868C8
:10531000FBF720FF40B1104B1B68552B04DD104BF1
:1053200018688AE7002CF0D1002086E7AFF30080F0
:1053300066666666666606409A99999999990140EB
:105340009A999999999901C05A0800205908002002
:10535000A5070020CC070020B0070020B8010020DE
:10536000B0010020C00700200000C040B4010020B0
:10537000AC010020000080C00000C0BF2DE9F74F45
:10538000DFF86C92FDF7DFFBFFF7D0FCFCF7B4FE13
:1053900099F80030C3B10524FDF772FBFA2006F03E
:1053A000C5FAFDF7DBFB4FF4967006F0BFFAFFF786
:1053B000BDFC013CF0D1012220468E4B1A7003B097
:1053C000BDE8F04FFFF79EBEFFF7B0FC8A4B1B789D
:1053D00003B3FDF7C3FB322006F0A8FAFDF7B3FBD9
:1053E0000023864C2360FCF787FE854B1968854BAC
:1053F0001868FBF707FCFBF7EBFEFBF7B9FC206036
:10540000FDF7ACFB322006F091FAFDF79CFB322051
:1054100006F08CFAFDF7A2FB002606F083FA35466B
:105420008046DFF8DCA1DFF8E0B1FFF77FFCFCF796
:1054300063FE99F80030B3B10020FFF763FE052446
:10544000FDF71EFBFA2006F071FAFDF787FB4FF41B
:10545000967006F06BFA013CF2D10122654B1A708E
:1054600003B0BDE8F08F694B1868FBF781FCDAF8F0
:105470000040DBF8007021460190FBF76BFE00282E
:1054800044D007F11400FBF773FC01462046FBF7FC
:1054900061FE00283AD0FDF756FB3C2006F046FAA4
:1054A000FDF75CFB2846FBF75FFC594B013619689A
:1054B000FBF7AAFBFBF7B2FE054640F27710FFF7B9
:1054C00021FE06F02FFA534BA0EB08001B68984210
:1054D00067D90122474B00201A700524FFF712FEFE
:1054E0004D4DFDF7CDFAFA2006F020FAFDF736FB18
:1054F0004FF4967006F01AFA284605F034F90028A1
:1055000001DDFEF7B9FB013CEBD1A9E707F11E0075
:10551000FBF72EFC01462046FBF73AFEC0B1FF2008
:10552000FFF7F0FDFDF70FFBC82006F0FFF9FDF7D0
:1055300015FBC82006F0FAF9FDF705FBC82006F0B8
:10554000F5F9FDF70BFB4FF4C87006F0EFF9B8E77B
:1055500007F10F00FBF70CFC01462046FBF718FE95
:1055600010B14FF49B70DBE7781DFBF701FC01469F
:105570002046FBF70DFE10B14FF4B470D0E7214682
:105580000198FBF705FE00289BD04FF4FA70FFF757
:10559000B9FDFDF7D8FAC82006F0C8F9FDF7DEFA24
:1055A0008FE7082E7FF441AF0020FFF7ABFD032407
:1055B000FDF7BEFAC82006F0B9F9FDF7CFFAC8200A
:1055C00006F0B4F9013CF3D10A4BE8081C70FBF774
:1055D000CBFB124B04461860114B1868FBF7C4FB59
:1055E00001462046FBF70EFB0E4B186038E700BF64
:1055F000A6070020A4070020D0010020D40100202D
:10560000C0070020CC070020BC010020C001002002
:10561000BC070020C4010020A0080020B80700201B
:10562000CC010020B40700200246014805F016B95D
:10563000B809002008B5174B1B7873B1164B1B78BF
:10564000C3B116491120FFF7EFFF4FF47A7006F04F
:105650006DF911201149FFF7E7FF0021172006F02F
:1056600025F9322006F062F9BDE808400121172033
:1056700006F01CB90A4B1B78002BEED009492C20F0
:10568000FFF7D2FF4FF47A7006F050F92C2005494D
:10569000E1E700BFF4010020450B00207401002069
:1056A000700200204801002010B50121182006F0EA
:1056B00093F80121172006F08FF801210C2006F045
:1056C0008BF80121202006F087F87D4B1B781BB159
:1056D0000121002006F080F801211C2006F07CF852
:1056E0000121C22006F078F80121162006F074F896
:1056F0000121C32006F070F80121212006F06CF88A
:105700000121222006F068F80121132006F064F838
:105710000121142006F060F80121152006F05CF844
:105720000021C12006F058F80121C72006F054F8E6
:105730000121192006F050F801210F2006F04CF845
:1057400000211C2006F0B2F80021C22006F0AEF8BD
:105750000021162006F0AAF80021C32006F0A6F8C2
:105760000021212006F0A2F80021222006F09EF858
:105770000021172006F09AF80021182006F096F86C
:10578000322006F0D3F80121172006F08FF801210E
:10579000182006F08BF84B4B4B4C196806224B48EF
:1057A00005F03AFAFEF7DCF82378002B78D0484B66
:1057B00006221968474805F02FFA4749434805F083
:1057C000C9FA237813B10C2005F03AFF082005F040
:1057D00045FF4FF47A7005F051FF404C404800F00F
:1057E000A3FB0121202006F061F82378002B5CD078
:1057F0003C4B1B68002B58D0FCF76FFB002120208E
:1058000006F054F8FCF708F8374B1878FCF7A8F9BD
:1058100005217220FBF7E4FF344B00201A68344B5B
:10582000B3FBF2F3334A1360FCF760FB0020FFF791
:1058300069FC00210846FBF769FE0021172006F0ED
:1058400035F8322006F072F80121172006F02EF804
:10585000C82006F06BF80021172006F027F8322048
:1058600006F064F80121172006F020F8224B1B787F
:105870003BB1224B1B7823B1214B1B780BB1FFF7B7
:105880007DFD2378D3B1174B1B68BBB1FCF729FB17
:105890004FF47A7006F04AF8BDE81040FFF7CABE30
:1058A000184B1B78002B88D081E7FCF71AFB4FF4CC
:1058B0007A7006F03BF8FFF7BDFE9FE710BD00BF12
:1058C000440B002088010020450B0020A008002088
:1058D0006C020020B8090020D1D40008E9010020A2
:1058E000D00A0020E4010020000800204802002027
:1058F00040420F0030030020DC010020C9010020DD
:10590000C801002070020020144B70B51B780446BB
:1059100053B1012809D1124D2B68012B04D00A2064
:105920001049FFF781FE2C6070BD0228FCD10C4E9F
:105930003368022BF8D005F0F5FF0B4D2B68C01A29
:105940000A4B1B689842EFD90A200949FFF76CFE01
:10595000346005F0E7FF2860E6E700BF7002002032
:10596000900100203E010020E4070020E00100201B
:1059700034010020000000002DE9F041764D2C6834
:105980002CB9FCF7AAFA2B6853B9BDE8F081012CB9
:1059900003D1FCF7A6FA0120C8E0022C00F0BE807B
:1059A00005F0C0FF04466D4E6D4FDFF8B8813046FC
:1059B00004F0D9FE0546002840F0BB8005F0B2FF98
:1059C0003A68031B9342F2D36422664C236D04F1C0
:1059D0004C00B3FBF2F3644A84F84D50136000F0BE
:1059E000E3FD624B186004F14C0000F0E7FD604BF2
:1059F000186004F14C0000F0EFFD5E4B186020468B
:105A000000F066FDFBF7AAF85B4B1860204600F03B
:105A100083FDFBF7A3F8594B84F87D501860D4F848
:105A20008400FAF739FD0022554BFAF7C9FEFBF75F
:105A300095F8544B84F85D501860606EFAF72CFDB1
:105A400041A3D3E9002306460F46FAF78FFD002253
:105A50004B4BFAF7B5FEFBF781F84B4B3946186014
:105A60003BA3D3E900233046FAF780FD0022444BE4
:105A7000FAF7A6FEFBF772F8444B454E1860D4F8CF
:105A80009430D4F8A40084F88D50336084F89D508D
:105A9000FAF702FD3A4B0022FAF792FEFBF75EF8A6
:105AA0003C4D3D4F2860FCF751FC3B6813B33B4C29
:105AB000237843B93368022B1CDC05F033FF384BE5
:105AC00018600123237005F02DFF354A1368C01AB2
:105AD0003B6898420ED93368022B4FF000032370C5
:105AE000136007DCFDF706F94FF47A7005F01EFF2E
:105AF000FFF7A0FD2B4B2C4C1B7813B32B492868C8
:105B0000FBF746FB38B92A4B2A49186820F00040B9
:105B1000FBF73EFBA8B10123237036E7FCF7E1F960
:105B20001B4B1B68062B7FF736AF2046FFF7ECFEBA
:105B300029E7304605F0B4F8C1B2404600F0C2FE95
:105B400035E70023E8E700BFCF16AD2F5476E03FDE
:105B50006F1283C0CAA1FD3FE4010020B8090020F4
:105B6000F0010020480B00203408002030080020FD
:105B70002C08002028080020600800205C08002075
:105B80000000594024080020200800201C080020A4
:105B90001808002014080020EC010020EC07002069
:105BA000E8070020D8070020D90700200000704136
:105BB000F8070020000096433D4B70B51B683D4C34
:105BC000034423603C4B1B782BB13C4B1B7813B137
:105BD00001223B4B1A703B4B1B78A3B33A4B1B681B
:105BE000032B30DC394B1B686BB3354B1B7853BB35
:105BF000FBF714FF0120FFF787FE1424344EFCF757
:105C0000B9FFFCF757FFFFF7B7FE304604F0ABFDD6
:105C1000002801DDFEF730F80525FFF7ABF801217C
:105C2000172005F043FEC82005F080FE0021172054
:105C300005F03CFE40F2EE2005F078FE013DECD18F
:105C4000013CDCD170BD41F286330138984229D93C
:105C5000204B1B780BB1FBF7E1FE05F063FE2368D8
:105C60009842EFD2FFF786F8FCF784FFFCF722FF9B
:105C7000FFF782FE002201211046FFF795FAFCF79C
:105C80003BFA012211461046FFF78EFAE5E7FFF7CF
:105C900071F8FCF76FFFFCF70DFF0022114610466C
:105CA000FFF782FA05F03EFE23689842EFD3C9E77A
:105CB000F0070020F4070020E8010020D8070020AA
:105CC000DA070020E901002018080020E401002084
:105CD000A00800205C02002010B5FFF74BF801215E
:105CE00000220846FFF760FAFCF744FFFFF744FE86
:105CF000FCF7E0FE002201211046FFF755FAFCF701
:105D0000FBF9012211461046FFF74EFAFDF722F883
:105D1000FFF730F8FCF72EFF012100220846FFF7BD
:105D200043FA324B1B7853B1FFF79EF9FFF722F885
:105D3000FCF720FF012100220846FFF735FA2C4B23
:105D40001B7853B1FDF772F9FFF714F8FCF712FF57
:105D5000012100220846FFF727FA264C237853B189
:105D6000FDF73AFAFFF706F8FCF704FF01210022DD
:105D70000846FFF719FAFEF7FDFFFCF7FBFE0121CD
:105D800000220846FFF710FA23781B4C8BB12378CA
:105D90007BB1FFF7F1FDFCF78DFE002201211046DB
:105DA000FFF702FAFCF7A8F9012211461046FFF7A7
:105DB000FBF9FEF7DFFFFCF7DDFE012100220846BC
:105DC000FFF7F2F9237853B1FDF76AFBFEF7D2FF34
:105DD000FCF7D0FE012100220846FFF7E5F9BDE8F7
:105DE0001040064B1868FFF7E7BE00BF710800209F
:105DF0002402002054020020450200205802002006
:105E00002DE9F0411C46454B1646C36601230D465D
:105E1000A0F870305C2200210746DDF8188005F0FC
:105E200093FFF3B2242B28D83D4A06F4E06652F8DB
:105E300023301E43EBB2242BFE6532D8384A05F4DA
:105E4000E06552F823301D43E3B2242B3D663CD875
:105E5000334A04F4E06452F823301C435FFA88F2BA
:105E6000242A7C6645D82E4908F4E06351F82220A4
:105E700013433846BB66BDE8F08106F0C002C02A75
:105E80000CD1C92B0AD8274B06F03F0253F8222029
:105E9000234B06F4E06653F82230CAE74FF0FF3692
:105EA000C8E705F0C002C02A0CD1C92B0AD81D4B87
:105EB00005F03F0253F82220194B05F4E06553F832
:105EC0002230C0E74FF0FF35BEE704F0C002C02A21
:105ED0000CD1C92B0AD8134B04F03F0253F82220EF
:105EE0000F4B04F4E06453F82230B6E74FF0FF3470
:105EF000B4E708F0C003C02B0CD1C92A0AD8094B5B
:105F000008F03F0253F82210054A08F4E06352F803
:105F10002120ADE74FF0FF33ABE700BF00093D00A4
:105F200048DB000820DB000800220123054910B4EB
:105F300010BC80F85120C16680F8703080F8712064
:105F400000F04EB800093D0007B5002A8DF8071093
:105F50000DF107014FF001030CBF0A46002200F0CB
:105F600079F99DF8070003B05DF804FB252307B518
:105F7000C6220093C721C5230248FFF741FF03B0A3
:105F80005DF804FB240C002091FAA1F3B3FA83F32B
:105F900070B50D0E0F2691FAA1F1B1FA81F14459B5
:105FA0009B0006FA03F3890024EA03048A40224393
:105FB000425170BD0346074A10684BB1064A9342EE
:105FC00001D101F05BBD054A934201D101F046BD0C
:105FD000704700BF980200200030014000380040A8
:105FE0002DE9F74F0E4615461F460446002800F0DF
:105FF000ED808F49006E03F031FF8E498146E06DE0
:1060000003F02CFF8C498346606E03F027FF8B4919
:106010008046A06E03F022FF8246B9F1000F00F027
:10602000D580BBF1000F00F0D180B8F1000F00F077
:10603000CD805946484603F038FF514681464046D8
:1060400003F033FF01468046484603F02EFFA0656B
:10605000B9F1000F00F0BA80B8F1000F00F0B6807F
:10606000002800F0B380A26E4FF48273511C0CBF65
:106070004FF400724FF480222060A2616360FFF74A
:1060800099FFB6EB500F80F0A480B6EB900F80F034
:10609000A280B6EBD00F80F0A080B6EB101F80F08E
:1060A0009E80B6EB501F80F09C80B6EB901F80F076
:1060B0009A80B6EBD01F2CBF30233823E361002D2C
:1060C00000F09380022D00F09280013D18BF012561
:1060D00001236D00C4E904530723E362B7FA87F391
:1060E00000265B09DB01C4E908365149206EA66031
:1060F000A662E66003F09AFE4E49E06D03F096FE5C
:106100004D49606E03F092FE2369B342636E18BF7F
:106110000125C3F3031208BF0225042A8CBF3046B1
:10612000474903F00F0398BF51F82200454A022D5A
:1061300052F8231091FAA1F24FEA1163B2FA82F2F7
:10614000C6584FF00F034FEA820203FA02F391FAA6
:10615000A1F2B2FA82F203EA06034FEA820223FABC
:1061600002F34FEA112544D0042B02D10822FFF795
:106170000BFFC268012322EA050295FAA5F5B5FADC
:1061800085F5AB401343C3602C49A06E03F04EFE6F
:1061900023682D4A934235D12C4B9A6942F48052A0
:1061A0009A619A6902F480520092009ADA6842F485
:1061B0008052DA60DA6822F48052DA60204601F018
:1061C000BEFC2268136843F04003136003B0BDE8CF
:1061D000F08F002372E7082370E710236EE718237F
:1061E0006CE720236AE7282368E72B4672E7002341
:1061F00070E7042B02D10822FFF7C6FEC36823EA2A
:106200000503C0E7124A9342D8D1104BDA6942F431
:106210008042DA61DA6902F480420192019A1A69D5
:1062200042F480421A611A6922F480421A61C5E779
:10623000D0D60008A0D6000870D6000840D60008C6
:1062400078020020E8D5000800300140001002402C
:10625000003800402DE9F0410D4616461C4633B388
:10626000076800F0C1FB8046BB689907FCD5D5B133
:1062700015F8013B3B73BB68DA07FCD53B7B0EB1DD
:1062800006F8013B00F0B0FBA0EB0800B0F57A7F08
:1062900004F1FF3409D2002CE6D12046BB681B066E
:1062A000FCD4BDE8F081FF23E4E70120F6E70220FB
:1062B000F7E7000008B54FF480620249024805F094
:1062C000DBFD08BD00FC0108980C002010B5044659
:1062D000FFF7F0FF014B185D10BD00BF980C0020C8
:1062E000002370B586B0CDE9013301230F4C05932F
:1062F000CDE9033401F076F8B0B940F215120C4B39
:1063000001A9DA6002A801F017F958B9094D0A4E3F
:106310002146F5E80223032001F0AAF810B9083459
:10632000B442F5D101F070F806B070BD00FC010870
:1063300000200240980C002000000208014B195474
:10634000FFF7CEBF980C0020302180F834104E218A
:10635000002280F83610022102808280826002735F
:106360000282426102768283026280F824200285E2
:10637000C26280F8302082870264A0F84C20026557
:10638000A0F85C204266A0F86C204267A0F87C2050
:10639000C0F88420A0F88C20C0F89420A0F89C209D
:1063A000C0F8A42080F8BD10A0F8BE2080F8C0205E
:1063B000C0E93122C0E93322C0E93522A0F8AC207F
:1063C00080F8AE207047A1F14103052B02D8A1F15E
:1063D00037007047A1F16103052B94BFA1F157006D
:1063E000A1F13000704738B5044605782D2D08BF5F
:1063F0000134204605F0BDFA64235843224614F8C0
:10640000013BA3F130010929F8D92E2B0BD1537888
:10641000303B092B07D80A2101FB03009378303B5E
:10642000092B98BFC0182D2D08BF404238BD000071
:1064300038B50D46044605F09CFA6423B0FBF3F230
:1064400003FB1203204611492A804B430278014680
:10645000A2F13004092C00F10100F7D92E2A0BD14A
:106460000A240A4803E0B0FBF4F000FB023311F801
:10647000012F303A092AF6D9032203EB83030133B3
:10648000B3FBF2F36B6000232B7238BD809698004B
:10649000C36910B54360036A0446836090F82430F2
:1064A0000373836A0361C36A436190F830300376F3
:1064B00090F8353080F8343090F8373080F8363046
:1064C00005F030FA40F20113A063238010BD0000F4
:1064D0000023D0B5044643708068F9F7CDFF0CA3C4
:1064E000D3E90023FAF76CF90646A0880F46F9F7BE
:1064F000D3FF0B46024639463046F9F781FE237B2F
:1065000013B101F100431946D0BD00BFAFF30080C5
:106510000000000065CDCD410023D0B50446437096
:106520004069F9F7A9FF0CA3D3E90023FAF748F96A
:106530000646208A0F46F9F7AFFF0B46024639465A
:106540003046F9F75DFE237E13B101F10043194691
:10655000D0BD00BFAFF300800000000065CDCD418D
:10656000836810B54360044605F0DCF940F201137E
:10657000E060238010BD836810B54360044605F0D9
:10658000D1F940F20113E060238010BD10B504463C
:106590000846FFF728FFA06010BD10B50446084666
:1065A00005F0E7F9A06010BD002343704068024B7E
:1065B000B0FBF3F0C0B2704740420F0000234370BD
:1065C00042F210734068B0FBF3F06423B0FBF3F2C7
:1065D00003FB1200C0B2704700234370642340687D
:1065E000B0FBF3F0B0FBF3F203FB1200C0B2704754
:1065F000C36810B58360044605F094F940F20113B6
:106600006060238010BD10B504460846FFF7EBFE1E
:10661000E06010BDC36810B58360044605F082F9E0
:1066200040F201136060238010BD10B50446084697
:1066300005F09FF9E06010BD014610B5044610302A
:1066400005F012FC05F06EF940F201132062A384FC
:1066500010BD0F2205F0B8BB70B590F8AD600446D0
:10666000002E65D090F8AE10FFF7ADFE94F8AF1095
:1066700002462046FFF7A7FE94F8AC3000EB02106C
:10668000C0B283424DD1D4F8D8300133C4F8D830E9
:1066900094F8C03023B1D4F8D0300133C4F8D030EE
:1066A00094F8BD301BB3012B15D104F13C00FFF76A
:1066B00057FF04F14C00FFF75EFF94F8C03053B170
:1066C0002046FFF7E5FE04F15C00FFF791FF04F1BF
:1066D0006C00FFF78DFFD4F8C85035B1D4F8C8303E
:1066E000A86A996AF9F774FDB0B1304670BD04F13B
:1066F0004C00FFF740FF94F8C03033B12046FFF75D
:10670000C7FE04F17C00FFF773FF04F18C00FFF774
:1067100081FF04F19C00DCE72846FFF78DFF2D6B1D
:10672000DBE7D4F8D4300133C4F8D4300026DCE7FA
:1067300090F8BE209ABB90F8AE30472B29D190F844
:10674000AF105D4805F033FB18B304F1B0052846DF
:106750005A49F9F73DFDF0B128465949F9F738FD96
:10676000003818BF01204000D4F8C45084F8BD00A0
:1067700004F1AE06C4F8C850002DD7D03146A86A3F
:10678000F9F726FD002808DBD0D00023C4F8C83074
:10679000CCE70220E8E70120E6E72D6BEAE790F876
:1067A000BD10022924D090F8AE300BB342EA41125A
:1067B000013A2B2A1CD8DFE802F0163C434A4D640C
:1067C0006D73771B1B1B1B1B1B1B1B1B1B1B1B1B13
:1067D0001B1B1B1B1B1B1B1B1B1B16353C434A4D4A
:1067E000545A5E1B1B7B00F1AE014C30FFF7CEFE0E
:1067F000D4F8C85004F1AE06002D97D0D4F8C830B4
:10680000A86A996AF9F7E4FC00288FD1EA6A94F83B
:10681000BE309A428ADC03D131462846FFF719FF81
:106820002D6BE9E7A3F141004342434184F8C030B6
:10683000DEE700F11C0104F1AE00FFF7F9FDD7E738
:10684000A3F153014B424B4180F82430D0E700F1D3
:106850002801F0E7A3F157025342534180F830304A
:10686000C6E700F1AE015C30FFF7CDFEC0E700F1F6
:10687000AE016C30F8E700F1AE013C30FFF78DFE61
:10688000B6E7302B94BF0022012280F8353080F823
:10689000C020ADE700F1AE018C30FFF7C6FEA7E7E0
:1068A00000F1AE019C30DFE700F1AE017C30DBE7A8
:1068B00080F837309CE700BF58D500085ED5000847
:1068C00062D5000838B5D0F8CC30242903F1010393
:1068D00004460D46C0F8CC302AD090F8BF301CD802
:1068E0000A2901D00D292FD10E2B4FF0000005D819
:1068F000234483F8AE002046FFF7AEFE94F8BE3086
:10690000013384F8BE30002384F8BF30A5F12A0398
:106910005D425D4184F8AD5038BD2A29E4D02C2970
:1069200012D190F8AC2082F02C0280F8AC20DBE78A
:1069300000230222A0F8AC3080F8BD20A0F8BE30C1
:1069400080F8C0300020E7E70D2B9FBF5A1C1B19B1
:1069500084F8BF2083F8AE5094F8AD30002BF1D10D
:1069600094F8AC305D4084F8AC50EBE77047000021
:1069700038B50E4B05461A784FF47A73B3FBF2F331
:106980000B4A1068B0FBF3F000F0CCFB044658B99A
:106990000F2D09D8024629464FF0FF3000F072FB58
:1069A0002046044B1D6038BD0120FCE77102002029
:1069B000980200207402002008B5032000F050FB6C
:1069C0000020FFF7D5FFFFF7D1FF002008BD000032
:1069D000034A044B11681B780B441360704700BFD7
:1069E0009810002071020020014B1868704700BF0A
:1069F00098100020F7B5002604460D460196FFF7D3
:106A0000F3FF236807469A68D10508D50120A36AD9
:106A100084F8246043F02003A36203B0F0BD5A68F9
:106A2000D20503D4DB6A13F4700F3DD03D4B022036
:106A30001E6801F04DF823683B4A1969B6FBF0F671
:106A400011423A4A51D1D868394908424DD11969A1
:106A500011425BD1DA68374B1A420CBF1423292349
:106A60005E43019BB34223D26A1C04D0002D53D154
:106A7000019BB3420AD3019B01330193F1E76E1CE2
:106A800013D065B923681B6898070DD4A36A032047
:106A900043F00403A362002384F82430BDE7FFF72A
:106AA000A3FFC01BA842EDD8226813689907E6D55A
:106AB0006FF0120322681360A36A43F40073A362A9
:106AC000936803F46023B3F5602F0CD1237B53B993
:106AD000A36A23F48073A362A36ADB0403D4A36ACA
:106AE00043F00103A362002097E71969114203D123
:106AF000D968104A11420BD019690F4A114209D1C5
:106B0000DB6813420CBF5423FC23A9E72923A7E722
:106B10005423A5E7FC23A3E7FFF766FFC01BA842A9
:106B2000A6D8A8E79802002024499224922449126A
:106B30002449920092244900499224000368D86CA9
:106B400070470000002373B5019390F82430044689
:106B5000012B6CD0012380F824304D680268062D8B
:106B6000086805EB850322D81F26556B053B9E4020
:106B700025EA060500FA03F32B43536309288B68C3
:106B800000EB40054FF0070129D9D6681E3DA9400A
:106B900026EA0101AB400B43D360A0F11003012BA7
:106BA00025D90020002384F8243002B070BD0C2DBC
:106BB0004FF01F0509D8166B233B9D4026EA0505BB
:106BC00000FA03F32B431363D8E7D66A413B9D4099
:106BD00026EA050500FA03F32B43D362CEE71069DA
:106BE000A94020EA0101AB400B431361D9E7114BE7
:106BF0009A4216D193681B02D3D49368102843F4A9
:106C000000039360CDD10C4B0C4A1B68B3FBF2F32D
:106C10000A2253430193019B002BC2D0019B013BED
:106C2000F8E7A36A012043F02003A362BAE7022039
:106C3000BBE700BF002401409802002040420F0043
:106C4000806A7047002337B50193036804469A6849
:106C5000D20702D5002003B030BD9A6842F001028D
:106C60009A60144B144A1B68B3FBF2F30193019B27
:106C7000E3B9FFF7B9FE054623689B68DB07E9D453
:106C8000FFF7B2FE401B0228F6D923689B6813F079
:106C90000103F1D1A26A012042F01002A262E26A6D
:106CA00084F8243042F00102E262D4E7019B013B08
:106CB000DCE700BF9802002040420F0010B590F8BA
:106CC00024300446012B3BD0012380F82430FFF709
:106CD000B9FF002830D1A36A23F4407323F00103E5
:106CE00043F48073A362A36A23F48013A36223682E
:106CF0005A68520541BFA26A22F4405242F48052BF
:106D0000A262A26A12F480521CBFE26A22F006025A
:106D1000E262002284F824206FF002021A609A686E
:106D200002F46022B2F5602F9A680CBF42F4A00210
:106D300042F480129A6010BD002384F82430FAE7F0
:106D40000220F8E738B5036804469A68D10701D4F1
:106D5000002038BD9A6822F001029A60FFF744FED5
:106D6000054623689B68DB07F2D5FFF73DFE401B15
:106D70000228F6D923689B68DA07F2D5A36A0120B6
:106D800043F01003A362E36A43F00103E362E0E728
:106D9000F8B5044600286DD0836A23B9C36280F831
:106DA000243002F08FFB2046FFF7CCFFA36A13F0DC
:106DB000100361D100285FD1A26A616822F4885271
:106DC00022F0020242F00202E569A668A262227B7A
:106DD0002943B6F5807F41EA420136D0771E7D42D5
:106DE0007D412D02277D012F06D182BBA269013A88
:106DF00045EA423242F400652268B6F5807F576862
:106E000027F4694745EA0705556097681D4D05EA6F
:106E1000070545EA0105956001D0012E02D12369DD
:106E2000013B1B05D56A25F470052B43D36292689C
:106E3000154B1340994213D10023E362A36A23F058
:106E4000030343F00103A362F8BD3546CAE7A26A13
:106E500042F02002A262E26A42F00102E262CBE763
:106E6000A36A23F0120343F01003A362E36A43F022
:106E70000103E3620120E7E7A36A43F01003A36282
:106E8000F8E700BFFDF7E1FFFE0E1FFF38B504462F
:106E9000002850D0836A43F002038362FFF752FF59
:106EA0000546002842D16FF01F02236820461A6071
:106EB0005968224A0A405A609968214A0A409A60F1
:106EC000DA6802F07F42DA601A6902F040421A6121
:106ED00059691C4A11405961996911409961D969F0
:106EE0001140D961196A11401962596A11405962F9
:106EF000996A0A409A62DA6A134902F07F42DA62BA
:106F0000DA6A02F07F42DA621A6B02F040421A63D8
:106F10005A6B02F040425A639A6B0A409A639A6B2A
:106F20000A409A6302F0EEFAE562A562002384F853
:106F30002430284638BD0125FBE700BF00003FFF95
:106F4000F00601FF00F0FFFF0000C0FF10B590F851
:106F500024300446012B11D0012380F82430FFF7A0
:106F6000F1FE38B9A36A23F4885323F0010343F0F8
:106F70000103A362002384F8243010BD0220FCE743
:106F8000002373B5019390F824300446012B62D09E
:106F9000012380F82430FFF7D5FE2046FFF752FE8C
:106FA000054600282FD1A36A022023F4885323F03A
:106FB000020343F00203A362284B1E6800F088FD21
:106FC000B6FBF0F676000196019B03BB226893683E
:106FD00043F008039360FFF707FD064623689A68AD
:106FE000110718D49A6842F004029A60FFF7FCFC7B
:106FF000064623689B685B0723D4A36A23F0030338
:1070000043F00103A362002384F8243016E0019BBF
:10701000013B0193D8E7FFF7E7FC801B0A28DDD985
:1070200023689B681807D9D5A36A012523F01203AA
:1070300043F01003A362002384F82430284602B0F2
:1070400070BDFFF7D1FC801B0A28D2D923689B684A
:107050005A07CED5E8E70225F0E700BF98020020E6
:1070600007490302CA6803F4E06322F4E0621204F1
:10707000120C134343F0BF6343F40033CB607047FB
:1070800000ED00E0154B30B5DC68C4F30224C4F118
:107090000703251D042B28BF0423062D4FF0FF35C1
:1070A00094BF0024033C05FA03F321EA0303A5403F
:1070B00022EA0502A340002843EA0203ACBF00F124
:1070C0006040074A4FEA0313DBB2ABBF00F56140F3
:1070D00000F00F0080F80033135430BD00ED00E0E5
:1070E00014ED00E0002807DB01234109034A00F00A
:1070F0001F00834042F82130704700BF00E100E0EC
:1071000000280CDB01220649430900F01F008240E1
:10711000203341F82320BFF34F8FBFF36F8F7047A9
:1071200000E100E00138B0F1807F0BD24FF0E023A6
:10713000F021054A586182F8231000200722986147
:107140001A6170470120704700ED00E0002808DB5D
:1071500001224309034900F01F008240603341F8D7
:107160002320704700E100E0704708B5FFF7FCFFFF
:1071700008BD704710B5044650B1437903F0FF02D3
:1071800013B90271FFF7F5FF01230020637110BDF1
:107190000120FCE710B5044668B1037903F0FF0253
:1071A00013B9427102F004F9022300202371012374
:1071B0002061237110BD0120FCE710B5044640B1E9
:1071C0000223037102F04EF90020206160712071EA
:1071D00010BD0120FCE7034630B530B342790220F0
:1071E000012A16D0187101201A6801F010041568E0
:1071F000A0402843106069B9116801F03C013C29A6
:1072000003D1516841F001015160012200201A713F
:10721000587130BD3C211068A14000F470108842C4
:10722000F3D1516841F00201EEE70120F1E70123BB
:1072300010B558B1046801F01001226803FA01F199
:1072400022EA010222600371002010BD1846FCE70B
:1072500013B50024019470B10068019041B90199FF
:10726000083100200A440192019A136002B010BD57
:1072700001991431F5E70120F8E730B503460C46D3
:1072800000B3F9B14179022001291AD040F6FE710C
:107290001871186802F010020568914025EA01058E
:1072A000D4E900142143C0249140294301600168BE
:1072B00004FA02F221EA02020260012200201A719D
:1072C000587130BD0120FCE790F821200346022AC6
:1072D00006D0042282630120002283F82020704718
:1072E0000268C06B116821F00E011160116821F075
:1072F0000101116001211A6C01FA02F242600020C2
:1073000083F82110E8E7000008B590F82130022B3F
:1073100003D004238363012008BD03681A6822F0A8
:107320000E021A601A6822F001021A60174A93428C
:107330001FD0143293421ED0143293421DD0143207
:1073400093421DD0143293421DD01432934214BF85
:107350004FF080734FF480130D4A5360012380F87F
:107360002130002380F82030436B03B19847002080
:10737000D2E70123F0E71023EEE74FF48073EBE749
:107380004FF48053E8E74FF48033E5E7080002400C
:1073900000000240114AD36813F0100305D01049D1
:1073A000CB6943F00203CB611023D268500706D5A6
:1073B0000B4943F00403CA6942F00102CA61074A5B
:1073C000D169C90708D50648C16941F00401C16106
:1073D000D16921F00101D161D360704700200240E2
:1073E000A0100020064B186910F0800007D0054A55
:1073F0005A6002F188325A601869C0F3C0107047B1
:107400000020024023016745034A0020136943F02E
:1074100080031361704700BF0020024070B505462D
:10742000FFF7E2FA0646114CE368D80712D4E36886
:10743000990644BF2023E360E368DA0606D4E369D3
:10744000DB0703D4E06810F0040007D0FFF7A2FFC9
:10745000012003E06B1CE7D00DB9032070BDFFF7DE
:10746000C3FA801BA842DFD9F7E700BF0020024023
:107470002DE9F84FDFF894A01F469AF8183005461A
:10748000012B884691463FD001234CF250308AF8B8
:107490001830FFF7C3FF90BB012D03D0022D14BF9E
:1074A0000425022500263346DFF864B03401C4F118
:1074B0002001A4F1200207FA01F129FA04F4CAF824
:1074C0001C300C4327FA02F21443DBF81020A4B25C
:1074D00042F00102CBF810204CF2503028F8164050
:1074E000FFF79CFFDBF8102022F00102CBF8102000
:1074F00028B90136F2B295424FF00003D6D80023E6
:107500008AF81830BDE8F88F0220FBE7A0100020B1
:10751000002002400022064BDA61064B1A6942F055
:1075200002021A6158611A6942F040021A617047FA
:10753000A0100020002002402DE9F041264F054612
:107540003B7E8846012B44D001243C7603684CF2F4
:107550005030022B1AD1FFF761FF20B10120002328
:107560003B76BDE8F0811D4CF86123694CF2503048
:1075700043F004032361236943F040032361FFF7D1
:107580004DFF236923F004032361E8E7FFF746FF7B
:107590000028E3D14FF0FF33C8F800302046AE6832
:1075A0000E4CD5E9023203EB8223B342D7D93046E1
:1075B000FFF7B0FF4CF25030FFF730FF236923F0A4
:1075C0000203236110B1C8F80060C8E706F58066C1
:1075D000E7E70220C5E700BFA0100020002002401E
:1075E000044A08B55169014202D0506102F028F9FD
:1075F00008BD00BF000401402DE9F341054638B342
:107600000368DB0710D42B689F075ED42B6819072B
:1076100000F195802B685A0700F1C180EB69002BBF
:1076200040F02C81002029E0904C636803F00C03AB
:10763000042B07D0636803F00C03082B0AD163689E
:10764000DE0307D523689C03DDD56B68002BDAD1F8
:10765000012013E06B68B3F5803F12D1236843F437
:1076600080332360FFF7C0F9064623689803CAD425
:10767000FFF7BAF9801B6428F7D9032002B0BDE8F0
:10768000F0819BB9236823F480332360236823F4BB
:1076900080232360FFF7A8F9064623689903B2D533
:1076A000FFF7A2F9801B6428F7D9E6E7B3F5A02F0E
:1076B000236803D143F480232360CFE723F480338E
:1076C0002360236823F48023CBE7684C636813F0BE
:1076D0000C0F07D0636803F00C03082B10D163680C
:1076E000DA030DD423689B0702D52B69012BAFD198
:1076F00023686A6923F0F80343EAC203236085E73D
:107700002A695B4B6AB101221A60FFF76DF90646E0
:1077100023689F07ECD4FFF767F9801B0228F7D98D
:10772000ABE71A60FFF760F90646236898077FF514
:107730006DAFFFF759F9801B0228F6D99DE7AA69BA
:107740004A4E4B4BE2B10122C3F88024FFF74CF9BB
:107750000446736A9B070DD54FF4FA52454B1B68DC
:10776000B3FBF2F3019300BF019B5A1E0192002B61
:10777000F9D14FE7FFF738F9001B0228E9D97CE778
:10778000C3F88024FFF730F90446736A9F077FF53A
:1077900041AFFFF729F9001B0228F6D96DE7334CFA
:1077A000E369D80024D40127E36943F08053E361FF
:1077B000E36903F080530093009B2F4E3368D90593
:1077C00018D5EB68012B26D1236A43F0010323620D
:1077D000FFF70AF941F288380646236A9B073FD52E
:1077E000002F3FF41BAFE36923F08053E36115E7FB
:1077F0000027E2E7336843F480733360FFF7F4F85F
:1078000080463368DA05DCD4FFF7EEF8A0EB080019
:107810006428F6D931E7ABB9236A41F2883823F0FE
:1078200001032362236A23F004032362FFF7DCF8D9
:107830000646236A9807D3D5FFF7D6F8801B404544
:10784000F7D91AE7052B236A03D143F00403236217
:10785000BAE723F001032362236A23F00403B6E7A7
:10786000FFF7C2F8801B4045B7D906E70010024079
:107870000000424298020020007000402A4C6268DA
:1078800002F00C02082A3ED00022022B274B1A6677
:107890002CD1FFF7A9F806462368990120D42B6A5A
:1078A000B3F5803F05D1E26AA96822F00F020A43CE
:1078B000E262696A62680B4322F474121343012284
:1078C00063601A4B1A66FFF78FF8054623689A0122
:1078D0003FF5A8AEFFF788F8401B0228F6D9CCE6A2
:1078E000FFF782F8801B0228D6D9C6E6FFF77CF89E
:1078F000054623689B017FF595AEFFF775F8401BA1
:107900000228F6D9B9E6012B3FF4A2AE60682B6AD3
:1079100000F480329A427FF49BAE6B6A00F47010E0
:10792000C01A18BF0120A9E6001002400000424220
:107930000D4A536803F00C01082912D10B48C3F318
:107940008341DB03405C09D5D36A094A03F00F0386
:107950005043084AD35CB0FBF3F07047064B5843E2
:1079600070470348704700BF00100240C8D50008A8
:1079700000127A00B8D5000800093D00F8B50546A8
:1079800008B90120F8BD0268304C12F0020F11D086
:10799000570742BF636843F4E0636360160742BF62
:1079A000636843F4605363606368816823F0F003A5
:1079B0000B436360D0071BD42A6851073FD41307D9
:1079C00006D563682A6923F4605343EAC2036360FF
:1079D000FFF7AEFF63681E4AC3F30313D35CD840BE
:1079E0001C4B18601C4B1868FEF7C2FF0020C9E74B
:1079F0006A682368012A1AD113F4003FC1D0636872
:107A000041F2883723F0030313436360FEF7ECFF72
:107A1000064663686A6803F00C03B3EB820FCBD0B1
:107A2000FEF7E2FF801BB842F3D90320AAE7022A3F
:107A300002D113F0007FE1E713F0020FDEE7636885
:107A4000E96823F4E0630B436360B8E70010024089
:107A500030D600089802002074020020044B054A2A
:107A60005B68C3F30223D35C034A1068D8407047B5
:107A70000010024028D6000898020020044B054A56
:107A80005B68C3F3C223D35C034A1068D8407047D5
:107A90000010024028D60008980200200F2303603F
:107AA0000A4B5A6802F0030242605A6802F0F00280
:107AB00082605A6802F4E062C2605B68DB0803F42B
:107AC000E063036100230B60704700BF00100240B9
:107AD000012808B503D002281FD0002013E040F28F
:107AE0000231154A136A1940B1F5817F20D003F4A1
:107AF0004073B3F5007F07D149F64040536A13F055
:107B0000020F08BF002008BDB3F5407FE5D1136820
:107B10004FF2244013F4003FF3E7FFF7AFFF064BAB
:107B20005B68C3F3813301335B00B0FBF3F0EAE73A
:107B30004FF40040E7E700BF00100240704710B567
:107B4000044600284DD0436A002B46D14268B2F566
:107B5000827F00D0C3610023A36294F8513003F008
:107B6000FF0223B9204684F85020FFF7E7FF0223E5
:107B7000216884F851300B68A06823F040030B6043
:107B8000636800F4044003F482730343E068A2696D
:107B900000F400600343206900F0020003436069C1
:107BA00000F00100034302F400700343E069120C8B
:107BB00000F038000343206A02F0040200F0800065
:107BC0000343A06A00F4005003430B60002001232C
:107BD0004A60606584F8513010BD0023C0E9043369
:107BE000B9E70120F8E70000036A026A70B522F0E5
:107BF00001020262446882690D6822F073022A431E
:107C00008D6823F002032B43104DA8420BD005F5DD
:107C1000A055A84207D005F58065A84203D005F518
:107C20008065A8420BD1CD6823F008032B4324F4D0
:107C30004074D1E90556354323F004032C434460D6
:107C400082614A684263036270BD00BF002C01403C
:107C5000036A026A70B522F4807202624468C269E3
:107C60000D6822F073022A438D6823F4007343EAFF
:107C70000523114DA8420ED1CD6823F4006343EAD9
:107C8000052323F4806324F44054D1E90556354399
:107C900044EA05140AE0094DA842F4D005F58065D0
:107CA000A842F0D005F58065A842ECD04460C261DE
:107CB0004A68C263036270BD002C0140004001406D
:107CC000036A026A30B522F4805202624468C269D3
:107CD0000D6822F4E64242EA05228D6823F400533F
:107CE00043EA05330C4DA8420BD005F5A055A84238
:107CF00007D005F58065A84203D005F58065A84248
:107D000004D14D6924F4804444EA85144460C2617E
:107D10004A680264036230BD002C014090F83D3097
:107D2000012B20D10223114A80F83D300368934291
:107D30000ED0B3F1804F0BD0A2F59432934207D00E
:107D400002F58062934203D002F59C32934204D143
:107D50009A6802F00702062A03D01A6842F001026C
:107D60001A60002070470120704700BF002C0140BE
:107D700090F83C200346012A4FF0020009D01A680F
:107D800083F83D0051610020012283F83C0083F814
:107D90003D20704770477047036870B5DD681E6905
:107DA0000446B1070DD5AA070BD56FF002021A6180
:107DB000012202779B699B0769D001F072FA0023C8
:107DC0002377710710D56A070ED56FF00402236878
:107DD00020461A61022222779B6913F4407F5CD00F
:107DE00001F05FFA0023237733070FD528070DD55D
:107DF0006FF00802236820461A6104222277DB69AB
:107E0000990750D001F04DFA00232377F20610D5E0
:107E1000EB060ED56FF01002236820461A61082287
:107E20002277DB6913F4407F43D001F03AFA002354
:107E30002377F00708D5E90706D56FF0010223681C
:107E400020461A6101F00AFA320608D52B0606D53B
:107E50006FF08002236820461A6100F048FB70062C
:107E600008D5690606D56FF04002236820461A61DE
:107E7000FFF791FFB20622D5AB0620D56FF02002A6
:107E800023682046BDE870401A6100F02FBB01F066
:107E900006FA2046FFF77EFF91E701F000FA204640
:107EA000FFF778FF9EE701F0FAF92046FFF772FF2F
:107EB000AAE701F0F4F92046FFF76CFFB7E770BDC1
:107EC000234A036890420AD0B0F1804F07D0A2F550
:107ED0009432904203D002F58062904208D14A6801
:107EE00023F070031343CA6823F4407313430AE07A
:107EF000184A9042F7D002F580629042F3D002F522
:107F000080629042EFD04A6923F0800313430360FC
:107F10008B68C3620B6883620D4B98420BD003F5EC
:107F2000A053984207D003F58063984203D003F52D
:107F30008063984201D10B690363012343610369A4
:107F4000DB0742BF036923F001030361704700BFF1
:107F5000002C01400040014010B5044630B390F8B9
:107F60003D3003F0FF021BB980F83C2002F04CF9D1
:107F70000223206884F83D30211DFFF7A1FF012373
:107F8000002084F8463084F83E3084F83F3084F88E
:107F9000403084F8413084F8423084F8433084F82B
:107FA000443084F8453084F83D3010BD0120FCE7B2
:107FB000036A026A70B522F01002026244688269A4
:107FC0000D6822F4E64242EA05228D6823F0200380
:107FD00043EA0513114DA8420ED1CD6823F080036A
:107FE00043EA051323F0400324F44064D1E9055625
:107FF000354344EA85040AE0094DA842F4D005F56A
:108000008065A842F0D005F58065A842ECD04460B8
:1080100082614A688263036270BD00BF002C014028
:108020000040014010B590F83C300446012B1DD0B3
:10803000082A17D007D862B1042A0FD001200023E4
:1080400084F83C3010BD0C2AF8D10068FFF738FEE8
:1080500002E00068FFF7C8FD0020F0E70068FFF7C6
:10806000A7FFF9E70068FFF7F3FDF5E70220E9E76E
:1080700038B590F83C300446012B4FD00120082A37
:1080800084F83C003AD006D8BAB1042A26D000239E
:1080900084F83C3038BD0C2AF9D12068FFF710FE77
:1080A000C3690A6943F40063C361C36923F480634D
:1080B000C361C36943EA02232EE02068FFF794FD01
:1080C00083690A6943F008038361836923F0040329
:1080D00083618369134383610020D8E72068FFF739
:1080E00067FF83690A6943F400638361836923F44A
:1080F00080638361836943EA0223ECE72068FFF72A
:10810000A7FDC3690A6943F00803C361C36923F08B
:108110000403C361C3691343C361DDE70220B9E708
:1081200070B5056A046A134E24F001040462B0427B
:1081300084691AD0B0F1804F17D0A6F59436B042BA
:1081400013D006F58066B0420FD006F59C36B042DB
:108150000BD044F0010263F3071201F00A0125F08D
:108160000A0319438261016270BD24F003042243B3
:10817000F1E700BF002C0140F8B590F83C3005460F
:10818000012B0C4600F081800120082A85F83C0074
:108190005BD006D842B3042A35D0002385F83C30A2
:1081A000F8BD0C2AF9D1D1E900272B68CE68186AEE
:1081B000196A120321F480511962D96920F4005020
:1081C00021F4407141EA072102F4005266F30F31B5
:1081D0000243D9611A62DA69A16822F44062DA6165
:1081E000DA6942EA01224EE02868CB6806C9FFF747
:1081F00097FF8369A26823F00C03836183691343AB
:1082000083610020C9E72B68D1E90027186ACE688E
:10821000196A120121F010011962996920F0A00079
:1082200021F4407141EA072102F0A00266F30F3108
:10823000024399611A629A69A16822F440629A61C4
:108240009A6942EA01229A61DBE72B68D1E90021B1
:10825000186A1E6AE76826F480761E62DE691202DA
:1082600026F00306314320F4007002F4007267F335
:1082700007110243D9611A62DA69A16822F00C027F
:10828000DA61DA690A43DA61BBE7022088E710B5F0
:108290000124036A01F01F018C4023EA04030362F6
:1082A000036A8A401A43026210BD000008B539B95A
:1082B00090F83E30013B18BF012373B1012034E038
:1082C000042902D190F83F30F4E7082902D190F850
:1082D0004030EFE790F84130ECE7022331BB80F803
:1082E0003E3000680122FFF7D2FF1D4B98420BD0B1
:1082F00003F5A053984207D003F58063984203D05A
:1083000003F5806398421DD1436C43F400434364FA
:10831000134B984203D003F5A05398421BD18368B6
:1083200003F00703062B16D1002008BD042902D153
:1083300080F83F30D5E708290CBF80F8403080F83E
:108340004130CEE7B0F1804FE9D0064B9842E6D0FD
:1083500003F58063E1E7036843F001030360E3E7AB
:10836000002C014000040040FFF7A0BF08B5034601
:1083700069BB90F83E0093F84220C0B20128D2B207
:1083800052D1012A22D10222002936D183F83E207F
:1083900083F8422018680122FFF779FF234B9842A7
:1083A0000ED0B0F1804F0BD0A3F59433984207D094
:1083B00003F58063984203D003F59C3398422ED195
:1083C000836803F00703062B29D1002008BD042988
:1083D00005D190F83F0093F84320C0B2CEE70829BA
:1083E0000BBF90F8400093F8410093F8442093F8B5
:1083F00045200CBFC0B2C0B2C0E7042904D183F845
:108400003F2083F84320C5E708290BBF83F84020AD
:1084100083F8412083F8442083F84520BAE70368B5
:1084200043F001030360D0E70120CFE7002C0140B7
:1084300010B50424036A01F00F018C4023EA040301
:108440000362036A8A401A43026210BD08B529B963
:1084500090F84230012B1DD0012042E0042907D1C1
:1084600090F84330012BF7D1022380F8433014E019
:10847000082907D190F84430012BEDD1022380F870
:1084800044300AE090F84530012BE5D1022380F812
:10849000453002E0022380F8423000680422FFF7F2
:1084A000C7FF436C43F4004343640E4B98420ED025
:1084B000B0F1804F0BD0A3F59433984207D003F569
:1084C0008063984203D003F59C33984204D18368BB
:1084D00003F00703062B03D0036843F00103036096
:1084E000002008BD002C0140FFF7B0BF7047704767
:1084F000026802F10C0353E8003F23F490730C323E
:1085000042E8003102680029F2D102F1140353E875
:10851000003F23F0010302F1140C4CE80031002964
:10852000F3D1036B012B0BD102F10C0353E8003F95
:1085300023F0100302F10C0C4CE800310029F3D1B8
:10854000202380F8423000230363704710B50446AF
:108550000268C168136923F440530B4313618368B5
:108560000069D1680343606921F416410343E0695F
:1085700021F00C0103430B43D3605369A16923F439
:1085800040730B4353611A4B9A4220D1FFF776FA9E
:108590001923E1695843D4E90023B1F5004F4FF0A6
:1085A000640117D15B00B0FBF3F0B0FBF1F401FB09
:1085B0001400C3003233B3FBF1F303F007015B0097
:1085C00001EB041103F4F8730B44936010BDFFF743
:1085D00045FADDE79B00B0FBF3F0B0FBF1F401FBE3
:1085E00014031B013233B3FBF1F303EB0413ECE789
:1085F00000380140704710B5044648B390F8413048
:1086000003F0FF021BB980F84020FFF7F3FF24239B
:10861000226884F84130D368204623F40053D360A5
:10862000FFF794FF236800201A6922F490421A6130
:108630005A6922F02A025A61DA6842F40052DA607A
:108640002023606484F8413084F84230606310BDB8
:108650000120FCE710B5044668B390F8413003F000
:10866000FF021BB980F84020FFF7C4FF24232268D3
:1086700084F84130D368204623F40053D360FFF7D9
:1086800065FF236800201A6922F490421A615A6932
:1086900022F022025A615A6942F008025A61DA68ED
:1086A00042F40052DA602023606484F8413084F898
:1086B0004230606310BD0120FCE790F84130202B70
:1086C00010D189B182B1C284828400232122016247
:1086D0000168436480F84120CA68184642F080026D
:1086E000CA607047022070470120704708B5002318
:1086F000406AC385C38401F07DFF08BD704790F8D0
:10870000423007B5222B42D181680268B1F5805F03
:10871000836A3FD1016900293FD15268C2F3080240
:1087200023F8022B8362C38D013B9BB2C385002BD0
:108730002DD10268D16821F02001D160D16821F4E7
:108740008071D160516921F001015161202280F8CE
:1087500042204363026B012A026828D1036302F1BD
:108760000C0353E8003F23F0100302F10C0C4CE81B
:1087700000310029F3D11368DB0605D50191136898
:10878000019353680193019B818DFFF7B7FF03B0FD
:108790005DF804FB39B9016929B95268D2B21A707F
:1087A000836A0133BEE7526802F07F02F7E701F007
:1087B0001BFFECE7036873B51A6804461607D9680F
:1087C0005D6908D1960668D58D0666D502B0BDE80C
:1087D0007040FFF794BF05F0010001F49075054368
:1087E0005BD0D60705D5CD0542BF636C43F00103CE
:1087F0006364530704D518B1636C43F002036364E8
:10880000960704D518B1636C43F00403636415073D
:1088100007D501F0200303431EBF636C43F0080338
:108820006364636C002B32D0920604D58B0602D5AC
:108830002046FFF764FF266820467369626C03F0E8
:10884000400302F0080253EA020522D0FFF750FE6F
:1088500073695E0618D5226802F1140353E8003FDD
:1088600023F04003143242E800310029F3D1E06BD9
:1088700050B1744B4363FEF747FD40B1E06B436B6F
:1088800002B0BDE870401847204601F0B3FE02B0C8
:1088900070BD01F0AFFE6564F9E7206B012840F080
:1088A0009480D50640F19180C80640F18E80002268
:1088B00001921A6801925A680192019A5A69520605
:1088C0004DD5E16B0A68526892B2002ADFD0A08DC4
:1088D0009042DCD9E2858A69202A36D003F10C0265
:1088E00052E8002F22F4807203F10C0040E80021CE
:1088F0000029F3D103F1140252E8002F22F0010203
:1089000003F1140040E800210029F3D103F114021F
:1089100052E8002F22F0400203F1140040E8002149
:108920000029F3D1202284F84220216303F10C02B4
:1089300052E8002F22F0100203F10C0040E8002161
:108940000029F3D1E06BFEF7BFFC02236363E38DE4
:10895000A18DC91A89B22046FFF7D0FE97E7E28DB4
:10896000E08DA18D80B292B2002890D0891A89B290
:1089700000298CD003F10C0252E8002F22F49072EF
:1089800003F10C0545E800200028F3D103F114029F
:1089900052E8002F22F0010203F1140545E80020FF
:1089A0000028F3D1202284F84220206303F10C0236
:1089B00052E8002F22F0100203F10C0545E80020D8
:1089C0000028F3D102236363C5E7160628D50D06F8
:1089D00026D594F84120212A7FF459AFA168226A54
:1089E000B1F5805F17D12169A9B932F8021BC1F333
:1089F000080159602262E28C013A92B2E284002AB4
:108A00007FF445AFDA6822F08002DA60DA6842F07B
:108A10004002DA603BE7511C216212785A60EAE7B3
:108A200050067FF534AF4A067FF531AFDA6820464D
:108A300022F04002DA60202384F8413001F0D7FDB3
:108A400025E700BFED86000890F84030012B11D0DB
:108A50002423026880F84130D36823F00C0343F0EC
:108A60000803D360202380F84130002380F8403091
:108A7000184670470220704790F84030012B11D003
:108A80002423026880F84130D36823F00C0343F0BC
:108A90000403D360202380F84130002380F8403065
:108AA000184670470220704790F8412090F8420025
:108AB000104370470023C2854364222382850269E4
:108AC00080F84230816203681AB1DA6842F4807239
:108AD000DA605A69002042F001025A61DA6842F015
:108AE0002002DA60704770B490F84260202E06D100
:108AF00041B13AB10024046370BCFFF7DBBF022030
:108B000070BC70470120FBE7836810B504462BB1A9
:108B10000322014698470023C4E9023310BD83684D
:108B200010B5044613B1032201469847204610BDF4
:108B30004B1E032B00D9FEE78900081F7047000079
:108B40000139435C13F0100004D0022916D80C4AF6
:108B500032F81100DB0712D503290FD8DFE801F046
:108B60000205080B40F00100704740F0100070470C
:108B700040F48070704740F480507047FEE77047C3
:108B8000E0D500080139032900D9FEE7014B585C04
:108B9000704700BFDCD500080139032900D9FEE782
:108BA000014B585C704700BFD8D500082DE9F04153
:108BB0000E460446FFF7BCFF06F10608054631469F
:108BC000204604EB0818FFF7DDFFD8F808302BB17A
:108BD000C24323691A61DA680243DA60771E04EB44
:108BE00047039B880B2B49D8DFE803F0511818186E
:108BF000060618184A4A4A2AE35DDE0604D52946C5
:108C000004F11000FFF770FCE35DD80736D5294664
:108C100004F11000BDE8F041FFF7A6BBE35DD90603
:108C200004D5294604F11000FFF710FCE35DDA07D4
:108C300024D5294604F11000BDE8F041FFF736BB0A
:108C4000294604F11000FFF791FB31462046FFF75B
:108C5000A3FF014606462046FFF772FF25692B6AEF
:108C60001843D8F80830286243B131462046FFF750
:108C700089FFC3432B61EB681843E860BDE8F081CE
:108C8000294604F11000BDE8F041FFF76FBB2369EE
:108C90001B68DB07F2D404F11000BDE8F041FFF7D8
:108CA0003DB870B5012504462946861C36F8023FBA
:108CB00023B129462046FFF779FF00210135052D14
:108CC000F4D1A36E3BB16FF0010223691A61DA6837
:108CD00042F00102DA6049B123691B68DB0705D461
:108CE00004F11000BDE87040FFF718B870BD000037
:108CF0002DE9F0438DB0044698460F46FFF718FF64
:108D00004FF6FF731646059305462369C0B95B6BA2
:108D1000002206930123CDE902329DF85030CDE9BF
:108D20000922079208920B92019204930B2E1DD8F0
:108D3000DFE806F00F1545484A5355575B59626402
:108D4000042801D19B6BE3E708280CBFDB6B1B6C8D
:108D5000DEE705922A4605A904F1100004E010237D
:108D60002A46059305A9E018FFF75CF9013F04EBDB
:108D700047039E8006B3B8F1FF3F1DD0404601F087
:108D80009FFAA84264D140463249083E01F04EF8AD
:108D9000032E05D8404602F09DFB002102F01CFD89
:108DA00040462C4901F07CF810F4801F0CBF0122D2
:108DB0001022E35D1343E3550DB0BDE8F08320239B
:108DC0000593C7E73023FBE760232A4605A904F192
:108DD00010000593FFF74CF9C8E77023F5E750231F
:108DE000EEE74023ECE7022301932A4601A904F1B0
:108DF0001000FFF7C1F9B9E70A23F5E74046154926
:108E000001F04EF810F4801000D0FEE7012304F1C9
:108E100010092A46019001A948460293FFF7ACF9D0
:108E200039462046FFF7B8FE431EE25C014642F099
:108E30000102E2540B2204EB43039A8002232046F2
:108E4000CDE90133FFF774FE01A902464846D0E799
:108E5000FEE700BFF0D70008013903299ABF00EBF5
:108E6000410080880020704701211030FEF780BF4C
:108E70000369186800F00100704710B502460C46FF
:108E8000FFF7F6FF80B9CB68DB070ED5CB6810463D
:108E900023F00103CB60FFF7E7FF6FF001032361CD
:108EA000E36843F00103E36010BD1046BDE81040E5
:108EB000FFF7DABF1D4A0346904224D0B0F1804F3D
:108EC00023D0A2F59432904221D002F580629042E4
:108ED0001FD002F5006290421DD002F580629042E0
:108EE0001BD002F59632904219D002F58062904272
:108EF00017D04FF6FF700E4A934214D04FF6FF730F
:108F0000984211D1FEE70020F5E70120F6E70220A4
:108F100070470320704704207047052070470620E3
:108F20007047072070470820704700BF002C0140A1
:108F300000480140014670B5044651F8100FFFF794
:108F4000B9FF0546084601F077F80023084A04F106
:108F5000600642F82530E36004F1B005B54204D064
:108F6000103D2846FFF7DBFDF8E7204670BD00BF47
:108F7000C0100020F8B504460846FFF79BFF2369A0
:108F800003B1FEE71B4D04F10C0245F820200E2230
:108F900004F110063046C4E90C33C4E90E33C4E9C9
:108FA0001033C4E91623216184F82C30A36484F8BB
:108FB0004C3084F84D30E46000F0ACFF04F1600503
:108FC00004F1B00728461035FFF79EFDBD42F9D1E8
:108FD00000234FF6FF72C4E90033C4E90632C4E946
:108FE0000833A360636180233046A362BDE8F84084
:108FF000FEF7B2BFC010002010B586B014220446A0
:10900000002101A802F0A0FE0023694601A80093F8
:10901000FEF744FD206901F01FF9012802D0022863
:109020000FD0FEE7049CFEF719FDB4F5C06F05D024
:109030000BD824F48074B4F5806F00D1400006B0E2
:1090400010BD059CFEF71AFDEFE7B4F5E06FF4E7FD
:10905000012A38B505460C460BD0022A16D004B1B9
:10906000013C29692846CC62EC61BDE83840FFF735
:1090700004BFFFF7C1FF084BB0FBF3F044432A697C
:10908000230C93620133B4FBF3F4E8E7FFF7B4FF7A
:10909000B0FBF4F4F3E700BF40420F00F8B505461B
:1090A00014461A46FFF744FD2B69822A9E6A07463A
:1090B00006F1010629D01FD8102A11D852BB4FF64D
:1090C000FF722969CB6A934203D1B4F5803F08BF90
:1090D0001C4637BB4C632846BDE8F840FFF7CDBEC1
:1090E000812AECD12846FFF787FF124BB0FBF3F043
:1090F0006043B0FBF6F4E2E7832AE0D1DB6A03FBCE
:1091000004436424B3FBF4F4D9E72846FFF774FF63
:109110006643EEE7DB6A03FB044301249440013C11
:10912000F0E7042F01D18C63D5E7082F0CBFCC6387
:109130000C64D0E740420F0010B5074C206810B116
:109140000430FEF729FEE06920B1BDE8104004308C
:10915000FEF722BE10BD00BFC0100020034B1868F0
:1091600010B10430FEF718BE704700BFC0100020D9
:10917000034B586810B10430FEF70EBE704700BFB5
:10918000C0100020034B986810B10430FEF704BEF5
:10919000704700BFC0100020034BD86810B10430E6
:1091A000FEF7FABD704700BFC0100020034B1869DE
:1091B00010B10430FEF7F0BD704700BFC0100020B2
:1091C000034B586910B10430FEF7E6BD704700BF8D
:1091D000C0100020034B986910B10430FEF7DCBDCD
:1091E000704700BFC0100020034B186A10B1043054
:1091F000FEF7D2BD704700BFC01000200022C0E9BA
:109200000022C0E902227047F8B504460E4600F17C
:10921000600500F1B00728461035FFF7EFFFBD42AB
:10922000F9D10023204631462361FFF7A3FE2046F3
:10923000F8BD826810B50AB903F0C0FCC368BDE888
:109240001040184708B500B9FEE700F061FE00685D
:10925000836E13B16030FFF7ECFF08BDFFF7F2BF7C
:1092600010B500B9FEE7037F013B072B10D8DFE8FC
:1092700003F004140F100F0F0F12012400F048FE2A
:109280000068063400EB041083680BB1FFF7D1FFD0
:1092900010BD0324F2E70424F0E70224EEE7FFF711
:1092A000DFBFFFF7DDBF02F069BB02F06FBB00005C
:1092B00086B0042841D8DFE800F003101C283400F1
:1092C0001F4B20489A6942F004029A619B6903F09F
:1092D00004030193019B06B07047194B1A489A6921
:1092E00042F008029A619B6903F008030293029B13
:1092F000F1E7134B15489A6942F010029A619B6995
:1093000003F010030393039BE5E70D4B10489A69A4
:1093100042F020029A619B6903F020030493049BAE
:10932000D9E7074B0B489A6942F040029A619B6962
:1093300003F040030593059BCDE70020CBE700BF7A
:109340000010024000080140000C014000100140E4
:10935000001401400018014008B5044900F0A0FDC8
:10936000C0F3C430112800D9FEE708BD9CDA00081C
:1093700041F20103984204D041F20203984202D024
:10938000FEE71020704711207047000008B507491C
:1093900000F086FDC0F3C430012802D0022802D0BC
:1093A000FEE7002008BD1020FCE700BF78DA0008C7
:1093B00002680A4B82B09A420AD103F5CE33DA69C9
:1093C00042F00052DA61DB6903F000530193019B24
:1093D000034B0449186802B000F028BD0074004037
:1093E0008C02002078DA0008F0B589B005460E46F8
:1093F00017460021142203A802F0A6FC00232846E9
:109400001649CDE9013300F029FD039018B3284631
:10941000FFF7BCFF30F0100304461CD1012F0BD026
:1094200033460022214603A8FDF712FF98B92146D2
:1094300003A8FDF7D0FE0EE0094B03A81D60FDF761
:10944000A9FE40B9CDE90100224601A903A8FDF714
:1094500014FF0028E4D009B0F0BD00BF78DA00089E
:109460008C0200200268094B9A420DD103F5CE33DD
:109470001A6942F000521A611A6922F000521A6108
:10948000DA6922F00052DA61704700BF00740040D0
:1094900010B50B4986B0044600F0E0FC019060B1C5
:1094A0002046FFF773FF30F01003014605D101A8F5
:1094B000FDF7BDFE01A8FDF780FE06B010BD00BFA0
:1094C00078DA000802680C4B82B09A420AD103F5A0
:1094D0006C439A6942F400729A619B6903F40073C9
:1094E0000193019B054B1868C30403D4044902B0DF
:1094F00000F09CBC02B07047002401408C020020A8
:109500009CDA00080268094B9A420DD103F56C43BE
:10951000DA6842F40072DA60DA6822F40072DA6023
:109520009A6922F400729A61704700BF00240140DA
:10953000F0B593B004463022002106A802F004FCE6
:109540000023E204CDE903330593ADF8063002931E
:1095500057D541F202039C4253D8324B2046069322
:10956000FFF706FF07260546002301274FF4602278
:10957000CDE907338DF824308DF82C300C931093FF
:109580000E938DF83C30284B06A80A970D921C606C
:10959000FDF7FEFB002840D1112D03953DD803A90E
:1095A00006A8CDE90476FDF7CDFA002835D106A846
:1095B000FDF7E6FC002830D106A8FDF77FFB60BB75
:1095C0000A2106A8FDF716FA38BB06A8FDF738FBF6
:1095D000830505D506A8FDF7B1FA80B2ADF80600FF
:1095E00006A8FDF7B3FCC0B906A8FDF74FFCA0B96B
:1095F0000C4A936823F400039360BDF8060080B220
:109600000CE00A49204600F029FC02A906902046F9
:10961000FFF7A2FE069B054613B9002013B0F0BD6C
:109620000226A1E7002401408C0200209CDA0008F9
:109630002DE9F3478A46254999469046064600F0AB
:109640000DFCFFF737FC224F044657F8203073B962
:10965000B020FFF728FE1D490546304600F0FEFB0E
:1096600001462846FFF7D0FD57F824301D6057F813
:109670002430164930461C6800F012FCC0F3C43593
:1096800029462046FFF7E8FB0428074607D00023B9
:1096900004220093294633462046FFF729FB022285
:1096A00051462046FFF7D4FC4B4642462946204609
:1096B000FFF7F4FC042F05D0204602B0BDE8F047C8
:1096C000FFF7EFBA02B0BDE8F08700BFF0D700089F
:1096D000C0100020F8B51449074600F0BFFBFFF7A3
:1096E000E9FB124E044656F8203073B9B020FFF75C
:1096F000DAFD0D490546384600F0B0FB0146284624
:10970000FFF782FD56F824301D6056F824301C689F
:1097100044B12046FFF70EFC2046BDE8F840B021DA
:10972000FFF7C3BDF8BD00BFF0D70008C010002090
:1097300037B54FF0E025FDF757F9AB6904460093C4
:10974000FDF752F9AB698442019369694FF47A736A
:1097500001F1010108D0019A8A1A5A43B2FBF1F2D1
:1097600003FB002003B030BD009A8A1A5A43B2FBB3
:10977000F1F203FB0420F5E7FDF736B9704708B5B1
:10978000FDF726F9FDF7F1FCFFF7F8FF08BD70477C
:109790000F4B84B0DA6942F08052DA61DA6902F084
:1097A00080520192019A9A6942F001029A619A6983
:1097B00002F001020292029A5A6942F040025A6192
:1097C0005B6903F040030393039B04B0704700BF41
:1097D000001002400C4BD3F8FC20D2015EBFD3F83E
:1097E000FC2042F08072C3F8FC200022074B5A6034
:1097F0001A6842F001021A6000BF00BF00BF58683B
:10980000B0FA80F04009704700ED00E0001000E081
:1098100008B5FFF7BDFFFFF7DDFFFDF7CDF8FFF758
:10982000B6FF00F077FFBDE808400148FDF7A2BC95
:10983000900200200023C0E90033C0E902337047E2
:109840000023012803F101020AD11422DBB25343A1
:10985000054A181D1044816829B11A441369184734
:1098600013464008EDE77047E41000200120FDF7A3
:10987000B7BE0220FDF7B4BE0420FDF7B1BE08203C
:10988000FDF7AEBE1020FDF7ABBE38B50524202590
:10989000A8B2FDF7A5FE013C4FEA4505F8D138BD59
:1098A00038B506244FF48065A8B2FDF799FE013C57
:1098B0004FEA4505F8D138BD344A08B510460623AD
:1098C00000F8043BFFF7B6FF072302F118001375F9
:1098D000FFF7B0FF082302F12C0082F82830FFF7D1
:1098E000A9FF092302F1400082F83C30FFF7A2FFF4
:1098F0000A23172102F1540082F85030FFF79AFF33
:1099000002F1680082F86410FFF794FF02F17C0016
:1099100082F87810FFF78EFF02F1900082F88C1029
:10992000FFF788FF02F1A40082F8A010FFF782FF82
:1099300082F8B410282102F1B800FFF77BFF02F192
:10994000CC0082F8C810FFF775FF02F1E00082F842
:10995000DC10FFF76FFF02F1F40082F8F010FFF760
:1099600069FF02F5847082F80411FFF763FF02F5C6
:109970008E7082F81811FFF75DFFBDE8084002F510
:10998000987082F82C11FFF755BF00BFE41000203B
:1099900038B5054CA4F5A075143C201DFFF7BFF8A1
:1099A000AC42F9D138BD00BF241200209F4B82B0D9
:1099B0009A69013842F001029A619B6903F0010340
:1099C0000193019B2F2838D8DFE810F030003900D0
:1099D000400047004C00530058005F0064006B00DB
:1099E00074007900800089008E0095009E00A70019
:1099F000AC00B300BC00C100C8003700370037001E
:109A0000CD00D4003700370037003700D900DE0022
:109A1000E500EC00F300F900FE00030108010D0170
:109A2000120117011C01210126012B01804A5368F4
:109A300043F0E06343F00103536002B070477C4A97
:109A4000536823F0010343F0E063F5E7784A536875
:109A500043F0E06343F00203EEE7754A536823F0F6
:109A60000203F0E7724A536843F0E06343F00403F3
:109A7000E2E76F4A536823F00403E4E76C4A536853
:109A800043F0E06343F00803D6E7694A536823F0E4
:109A90000803D8E7664A536843F0E06343F03003B5
:109AA000CAE7634A536823F0300343F0E06343F0AE
:109AB0001003C1E75E4A536823F03003C3E75C4AF2
:109AC000536843F0E06343F0C003B5E7584A536876
:109AD00023F0C00343F0E06343F04003ACE7544A93
:109AE000536823F0C003AEE7514A536843F0E06384
:109AF00043F44073A0E74E4A536823F4407343F0A5
:109B0000E06343F4007397E7494A536823F44073D2
:109B100043F0E06343F480738EE7454A536823F4CF
:109B2000407390E7424A536843F0E06343F4406374
:109B300082E73F4A536823F4406343F0E06343F411
:109B4000006379E73A4A536823F440637BE7384A75
:109B5000536843F0E06343F480536DE7344A53683D
:109B600023F480536FE7324A536843F0E06343F4D1
:109B7000004361E72E4A536823F4004363E72C4A0D
:109B8000536823F0E06357E7294A536823F0E06302
:109B900043F0807350E7264A536823F0E06343F0B4
:109BA000007349E7224A536823F0E06343F080637F
:109BB00042E71F4AD36943F00103D3613DE71C4AE2
:109BC000D36923F00103F8E7194AD36943F002038C
:109BD000F3E7174AD36923F00203EEE7144AD36987
:109BE00043F00403E9E7124AD36923F00403E4E7EE
:109BF0000F4AD36943F00803DFE70D4AD36923F026
:109C00000803DAE70A4AD36943F01003D5E7084AA4
:109C1000D36923F01003D0E7054AD36943F4006306
:109C2000CBE7034AD36923F40063C6E70010024080
:109C30000000014091FAA1F3B3FA83F370B50D0E61
:109C40000F2691FAA1F1B1FA81F144599B0006FA6D
:109C500003F3890024EA03048A402243425170BD81
:109C600091FAA1F3B3FA83F370B50D0E042691FABD
:109C7000A1F1B1FA81F144599B0006FA03F389007E
:109C800024EA03048A402243425170BD431C04D09D
:109C90000C3151F80C3C5A1C01D100207047834212
:109CA00001F10C01F5D1012070470000431C2DE9A2
:109CB000F34106460F4600D1FEE7594B00F00F0274
:109CC000C0F3031001F0070853F82240FFF7F0FA41
:109CD000B8F1010F054615D194FAA4F3B3FA83F352
:109CE0000321200E2A589B0001FA03F322EA030203
:109CF00094FAA4F3B3FA83F39B00994011432950DB
:109D0000012213E0C7F30620B8F1030F0AD801A31C
:109D100053F828F0279D0008019D00088B9D00083E
:109D2000999D0008FEE7FFF741FE082221462846DC
:109D300008F1FF38FFF77EFFB8F1010F06D817F0E2
:109D4000080218BF04222146FFF78AFF94FAA4F202
:109D5000230EB2FA82F2E9580F239200934094FA4C
:109D6000A4F2B2FA82F2C7F301170B409200012F5E
:109D700023FA02F312D0022F3BD0082B21D1042268
:109D800021462846FFF756FF1BE07F2801D1092214
:109D9000CCE7FFF70BFEFAE70022C7E7042B04D15C
:109DA000082221462846FFF745FF230A93FAA3F32A
:109DB000B3FA83F20123E968934021EA14210B43AB
:109DC000EB60184B9A6942F001029A619B6903F0BB
:109DD00001030193019BA6F10D03012B14D8124A34
:109DE000536823F0E06343F08063536002B0BDE842
:109DF000F081042B04D1082221462846FFF71AFFE0
:109E0000EB6823EA1423DBE70F2E02D0133E012E6A
:109E1000ECD8054A536823F0E06343F00073E4E7AD
:109E2000E8D500080010024000000140431C06D1A4
:109E30007047834202D18968FFF738BF0C310B6845
:109E40005A1CF6D1FEE70B685A1C01D1002070475E
:109E5000834201D1486870470C31F4E7431C01D0BC
:109E6000FFF7F1BF002070474B6813B94FF0FF3088
:109E70007047834201D1086870470C31F4E708B19C
:109E8000FFF7F2BF4FF0FF30704703460868421CEF
:109E900000D17047984201D1886870470C31F5E7CE
:109EA000431C01D0FFF7F1BF704703468B420846C1
:109EB00004D01BB100290CBF1846002070470000D9
:109EC000104B1A6842F001021A6059680E4A0A40A3
:109ED0005A601A6822F0847222F480321A601A687A
:109EE00022F480221A605A6822F4FE025A604FF46B
:109EF0001F029A600022DA624FF00062034B9A6000
:109F0000704700BF001002400000FFF800ED00E0C5
:109F10000438704703683F4A8AB0934218D102F56B
:109F20006442916941F400619161926902F40062B6
:109F30000192019A384A934217D1384BDA6942F0BC
:109F40002002DA61DB6903F020030693069B5FE0E1
:109F5000B3F1804F17D1314AD16941F00101D1618C
:109F6000D26902F001020292029A2D4A934218D15C
:109F70002A4B9A6942F480329A619B6903F48033D8
:109F80000793079B44E0274A934218D102F5033216
:109F9000D16941F00201D161D26902F0020203925B
:109FA000039A214A934218D11C4B9A6942F4003219
:109FB0009A619B6903F400330893089B28E01B4ACD
:109FC000934218D102F50232D16941F00401D16106
:109FD000D26902F004020492049A154A934217D1FE
:109FE0000E4B9A6942F480229A619B6903F48023A4
:109FF0000993099B0CE00F4A93429BD1074BDA6906
:10A0000042F01002DA61DB6903F010030593059B4F
:10A010000AB07047002C01400014004000100240BC
:10A02000004001400004004000440140000800409E
:10A0300000480140001000400368274A93420DD1B8
:10A0400026498A6922F400628A61254A93420DD129
:10A0500002F5FE32D36923F020033BE0B3F1804FD9
:10A060000ED11E49CA6922F00102CA611D4A9342FB
:10A070000ED102F55042936923F480339361704707
:10A08000194A93420DD11549CA6922F00202CA61E8
:10A09000164A93420DD102F54C42936923F40033E2
:10A0A000ECE7134A93420DD10C49CA6922F004022D
:10A0B000CA61104A9342E2D102F54842936923F4FF
:10A0C0008023DBE70C4A9342BFD102F50032D3690B
:10A0D00023F01003D3617047002C014000100240B0
:10A0E00000140040004001400004004000440140D2
:10A0F000000800400048014000100040431C26D0EA
:10A100001B4B984226D010D8A3F54063984223D029
:10A1100007D8B0F1804F21D0A3F5806398421FD0BB
:10A12000FEE7144B98421DD0FAE7134B98421BD020
:10A1300008D8A3F5C053984216D003F5A05398420F
:10A1400014D0EDE70D4B9842EAD11A2070476FF01A
:10A150000D007047372070471E2070471C20704745
:10A160001D2070473620704719207047182070470F
:10A17000001400400010004000440140004801402D
:10A18000431C26D01C4B984226D010D8A3F5406320
:10A19000984223D007D8B0F1804F21D0A3F5806337
:10A1A00098421FD0FEE7154B98421DD0FAE7144B9A
:10A1B00098421BD008D8A3F5C053984218D003F595
:10A1C000A053984216D0EDE70E4B9842EAD11A20E0
:10A1D00070476FF00D007047372070471E207047A2
:10A1E0001C2070471D20704736207047192070478B
:10A1F0001B207047182070470014004000100040DA
:10A20000004401400048014038B50446FFF782FE93
:10A210000068FFF773FFD4E91212FCF733FF2068E0
:10A22000FFF76CFFFCF75EFF22681046FFF7A8FF00
:10A2300005461046FFF762FF85420BD0D4E91212A3
:10A240002846FCF71FFF2068FFF79AFFBDE838405B
:10A25000FCF748BF38BD0000431C24D0144B984283
:10A2600023D00ED8A3F5406398421ED005D820F421
:10A270008060B0F1804F18D0FEE70E4B984214D0AA
:10A28000FAE70D4B98420CD008D8A3F5C05398427A
:10A2900007D003F5A053984203D0EDE7074B98424F
:10A2A000EAD102207047002070470120704700BFAC
:10A2B00000140040001000400044014000480140EC
:10A2C00008B50649FFF7ECFDC0F3C430431E032B6D
:10A2D00000D9FEE78000043808BD00BFF0D70008B1
:10A2E0002DE9F04F87B09846109B04468A46406D92
:10A2F000624991460193FFF7B1FD61498346A06D24
:10A30000FFF7ACFD5F490646E06DFFF7A7FD5E492C
:10A310000546206EFFF7A2FD0746BBF1000F00F0D7
:10A32000A980A26D013202D0002E00F0A380E26D60
:10A33000013202D0002D00F09D80226E013202D049
:10A34000002F00F0978031465846FFF7AEFD2946B2
:10A350002060FFF7AAFD39462060FFF7A6FD2060C8
:10A36000002800F08780494B98424CD103F55843B0
:10A37000DA6842F48042DA60DA6822F48042DA6015
:10A380009A6942F480429A619B6903F48043039383
:10A39000039B2523A4F864303849606DFFF746FD20
:10A3A0001EB13749A06DFFF741FD2DB13549E06D74
:10A3B000FFF73CFD4FF480752FB13349206E45F413
:10A3C0000075FFF733FD94F86520314B271D43F8E6
:10A3D000227023680022C4E9013A019B94F96400C9
:10A3E000C4E904380C230121C4E90635C4F80C90F3
:10A3F0002262FCF747FE3846002E36D107B0BDE892
:10A40000F04FFEF727B9234B984215D103F5E633F9
:10A410001A6942F400321A611A6922F400321A6190
:10A42000DA6942F40032DA61DB6903F40033049341
:10A43000049B4FF49373ADE7174B9842ACD103F5EF
:10A44000E4331A6942F480221A611A6922F48022E4
:10A450001A61DA6942F48022DA61DB6903F480234D
:10A460000593059B40F2272394E707B0BDE8F04F22
:10A47000FEF7C1B807B0BDE8F08F00BFB4D7000841
:10A4800078D700083CD7000800D700080038014002
:10A4900024120020004400400048004010B4019CF9
:10A4A00018B1019410BCFFF71BBF10BC704700002F
:10A4B00008B5074B90F8652053F82200FEF7F4FA30
:10A4C00000F02200A0F122035842584108BD00BF0D
:10A4D0002412002008B5074B90F8652053F822009D
:10A4E000FEF7E2FA00F02100A0F1210358425841A2
:10A4F00008BD00BF2412002070B50E46054610B9F5
:10A500004FF0FF3070BDFFF7D3FF04460028F7D1AE
:10A51000294611F8663F0122337095F86500034B18
:10A5200053F82000FEF7DFFA2046EBE72412002064
:10A5300038B50D460446B8B1FFF7BAFFA0B994F993
:10A540006400E564FCF7DCFD94F86500074B04F15A
:10A55000660153F820000122FEF7C5FA94F9640061
:10A56000BDE83840FCF7BEBD38BD00BF2412002056
:10A5700038B515460446B8B1016590F96400FCF79A
:10A58000BFFDB4F87630E16E9BB294F865001944D3
:10A59000064BAAB253F82000FEF78FF894F9640036
:10A5A000BDE83840FCF79EBD38BD00BF2412002036
:10A5B00048B1836D013306D190F86520024B53F802
:10A5C0002200FEF741BA70472412002048B1836D83
:10A5D000013306D190F86520024B53F82200FEF7B4
:10A5E0004BBA704724120020836C04381847C36CA0
:10A5F0000438184730B5044650F8043985B01D6852
:10A6000015F0010512D0002200921A6800925B68D2
:10A610000093009BFFF74CFF40BB0122204604F152
:10A62000620105B0BDE83040FEF75DBA196811F06F
:10A63000020106D001951A6801925B680193019BA3
:10A64000E8E71A6812F0040206D002911A68029232
:10A650005B680293029BDDE719680907DAD503926C
:10A660001A6803925B680393039BD3E705B030BD80
:10A6700008B52520FCF76AFD024B1868BDE80840C4
:10A68000FEF798B824120020262008B5FCF75EFDDE
:10A69000034B586818B1BDE80840FEF78BB808BDF9
:10A6A00024120020272008B5FCF750FD034B9868C2
:10A6B00018B1BDE80840FEF77DB808BD241200209F
:10A6C00003460A4910B508680344EFF30882934231
:10A6D00005D90C224FF0FF30054B1A6010BD054A1A
:10A6E000054C121B9342F4D20B60F7E79C0200204A
:10A6F000A01400200020002000040000FEE700005D
:10A700001622024B4FF0FF301A607047A014002051
:10A710000120704710B590B02022002107A801F059
:10A7200013FB0021142201A801F00EFB01221023CB
:10A730000224CDE90A234FF4801306A806940D9451
:10A740000F93FCF759FF014600B1FEE70F23CDE957
:10A750000300059001A8CDE90134FDF70FF900B120
:10A76000FEE710B010BDB0F80831B0F80421981A17
:10A7700000F03F007047B0F80831B0F804219BB2F8
:10A7800093421ABFD0F8FC30985C4FF0FF3070470E
:10A7900090F80631B0F80A01C0B2834227BFC3F176
:10A7A0003F03C018C01A00F1FF30704707B50368B7
:10A7B0008DF8071001225B680DF10701984703B07F
:10A7C0005DF804FB13B50DF107010446FFF794FE95
:10A7D00088B9B4F87430B4F87020013303F03F0343
:10A7E000934208D0B4F874209DF80700A16E92B28D
:10A7F0008854A4F8743002B010BD0000B0F8761090
:10A80000826F10B50A4402F03F02A0F87620B0F83B
:10A810007610B0F8722089B28A421AD0B0F8764029
:10A820004032A4B2B0F87610121B544289B204F040
:10A830003F0402F03F02C1F1400158BF62428A4228
:10A8400028BF0A4604498267FFF792FE4FF0FF30A7
:10A8500010BD0020FCE700BFFDA700082DE9F8436C
:10A86000036804469B68884616469847012323746C
:10A87000D4F8EC30B4F8067101338146C7F14007D3
:10A8800009D194F8103133B1002304F1940084F815
:10A890001031FFF78DFE236820469B6898470028FB
:10A8A000F9D03546AF4225D34D4523D8B4F806310B
:10A8B000D4F800015A19402A184430D82A46414693
:10A8C00001F0DAFA2F46B4F806311D4405F03F05D1
:10A8D000A4F8065104F194052846FFF7FBFD30B9B2
:10A8E0003A4628461549C4F80C71FFF741FE304638
:10A8F000BDE8F8834F4528BF4F4623683A46414696
:10A900005B6820469847236820469B689847ED1B64
:10A91000B844B4F806718146C7F14007C2E7C3F1F5
:10A9200040073A46414601F0A7FAD4F80001EA1B75
:10A9300008EB070101F0A0FAC5E700BFFDA700087A
:10A94000C0F8F030009B914208BF4FF0FF31C0F8D3
:10A95000F43000F11103C0F8FC300023C0E93A21C3
:10A9600000F15102A0F80831C0E94023A0F80A31F3
:10A970007047000073B54FF47A750026C0E9016591
:10A980003D4D069C0560CDB2242D25D83B4E01F4EB
:10A99000E06156F825502943D5B2242D30D8374EE2
:10A9A00002F4E06256F825502A43DDB2242D3BD84C
:10A9B000324E03F4E06356F825502B43E5B2242DC4
:10A9C00046D82E4E04F4E06456F825502C430094EB
:10A9D000FFF7B6FF02B070BD01F0C006C02E0CD16B
:10A9E000C92D0AD8264D01F03F0655F82660234DA3
:10A9F00001F4E06155F82650CDE74FF0FF31CBE789
:10AA000002F0C006C02E0CD1C92D0AD81C4D02F090
:10AA10003F0655F82660194D02F4E06255F82650BD
:10AA2000C2E74FF0FF32C0E703F0C006C02E0CD1E2
:10AA3000C92D0AD8124D03F03F0655F826600F4D78
:10AA400003F4E06355F82650B7E74FF0FF33B5E75E
:10AA500004F0C006C02E0CD1C92D0AD8084D04F050
:10AA60003F0655F82660054D04F4E06455F826507D
:10AA7000ACE74FF0FF34AAE7ECDB000848DB000846
:10AA800020DB0008037C70B504460D46A3B1FBF73C
:10AA9000ABFF0646B4F80621B4F80A319BB29A42DD
:10AAA0000AD0002DF8D0FBF79FFF801B8542F1D81C
:10AAB000B4F80A31A4F8063170BD0021FFF7E2BFF7
:10AAC000CBB2242B08D80E4A01F4E06152F82330AF
:10AAD0001943C0F8EC10704701F0C002C02A0CD135
:10AAE000C92B0AD8074B01F03F0253F82220044B30
:10AAF00001F4E06153F82230EAE74FF0FF31E8E774
:10AB000048DB000820DB0008CBB2242B08D80E4A13
:10AB100001F4E06152F823301943C0F8E81070479F
:10AB200001F0C002C02A0CD1C92B0AD8074B01F092
:10AB30003F0253F82220044B01F4E06153F8223025
:10AB4000EAE74FF0FF31E8E748DB000820DB0008C8
:10AB500073B54FF47A7316460022C0E901231D4BEA
:10AB6000044603604FF0FF33C0F8EC301A4B0D463B
:10AB7000984215D1C321FFF7A3FFC221FFF7C4FFFD
:10AB80004FF0FF33012E08BFC4F8EC30009320468D
:10AB9000D4E93A214FF0FF33FFF7D2FE02B070BD87
:10ABA0000E4B0F499A680F4B53F82200FFF756F9E6
:10ABB000854202D1C3212046DDE70B492846FFF735
:10ABC0005EF90749C4F8EC002846FFF758F9C4F8C5
:10ABD000E800D5E7ECDB00083012002020DB00089D
:10ABE000B4D7000848DB000878D70008D0F8EC306C
:10ABF00010B5013304460ED10368DB68984794F81A
:10AC0000103143B9012304F1940084F81031BDE8F8
:10AC10001040FFF7DBBC10BD73B5144602F007030C
:10AC2000023BDBB2042B80F8112196BF1A4A0022A6
:10AC3000D25C04F03003302B0546C0F8141107D164
:10AC40004FF4C0630132082A09D0092A1BD0FEE75D
:10AC500014F020031CD04FF480630132F3E700228C
:10AC6000C4F3C00405F19406640330460094FFF772
:10AC700015FC2846FFF7BAFF3046084902B0BDE888
:10AC80007040FFF755BC4FF48052E9E71A46E7E7FA
:10AC9000082AFBD0DBE700BFDCDB0008C5A7000803
:10ACA00010B50446FFF7A2FFB4F80821B4F8043148
:10ACB00092B29A4217BFD4F8FC204FF0FF30D05C1C
:10ACC00001331CBF03F03F03A4F8043110BD0000A2
:10ACD000002202490248FFF73BBF00BF004400408A
:10ACE0003012002070B505460C46084649B1F5F70C
:10ACF00079FA2B68024621462846BDE870405B6819
:10AD0000184770BD03688A685B680968184708B50A
:10AD1000FFF7E8FF08BD03681B68184708B502493C
:10AD2000FFF7E0FF08BD00BF66D5000838B505464F
:10AD3000FFF7D8FF04462846FFF7F0FF204438BD50
:10AD400038B50546FFF7DEFF04462846FFF7E6FF65
:10AD5000204438BDFFF7EABF38B50546FFF7DBFFF3
:10AD600004462846FFF7DAFF204438BD0023012AB5
:10AD700098BF0A2230B58BB00C468DF8243009A953
:10AD80002546B4FBF2F404FB1253DBB2092B94BF4B
:10AD900030333733DBB2AA4201F8013DF0D9FFF777
:10ADA000A1FF0BB030BD2DE9F04107460E46144619
:10ADB0002AB9BDE8F0410368C9B21B6818470A2ADE
:10ADC00005D1002905DBBDE8F041FFF7CFBFD2B2C6
:10ADD000F9E72D21FFF79FFF2246054671423846CD
:10ADE000FFF7C4FF2844BDE8F08138B50546FFF7FA
:10ADF000DAFF04462846FFF791FF204438BD10B41F
:10AE000022B9026810BC1268C9B2104710BCD2B295
:10AE1000FFF7ACBF38B50546FFF7F1FF04462846FB
:10AE2000FFF77CFF204438BD38B50546FFF7E7FF44
:10AE300004462846FFF772FF204438BD2DE9F84349
:10AE4000074608460D461646F6F7ACF938B13D49B7
:10AE50003846FFF747FF04462046BDE8F88325F053
:10AE6000004420463849F6F79DF930B92046364966
:10AE7000F6F77AF908B93549EAE728463449F6F78A
:10AE800087F908B13349E3E76FF042512846F6F7F6
:10AE900061F90028F6D100212846F6F75BF904464F
:10AEA00030B12D213846FFF736FF044605F1004545
:10AEB0004FF000084FF07C50DFF89C905FFA88F369
:10AEC0009E4239D801462846F5F79EFE8046F6F7A1
:10AED000A5F90A22014605463846FFF747FF044414
:10AEE000002EB9D02846F5F73FFF01464046F5F75A
:10AEF00089FE2E2105463846FFF70DFFDFF8588002
:10AF00000444002EA8D041462846F5F785FF814627
:10AF1000F6F784F90A22014605463846FFF726FF70
:10AF200004442846F5F720FF01464846F5F76AFE37
:10AF3000013E0546F6B2E4E74946F6F721F808F186
:10AF40000108BBE769D50008FFFF7F7F6DD50008CA
:10AF5000FFFF7F4F71D500080000204108B5D2B235
:10AF6000FFF76CFF08BD38B5D2B20546FFF766FFA4
:10AF700004462846FFF7D2FE204438BD10B50446EB
:10AF800000F0D0FCE060236820465B699847002809
:10AF900008DA00F0C7FCE368C01AA3689842F2D34D
:10AFA0004FF0FF3010BDF8B507460D460C468E1821
:10AFB000B44201D1601BF8BD3846FFF7DFFF031E26
:10AFC000F8DB04F8013BF3E72DE9F041074688463A
:10AFD00016461D4673B100243846FFF7CFFF031E07
:10AFE00005DB434503D033550134A542F4D1204657
:10AFF000BDE8F0811C46FAE710B5441A0298521ACF
:10B00000C01A444394FBF2F4E01810BD10B5044696
:10B01000006800F0BBFC204610BD10B50446006877
:10B0200008B100F0B3FC0023C4E90133236010BD74
:10B0300038B504460D460068013100F05DFD10B1E1
:10B04000C4E90005012038BD036810B5044613B1FA
:10B0500043688B4207D22046FFF7EAFF20B1A3687E
:10B060000BB922681370012010BD70B50E46114651
:10B0700004461546FFF7E8FF20B92046FFF7CDFF4D
:10B08000204670BD31462068A56000F0EDFEF7E770
:10B0900038B5002304460D46C0E90033836039B15A
:10B0A0000846F5F79FF8294602462046FFF7DDFFE0
:10B0B000204638BD38B5054600680C46096830B1F1
:10B0C00019B16A68A3689A420BD200F05FFC23684A
:10B0D0002B6063686B60A368AB600023C4E9003336
:10B0E00003E000F0C1FEA368AB600023A36038BD9D
:10B0F000884210B50B46044604D0096821B19A680D
:10B10000FFF7B3FF204610BDFFF787FFFAE70023E4
:10B1100010B50446C0E900338360FFF7E9FF20461D
:10B1200010BD884210B5044601D0FFF7C3FF20468A
:10B1300010BD38B505460C4649B10846F5F752F83A
:10B14000214602462846FFF790FF284638BDFFF704
:10B1500064FFFAE710B5002304468AB0C4E900335F
:10B16000A360084601A900F071F9204601A9FFF784
:10B17000E0FF20460AB010BD10B5002304468AB097
:10B18000C4E90033A360084601A900F08FF9204606
:10B1900001A9FFF7CEFF20460AB010BD002370B50D
:10B1A00015468CB00446C0E900338360961C0846FF
:10B1B000F5F784F976B203AB324600932B4600F0E4
:10B1C00059F801462046FFF7B4FF20460CB070BD89
:10B1D00070B504460E46856809B9002070BD62B19D
:10B1E00015442946FFF730FF0028F6D02068A368F1
:10B1F0003146184400F038FEA5600120EEE7002338
:10B2000007B501228DF8041001A98DF80530FFF76C
:10B21000DFFF03B05DF804FB10B58A6809680446D7
:10B22000FFF7D6FF10B92046FFF7F7FE204610BD06
:10B2300038B504460D4621B92046FFF7EEFE2046FC
:10B2400038BD0846F4F7CEFF294602462046FFF7F0
:10B25000BFFF0028F0D0F2E783688B4201D9006875
:10B2600018B900230248037070470844704700BFB4
:10B27000481300202DE9F04F1446A7B01F460022C6
:10B28000002380468946F5F7E3FB309D064618B15A
:10B2900009F10043994601264FF0000A0020464973
:10B2A000574571DC02460B4640464946F4F7A8FF75
:10B2B00002460B46CDE90223F5F730FC8246002F0B
:10B2C0006BD04FF0000B4FF00008DFF8F0904046D5
:10B2D000494600223A4BF5F749F90BF1010B5F455E
:10B2E00080468946F3DC5046F5F7C6F802460B4621
:10B2F000DDE90201F4F782FF42464B46F5F736F9E5
:10B30000F5F7E4FB3B4652460090002E43D02D4912
:10B31000284600F0DFFC8122002105A800F014FD82
:10B32000002C2846AEBF002601266442F4F75AFFDF
:10B33000A04225D28022202105A800F005FD284644
:10B34000F4F750FF241A04F198030DEB03040023D3
:10B3500004F8843C56BB2846F4F744FF013000F063
:10B360000DFB0446294600F07FFD05A9284600F0A4
:10B370007BFD2146284600F00BFD204600F006FB31
:10B38000284627B0BDE8F08F00220D4BF5F718FADC
:10B390000AF1010A84E70C49BAE7024626B10B49D3
:10B3A000284600F097FCB6E70949F9E7284605A9C1
:10B3B00000F0EEFCE4E700BF0000E03F0000F03FDB
:10B3C0000000244075D5000876D5000880D5000817
:10B3D00081D50008F0B503468BB0084669B3911ECD
:10B3E000222931D80A2A06D1002B04DA01265B4231
:10B3F00001AD29460EE00026FAE7B3FBF2F402FBAA
:10B4000014372346092FFCB294BF30345734E4B2CA
:10B4100001F8014B002BF0D1A942EED0034616B142
:10B420002D2203F8012B0A465C1EAA4207D84A1BAC
:10B430008D4288BF0022002199540BB0F0BD12F854
:10B44000016D04F8016FF0E70020F6E7FFF7C2BFD7
:10B4500070B504468AB0084689B1931E222B23D8C2
:10B4600001AD29466CB9A9420BD00B46421EAB4236
:10B4700015D84B1B8D4288BF00230022C2540AB04E
:10B4800070BDB4FBF2F302FB13461C46092EF3B267
:10B4900094BF30335733DBB201F8013BE2E713F8D6
:10B4A000014D02F8014FE2E70020E8E7FFF7D0BFC7
:10B4B00008B50320FBF7D4FDBDE8084000F052BA00
:10B4C00008B5AFF30080FAF7EFF8FAF705FC00F0E3
:10B4D0003BFAFAE7C0F30312042A034610B50ED86C
:10B4E0000020084AD9B252F8044B8C4203D103F42D
:10B4F000E063184310BD01302528F4D1FAE7252078
:10B50000F8E700BF48DB000810B5C4B2092C0346B9
:10B5100017D82D4900F4E06251F824100A43C9B24B
:10B52000242926D8294A092C52F8210017D8264A5E
:10B5300052F824201A4302F4E0621043421C1ED049
:10B5400010BD00F0C002C02A19D1C92C17D81E495D
:10B5500000F03F0051F8201003F4E062DEE703F052
:10B56000C002C02A2AD1184A03F03F0152F8212014
:10B57000E0E702F0C000C02801D1C92908D9CA2BD0
:10B580001FD0CB2B41F2020018BF4FF0FF30D7E79E
:10B590000D4902F03F0251F822000C4A092C52F8E2
:10B5A000200002D851F82420C4E703F0C002C02ACA
:10B5B00004D103F03F0251F82220BBE74FF4E062D0
:10B5C000BBE741F20100BBE720DB000848DB0008D5
:10B5D000FEF776FC0B480C490C4A002302E0D458D5
:10B5E000C4500433C4188C42F9D3094A094C0023CF
:10B5F00001E013600432A242FBD300F00FFCFFF71E
:10B600005FFF7047000000200403002054DD0008A5
:10B6100008030020A8140020FEE791420FD008D9AB
:10B620000123891A8B40984208D30130C840013861
:10B63000704720B10130521A9040F8E7002070475F
:10B64000431E1F2B05D80C22024B1860024B1A60B8
:10B650007047FEE7B0020020AC020020431E1F2B03
:10B6600007D8044B10281860A8BF1020024B1860A0
:10B670007047FEE7A8020020A4020020014B1860DA
:10B68000704700BFA002002010B5FFF73DFF431C2C
:10B690000AD0064C2168FDF74BFF054B21681A685C
:10B6A000BDE81040FFF7B9BF002010BDAC0200207C
:10B6B000B0020020C3B2242B2DE9F04105460E460E
:10B6C0002DD83D4A00F4E06452F823301C43671C37
:10B6D0006FD020463949FEF7D9FA394F80B3394A3D
:10B6E000C4F3031152F8210004F00F0320FA03F50C
:10B6F000ED075FBF012505FA03F3034342F821304C
:10B70000304639684FF00C0248BF0025FFF785FF2F
:10B710002A4601462046BDE8F041FDF765BE00F02F
:10B72000C002C02A45D1C92B43D8274B00F03F02A5
:10B7300053F82220204B00F4E06453F82230C5E790
:10B7400020462249FEF7A2FA8046F8B11D4AC4F30A
:10B75000031152F8210004F00F0520FA05F3DB076E
:10B760005FBF0123AB40034342F82130184B3968D7
:10B770001D6830462A46FFF750FF16490246EBB2D5
:10B780002046BDE8F0410968FDF752BF2846012177
:10B7900000F022F8396830460822FFF73EFF7F2884
:10B7A00098BF41462846BDE8F04188BF012100F01E
:10B7B0007DB8BDE8F08100BF48DB000878DA0008FA
:10B7C000A80200204C13002020DB0008F0D700085E
:10B7D000A4020020A0020020C3B2242B2DE9F041D6
:10B7E0000D462AD82C4A00F4E06452F823301C435A
:10B7F000621C4ED0294EC4F3031756F8273004F0CC
:10B800000F0823FA08F3DB0710D520462449FEF77A
:10B810003DFA18B32046FDF73BFE012256F82730CB
:10B8200002FA08F223EA020346F82730052D1FD852
:10B83000DFE805F01F2B2527292D00F0C002C02AC4
:10B8400027D1C92B25D8174B00F03F0253F82220EF
:10B85000114B00F4E06453F82230C8E72046124947
:10B86000FEF714FA0028D8D02046FDF733FFD4E7BE
:10B87000FEE700212046BDE8F041FEF717BA10218F
:10B88000F8E72021F6E70321F4E70121F2E7092197
:10B89000F0E7BDE8F08100BF48DB00084C13002052
:10B8A00078DA000820DB0008F0D70008C3B2242BA8
:10B8B00019D8184A00F4E06052F823301843C0F356
:10B8C0000313042B98BF144A00F00F0098BF52F8DE
:10B8D0002320124B88BF002253F82030C3F30F23DC
:10B8E000A9B11361704700F0C002C02A0CD1C92B66
:10B8F0000AD80B4B00F03F0253F82220054B00F40E
:10B90000E06053F82230D9E74FF0FF30D7E75361BA
:10B91000704700BF48DB000878020020E8D5000827
:10B9200020DB0008FDF728BFFDF702BF38B504464D
:10B9300048B1FDF721FF054600F016F8FDF71CFFA2
:10B94000431BA342F8D338BD08B5044B2BB10448C0
:10B95000FEF709FF08B1AFF3008008BD000000004A
:10B9600030120020FDF754BF70470A22002100F07A
:10B9700073B90A22002100F06FB90000024B0146A2
:10B98000186800F02DB800BFB4020020024B014639
:10B99000186800F083BA00BFB402002070B50F4EE3
:10B9A0000C463168054611B900F022FA3060214694
:10B9B000284600F01DFA431C03D14FF0FF34204607
:10B9C00070BDC41C24F00304A042F8D0211A2846FC
:10B9D00000F00EFA0130F2D1EFE700BF6013002053
:10B9E0002DE9F843CD1C25F0030508350C2D38BF93
:10B9F0000C25002D064601DBA94204D90C23336037
:10BA00000020BDE8F883DFF8D48000F069F8D8F8AA
:10BA100000301C4644BB29463046FFF7BFFF431C9D
:10BA2000044658D1D8F800402746002F43D1002CB7
:10BA30004BD023683946304604EB030900F0D8F9AF
:10BA4000814542D1216830466D1A2946FFF7A6FF8D
:10BA500001303AD023682B442360D8F800305A686C
:10BA600062BBC8F800700FE02268521B20D40B2A7A
:10BA700017D96119A342256018BF5960636808BFD0
:10BA8000C8F8001062514B60304600F02FF804F106
:10BA90000B00231D20F00700C21A1CBF1B1AA35065
:10BAA000AFE76268A3420CBFC8F800205A60EBE71A
:10BAB00023466468AEE73C467F68B6E71A465B6893
:10BAC000A342FBD100235360DEE70C2330463360F2
:10BAD00000F00CF894E70560D6E700BF641300207F
:10BAE000014800F0BFB900BFA4140020014800F0D5
:10BAF000BAB900BFA4140020024B0A4601461868D8
:10BB000000F002B8B40200202DE9F04107461446C7
:10BB10000D4621B91146BDE8F041FFF761BF2AB9D2
:10BB200000F0BCF925462846BDE8F08100F0FEF99A
:10BB30008442064602D8B4EB500FF4D8214638466A
:10BB4000FFF74EFF804608B94546ECE7B44222466F
:10BB5000294628BF324600F08FF92946384600F0C2
:10BB60009DF9F1E7242B2DE9F0478646904601D850
:10BB7000012B06D100F04CF9162303600020BDE82C
:10BB8000F0870D4633482A4615F8014B065D16F03E
:10BB90000806F8D12D2C10D101262C78951C33F0F5
:10BBA000100215D1302C0DD12A7802F0DF02582A6C
:10BBB00008D16C78023510230AE02B2C04BF2C78B6
:10BBC000951CECE7002BF6D1302C14BF0A23082378
:10BBD000002206F1004C0CF1FF3CBCFBF3F91046CF
:10BBE00003FB19CAA4F13007092F0FD83C46A34222
:10BBF0001BDD571C07D0814514D301D1A24511DBB1
:10BC0000012200FB034015F8014BEBE7A4F14107CB
:10BC1000192F01D8373CEAE7A4F16107192F04D89E
:10BC2000573CE4E74FF0FF32EDE7531C08D12223E5
:10BC30006046CEF80030B8F1000FA0D0691E06E0D3
:10BC400006B14042B8F1000F99D0002AF6D1C8F8E9
:10BC5000001094E711DC000813460A46014602482A
:10BC60000068FFF77FBF00BFB40200200CB430B5FE
:10BC7000174B0C1E1D689DB008DA8B234FF0FF3068
:10BC80002B601DB0BDE8304002B070474FF4027326
:10BC9000ADF814300CBF234604F1FF33049307932F
:10BCA0004FF6FF7302900690ADF81630284621AB90
:10BCB000209A02A9019300F09DF9431CBCBF8B237D
:10BCC0002B60002CDDD00022029B1A70D9E700BF48
:10BCD000B40200200EB46FF0004100B59CB01DAB63
:10BCE00002900690079104910848094953F8042BE3
:10BCF0000591006802A9019300F07CF90022029BE3
:10BD00001A701CB05DF804EB03B07047B402002059
:10BD10000802FFFF884210B501EB020402D98442F9
:10BD2000234607D8431EA14208D011F8012B03F87F
:10BD3000012FF8E7014602448A4200D110BD13F8F2
:10BD4000014D02F8014DF7E703460244934200D14A
:10BD5000704703F8011BF9E7024630B50B4D12F8A6
:10BD6000013BE85C00F00300012811F8010B08BF5B
:10BD700020332C5C04F00304012C08BF20301B1A74
:10BD800002D10028EBD130BD1846FCE711DC0008D9
:10BD9000024610B5147813460132002CFAD1013B4B
:10BDA00011F8012B03F8012F002AF9D110BD034629
:10BDB000C9B2184613F8012B12B18A42F9D1704763
:10BDC000002918BF00207047034610B5013932B171
:10BDD00011F8014F013A03F8014B002CF7D1002173
:10BDE0001A44934200D110BD03F8011BF9E700008B
:10BDF00038B50023054D044608462B60FEF760FC6D
:10BE0000431C02D12B6803B1236038BDA01400206D
:10BE1000014B1868704700BFB402002070B50026BF
:10BE20000C4D0D4C641BA410A64209D100F0CAFEB3
:10BE300000260A4D0A4C641BA410A64205D170BD11
:10BE400055F8043B98470136EEE755F8043B984710
:10BE50000136F2E730DD000830DD000830DD000893
:10BE600048DD000870477047034611F8012B03F8BE
:10BE7000012B002AF9D170470A44914200F1FF33A7
:10BE800000D1704710B511F8014B914203F8014FF2
:10BE9000F9D110BD004870470000C07F38B5054695
:10BEA000002940D051F8043C0C1F002BB8BFE41807
:10BEB000FFF716FE1C4A136833B963601460284606
:10BEC000BDE83840FFF712BEA34208D92068211808
:10BED0008B4201BF19685B6809182160EDE71A46BB
:10BEE0005B680BB1A342FAD911685018A0420BD17C
:10BEF00020680144501883421160E0D118685B68E3
:10BF0000084410605360DAE702D90C232B60D6E7AF
:10BF1000206821188B4201BF19685B6809182160ED
:10BF200063605460CBE738BD6413002051F8043CD3
:10BF3000181F002BBCBF0B58C01870472DE9F047E5
:10BF40001F468E688246BE420C4690460B682DD82E
:10BF5000B1F90C2012F4906F26D06569096905EBE0
:10BF60004505A3EB010905EBD5757B1C4B446D1012
:10BF70009D4238BF1D46530527D52946FFF730FDA2
:10BF8000064660B34A462169FFF776FFA38923F48A
:10BF9000906343F08003A38126614E4426603E46B1
:10BFA0006561A5EB0905A560BE4200D93E46324653
:10BFB00041462068FFF7AEFE0020A3689B1BA360EC
:10BFC000236833442360BDE8F0872A46FFF79CFDD1
:10BFD00006460028E0D150462169FFF75FFF0C2399
:10BFE000CAF80030A3894FF0FF3043F04003A3812B
:10BFF000E9E700002DE9F04F98468B8907461B06BC
:10C000000D4614469DB010D50B6973B94021FFF75A
:10C01000E7FC2860286130B90C233B604FF0FF300B
:10C020001DB0BDE8F08F40236B61002309932023EE
:10C030008DF8293030234FF00109CDF80C80DFF85E
:10C0400098818DF82A3023469A4613F8012B0AB1BD
:10C05000252AF9D1BAEB040B0BD05B4622462946C0
:10C060003846FFF76BFF013000F0A780099A5A4469
:10C0700009929AF80030002B00F09F8000234FF0C7
:10C08000FF32CDE905230AF1010A049307938DF8E5
:10C0900053301A935446052214F8011B4E4800F001
:10C0A00035FA049AD8B9D00644BF20238DF853300E
:10C0B000110744BF2B238DF853309AF800302A2BF8
:10C0C00015D0544600204FF00A0C079A214611F86B
:10C0D000013B303B092B4BD9B0B1079214E0A0EBE8
:10C0E000080309FA03F31343A2460493D2E7039B20
:10C0F000191D1B680391002BBBBF5B4242F002027B
:10C1000007930793B8BF049223782E2B0AD1637844
:10C110002A2B32D1039B02341A1D1B68039243EA77
:10C12000E3730593DFF8B4A003225046217800F0B2
:10C13000EDF938B14022049BA0EB0A008240134382
:10C140000134049314F8011B062225488DF82810A9
:10C1500000F0DCF9002836D0224B1BBB039B0733D1
:10C1600023F0070308330393099B334409936AE7D9
:10C170000C4601200CFB0232A8E700234FF00A0C0A
:10C18000194601340593204610F8012B303A092A4C
:10C1900003D9002BC6D00591C4E7044601230CFB4C
:10C1A0000121F0E703AB00932A4638460E4B04A961
:10C1B000AFF30080421C0646D6D1AB895B063FF543
:10C1C0002DAF09982CE703AB00932A463846064B5F
:10C1D00004A900F07DF8EDE785D500088BD50008AF
:10C1E0008FD50008000000003DBF00082DE9F04792
:10C1F000164698468A680B6907469342B8BF1346AD
:10C20000336091F843200C46DDF820900AB10133E9
:10C2100033602368990642BF336802333360256870
:10C2200015F0060506D104F1190AE36832689B1A75
:10C23000AB422BDC94F843302268003B18BF01234B
:10C24000920630D44146384604F14302C8470130D3
:10C2500023D02368226903F00603042B14BF0025B2
:10C2600033684FF0000608BFE56804F11A0408BF00
:10C27000ED1A54F8123C08BF25EAE5759342C4BF95
:10C280009B1AED18B5421AD1002008E0012352464E
:10C2900041463846C847013003D14FF0FF30BDE872
:10C2A000F0870135C1E73020E11881F843005A1CBE
:10C2B00094F845102244023382F84310C2E7012368
:10C2C000224641463846C8470130E6D00136D9E714
:10C2D0002DE9FF470F7E9146782F80460C469A46FF
:10C2E0000C9E01F1430207D8622F0AD8002F00F0FC
:10C2F000D180582F00F0B88004F1420684F84270D3
:10C300003AE0A7F16303152BF6D801A151F823F009
:10C3100069C300087DC30008F9C20008F9C200081B
:10C32000F9C20008F9C200087DC30008F9C200087C
:10C33000F9C20008F9C20008F9C200087BC400086D
:10C34000A7C3000835C40008F9C20008F9C20008F4
:10C350009DC40008F9C20008A7C30008F9C200087C
:10C36000F9C200083DC4000833681A1D1B6832601A
:10C3700004F1420684F8423001239CE033682068CF
:10C38000191D3160060601D51D6803E04506FBD581
:10C39000B3F90050002D03DA2D236D4284F84330A9
:10C3A0000A23584811E021683368080653F8045BF3
:10C3B00002D4490648BFADB26F2F336014BF0A23C1
:10C3C00008235048002184F843106668002EA660B8
:10C3D00005DB21682E4321F0040121604BD0164675
:10C3E000B5FBF3F103FB1157C75D06F8017D2F463E
:10C3F000BB420D46F4D9082B0BD12368DF0708D5C3
:10C40000236961689942DEBF302306F8013C06F1DA
:10C41000FF36921B22614B4621464046CDF800A0D4
:10C4200003AAFFF7E3FE01304AD14FF0FF3004B01A
:10C43000BDE8F087236843F0200323607827324863
:10C4400084F84570236831681F0651F8045B02D4F4
:10C450005F0648BFADB23160D90744BF43F0200347
:10C4600023601DB11023ADE72648E9E7236823F0D8
:10C4700020032360F6E71646BDE733682568181DDC
:10C48000616930602E061B6801D5196002E06806FC
:10C49000FBD51980002316462361BCE733680021D1
:10C4A0001A1D32601E686268304600F02FF808B12D
:10C4B000801B606063682361002384F84330AAE72F
:10C4C0003246494640462369D0470130ADD0236803
:10C4D0009B0713D4E068039B9842B8BF1846A6E7B1
:10C4E0000123324649464046D04701309DD00135B0
:10C4F000E36803995B1AAB42F2DCEBE7002504F139
:10C500001906F5E796D50008A7D50008034610B52B
:10C51000C9B202449342184601D1002003E00478D6
:10C5200001338C42F6D110BD062008B500F02CF87E
:10C530000120FEF7E3F81F2938B505460C4604D95B
:10C54000162303604FF0FF3038BDC26B12B152F8B2
:10C5500021304BB9284600F031F8224601462846E2
:10C56000BDE8384000F018B8012B0AD0591C03D19F
:10C57000162303600120E7E70021204642F824103B
:10C5800098470020E0E70000024B01461868FFF7DB
:10C59000D2BF00BFB402002038B50023064D0446C8
:10C5A000084611462B60FEF7ABF8431C02D12B68FE
:10C5B00003B1236038BD00BFA0140020FEF7A8B867
:10C5C0002DE9F8438046894614461D4600F04EF892
:10C5D000224606460F46404649462B46F4F760FA87
:10C5E00030B92046294600220023F4F727FA18B96B
:10C5F00030463946BDE8F883FFF70AFC00220023E5
:10C600002121016010461946F4F7DAF806460F4674
:10C6100030463946BDE8F88338B5044600F0A2F943
:10C62000214605462046F4F7BDFD70B9204600219D
:10C63000F4F7AEFD48B920460021F4F781FD30B192
:10C64000FFF7E6FB2223074D0360284638BDFFF7BE
:10C65000DFFB2122034604481A60BDE83840FFF79B
:10C6600019BC00BF000080FF14DD00082DE9F04771
:10C6700023F000480D4652EA0801044646D0B3496B
:10C6800025F0004A8A45A94640D85042B04E40EABB
:10C69000020148EAD171B142964637D8C2451F46D9
:10C6A000214605F0004C3BDCC0F28180A2427ED8DE
:10C6B00000F0B380354243D1BAF1000F32D1002CE3
:10C6C000234640F32381A34A5B00002B02F1FF3293
:10C6D000FADC9F4B3B40002B40F09180B8F1000FFB
:10C6E00040F0DB80BEF1000F73466BDC994E9A4838
:10C6F000801A1F2800F3EB8002F21E4321FA03F395
:10C700000AFA00FA43EA0A03814068E02046294613
:10C71000F3F72CFF02460B46F4F752F8BDE8F0871A
:10C7200035420DD18C4A4FEACA235B00002B02F13F
:10C73000FF32CEDD5B00002B02F1FF32F5DCC8E7F3
:10C74000834B4FEA2A523B40A2F2FF3293B34FEAA7
:10C750002850C9F31303A0F2FF3643F48013A1EB72
:10C760000E00C7F3130545F48015921B0BD163E04F
:10C77000013858D4A1EB0E04E30F013A03EB400358
:10C780004FEA440156D07145A3EB0500F0D30028D1
:10C79000A1EB0E0447DB50EA0403EDD16F4B4FEAE7
:10C7A000DC7C03EBCC03D3E90001BDE8F087204635
:10C7B0002946B3E7B8F1000F6FD1BEF1000F734601
:10C7C00040F3AF80634E5B00002B06F1FF36FADCCE
:10C7D000614B9A428BDBC9F3130343F480135E4C25
:10C7E000A41B1F2C4ADC06F21E452EFA05F508FA9A
:10C7F00004F00EFA04FE0543A1EB0E00B5E7564C1B
:10C800004FEA2858A41A1F2CA8F2FF366EDD544BAD
:10C810009B1A01FA03F30021A3E7504B03EB1C73AF
:10C82000D3E900017AE7C80F013A00EB43034FEA6E
:10C830004101A8D1A1EB0E005A1B8E4588BF02F121
:10C84000FF32002ABCBF08461A4652EA000305D14F
:10C85000A4E7C30F03EB42024000013EB2F5801F84
:10C86000F7DB3D4B9E4221DBA2F5801206F2FF363C
:10C8700042EA0C0242EA065529464FE7384D921B20
:10C88000A5EB06050EFA05F518BF4FF0000E7FF474
:10C890007AAF08465A1BD4E72E4A2F4E4FEAC823D8
:10C8A0005B00002B06F1FF36FADC91E79B1B142B93
:10C8B00013DC06F21E41D84002FA01F142FA03F3FA
:10C8C00043EA0C0C41EA00026146104626E7244B7D
:10C8D0009B1A01FA03F3002181E71F2B12DC06F2F9
:10C8E0001E4120FA03F38A401A43EDE702F21E4389
:10C8F00021FA03F30AFA04FA43EA0A03A140A1EB7E
:10C900000E002EE7164B9B1B1A41DDE7104B3B40F8
:10C910007BB14FEA28500F4AA0F2FF36E30A6105C7
:10C92000EDE7C9F313030B2515240A4E43F48013D6
:10C930005BE7B8F1000FAFD1BEF1000F1346054A17
:10C940003FF740AF15201646D6E600BFFFFFEF7F4A
:10C950000000F07FEDFBFFFF02FCFFFF18DD000889
:10C96000E2FBFFFF2DE9F84F30F000432BD0002809
:10C970000146034640DBB0F1FF4F39DAB0F5000F56
:10C9800041DB0021804AC3F316052A44DC1502F47A
:10C9900000007F3C80F07E500C4428434FF07E51D5
:10C9A00004EBD254F4F72EF9784B05F10F02134043
:10C9B000064683BB0021F4F7C3FB002800F0A380E8
:10C9C00044B9002004E000214FF04C40F4F7D8FABD
:10C9D000BDE8F88F2046F4F7CBF96D490546F4F72A
:10C9E0001BFA6C4904462846F4F716FA014620461D
:10C9F000F4F70AF9BDE8F88FF4F704F90021F4F729
:10CA0000BFFABDE8F88F4FF09841F4F705FA6FF0E0
:10CA100018010346B6E74FF08041F4F7F5F80146F8
:10CA20003046F4F7ADFA80462046F4F7A1F94146C6
:10CA300081464046F4F7F0F901468246F4F7ECF9F6
:10CA400007465549F4F7E8F95449F4F7DDF8394653
:10CA5000F4F7E2F95249F4F7D7F83946F4F7DCF97C
:10CA60005049F4F7D1F85146F4F7D6F94E498246C9
:10CA70003846F4F7D1F94D49F4F7C6F83946F4F7DA
:10CA8000CBF94B49F4F7C0F83946F4F7C5F901463C
:10CA90005046F4F7B9F8DFF81CB10746AB44C5F5CA
:10CAA000571505F5227545EA0B05002D4CDD4FF0B5
:10CAB0007C513046F4F7B0F93146F4F7ADF905464C
:10CAC00038462946F4F7A0F84146F4F7A5F9074699
:10CAD000002C47D02E494846F4F79EF92D490446CC
:10CAE0004846F4F799F93946F4F78EF80146284696
:10CAF000F4F788F83146F4F785F801462046F4F754
:10CB000081F8BDE8F88F2C493046F4F785F90146E5
:10CB10004FF07C50F4F776F8314605463046F4F78E
:10CB20007BF901462846F4F777F90546ACB1204673
:10CB3000F4F71EF916490746F4F76EF9044638462D
:10CB40001449F4F769F9D1E701463046F4F75AF889
:10CB50004146F4F761F905466CB929463046F4F7C9
:10CB600051F835E701462846F4F74CF801463046BF
:10CB7000F4F748F82CE706494846F4F74DF905491B
:10CB800004464846DDE700BF20FB4A00F0FF7F0077
:10CB90008071313FD1F717379788173E25333A3EDA
:10CBA0002549923EABAA2A3F4FD01C3E298E633EB8
:10CBB000CDCCCC3E305CCFFFABAAAA3E08B5FFF788
:10CBC000B3FC0000F8B500BFF8BC08BC9E46704737
:0CCBD000F8B500BFF8BC08BC9E467047DA
:10CBE0000000000000003440000000000000004091
:10CBF0001975ADBD4F55B53F2C0FD253E410813F91
:10CC0000E5BEC26F30C1363F000000000000244086
:10CC1000000000000000F03F1975ADBD4F55A53F65
:10CC20007D09151C5E10713F4FB7C67A7DC0263F47
:10CC300041505A4E4657006025632563256325639E
:10CC400025632563256325630025732563256325F7
:10CC5000637D0025303264253032642E2530326405
:10CC600025630025303364253032642E253032644C
:10CC70002563002125732563257325630025303244
:10CC8000643A253032643A25303264002564002C41
:10CC900000253034580024242424002A002F413D4C
:10CCA000253036642F502564532564542530326472
:10CCB00056253034644330302025730020616C7475
:10CCC0003A25646D202573002125732F25735F633A
:10CCD000253033647325303364672530336474251D
:10CCE0003033646825303264622530356420545F07
:10CCF0004578743D25644320545F496E743D256436
:10CD0000432052483D2564252520556261743D2508
:10CD1000646D562C20257300212000414C542000C6
:10CD20004D20004E3043414C4C004F4E00575800B0
:10CD30004E4F524D414C0046554C4C0052454455C7
:10CD400043454400484F525553465251000A4F4BF9
:10CD5000003E000A4672657175656E6379206F75D5
:10CD600074206F662072616E6765004150525346B1
:10CD700052510052545459465251004D4F5253454E
:10CD80004652510055415254424452000A4F4B20E2
:10CD9000284F6E6C792076616C69642061667465D9
:10CDA00072207265626F6F7429000A5541525420D7
:10CDB0006261756472617465206973206F75742097
:10CDC0006F662072616E6765004D4F525345535038
:10CDD00045454400524144494F505752000A504F74
:10CDE000574552203020746F203700484F5255531A
:10CDF0004944000A486F727573205061796C6F6105
:10CE000064204944206F7574206F662072616E67DC
:10CE10006500484F525553424452000A486F72759C
:10CE200073204261756472617465206F7574206F40
:10CE3000662072616E676500525454594244520034
:10CE40000A52545459204261756472617465206FAE
:10CE50007574206F662072616E6765005254545974
:10CE60005348494654000A5254545920536869663D
:10CE70007420313D3237302C20323D353430202E75
:10CE80002E2E487A005254545942495453000A52A3
:10CE900054545920626974732037206F722038000F
:10CEA0005254545953544F50000A525454592073F9
:10CEB000746F706269747320312C20312E35206FAD
:10CEC000722032004150525353534944000A41509A
:10CED000525320535349442030202D2031350041F6
:10CEE00050525353594D424F4C00415052535441AC
:10CEF000424C4500484F4C444F4646004150525327
:10CF000043414C4C000A4E6F2043414C4C5349471F
:10CF10004E20646566696E656400525454594341FD
:10CF20004C4C00415052534D5347000A4E6F204D18
:10CF300045535341474520646566696E6564004802
:10CF40004F525553454E41424C45000A4572726F4F
:10CF5000720052545459454E41424C450041505282
:10CF600053454E41424C45004D4F525345454E416D
:10CF7000424C4500415052534D4F4445004D4F5295
:10CF800053454D4F444500415052534841420041A2
:10CF90005052534D4943450048454C50004176613D
:10CFA000696C61626C6520636F6D6D616E647300A6
:10CFB000636F6D6D616E643C53504143453E7061DB
:10CFC00072616D657465723C454E5445523E202831
:10CFD000636F6D6D616E647320616C6C77617973E2
:10CFE00020776974686F7574205350414345212937
:10CFF0000064697370202873657420706172616DBC
:10D0000065746572732900686F727573667271203A
:10D0100066727175656E63792028696E20487A2C76
:10D02000206B487A206F72204D487A290061707217
:10D03000736672712066727175656E6379007274C1
:10D0400074796672712066727175656E6379006DB0
:10D050006F7273656672712066727175656E637941
:10D0600000686F6C646F66662074696D6520287453
:10D07000696D6520696E207365632E206D696E2E63
:10D080002031352900686F727573656E61626C6559
:10D0900020782028302D64697361626C6520312D01
:10D0A000656E61626C65290061707273656E6162A4
:10D0B0006C6520782028302D64697361626C65206E
:10D0C000312D656E61626C65290072747479656ECC
:10D0D00061626C6520782028302D64697361626C10
:10D0E0006520312D656E61626C6529006D6F72730C
:10D0F00065656E61626C6520782028302D646973E7
:10D1000061626C6520312D656E61626C652900611C
:10D110007072736D736720636F6D6D656E74202818
:10D120006170727320636F6D6D656E74206D6178D0
:10D13000203132302063686172290061707273633C
:10D14000616C6C2063616C6C20286D6178203620E6
:10D150006368617229007274747963616C6C206316
:10D16000616C6C20286D61782031352063686172B4
:10D170002900686F7275736964207820285061797E
:10D180006C6F61642049442900686F727573626432
:10D190007220782028686F727573206261756472DE
:10D1A0006174652900727474796264722078202831
:10D1B0007274747920626175647261746529007299
:10D1C000747479626974732078202837206F722014
:10D1D0003829007274747973746F70207820283144
:10D1E0002C20312E35206F72203229007274747910
:10D1F0007368696674207820287368696674203DB6
:10D200002078202A20323730487A290061707273E2
:10D2100073736964207820283020746F2031352999
:10D22000006170727373796D626F6C20782028735F
:10D23000796D626F6C2066726F6D20617072732001
:10D240007461626C652900617072737461626C65EF
:10D2500020782028617072732073796D626F6C2062
:10D260007461626C65202F206F72202900617072DA
:10D27000736D6F646520782028302D6E6F726D613C
:10D280006C2C20312D77782900617072736861628F
:10D2900020782028302D6F66662C20312D6F6E2966
:10D2A00000617072736D69636520782028302D6F7E
:10D2B00066662C20312D6F6E29006D6F7273657359
:10D2C000706565642078202857504D29006D6F7275
:10D2D00073656D6F646520782028302D72656475E4
:10D2E0006365642C20312D66756C6C290072616455
:10D2F000696F70777220782028302D37290075618A
:10D30000727462647220782028313230302C3234CA
:10D3100030302C343830302C393630302C313932F2
:10D3200030302C33383430302C35373630302C37E1
:10D33000363830302C3131353230302900444953C1
:10D34000500053657420706172616D65746572730D
:10D3500000415052533A2000415052532043414C17
:10D360004C3A200041505253204672657175656EEB
:10D3700063793A2000204D487A00415052532043AF
:10D380006F6D6D656E743A200041505253205353B7
:10D3900049443A2000415052532053796D626F6CDA
:10D3A0003A2000415052532053796D626F6C2054E3
:10D3B00061626C653A200041505253204D4F444504
:10D3C0003A200041505253204841423A20004150F7
:10D3D0005253204D49432D453A2000525454593A56
:10D3E0002000525454592043414C4C3A200052548E
:10D3F0005459204672657175656E63793A20005202
:10D4000054545920426974733A200052545459209C
:10D4100053746F7020426974733A20005254545907
:10D420002042617564726174653A20005254545907
:10D430002053686966743A2000484F5255533A2089
:10D4400000484F5255532049443A2000484F525506
:10D4500053204672657175656E63793A2000484FB6
:10D460005255532042617564726174653A20004DD3
:10D470004F5253453A20004D4F5253452046726556
:10D480007175656E63793A20004D4F5253452053B4
:10D49000706565643A20004D4F525345204D6F64CE
:10D4A000653A2000524144494F20504F5745523A67
:10D4B0002000484F4C44204F46463A2000554152E8
:10D4C000542062617564726174653A20000A3E3FBF
:10D4D0000052533431206261736564207061796C4D
:10D4E0006F616420666F722053544D333246313081
:10D4F00030002D2E2D2E002E2E2D2E002E2D2E2ED8
:10D50000002E2D2D2E002D2D2E2D002D2E2E2D00FA
:10D510002D2E2D2D002D2D2D2D2D002E2D2D2D2D93
:10D52000002E2E2D2D2D002E2E2E2D2D002E2E2EAA
:10D530002E2D002E2E2E2E2E002D2E2E2E2E002D98
:10D540002D2E2E2E002D2D2D2E2E002D2D2D2D2E5F
:10D55000002E2D2E2D2E2D00504E41424C00524DAE
:10D560004300474741000D0A006E616E00696E6618
:10D57000006F7666002D256C642E25302A6C6400C1
:10D580002D256C6400232D302B2000686C4C006529
:10D5900066674546470030313233343536373839DF
:10D5A0004142434445460030313233343536373812
:10D5B00039616263646566000102030405060708B9
:10D5C000090A0B0C0D0E0F100203040506070809CB
:10D5D0000A0B0C0D0E0F10100201040302040810B8
:10D5E00004004000000400000101000002020000ED
:10D5F00004040000080800001010000020200000B3
:10D60000404000008080000001000104020002048C
:10D610000400040408000804100010042000200482
:10D620004000400480008004000000000102030468
:10D6300000000000000000000102030406070809C2
:10D640000400000000300140120200000F00000042
:10D6500000300140120100001C00000000380040B2
:10D6600012000000FFFFFFFF0000000000000000AC
:10D67000050000000030014012020000130000000D
:10D6800000300140120100001D0000000038004081
:10D6900012000000FFFFFFFF00000000000000007C
:10D6A00006000000003001401202000014000000DB
:10D6B00000300140120100001E0000000038004050
:10D6C00012000000FFFFFFFF00000000000000004C
:10D6D00007000000003001401202000015000000A9
:10D6E00000300140120100001F000000003800401F
:10D6F00012000000FFFFFFFF00000000000000001C
:10D700000000000000440040120000000B00000078
:10D7100000380140120000001D00000000480040D9
:10D72000120B00001D01000000480040120A00001A
:10D73000FFFFFFFF000000000000000001000000EC
:10D7400000440040120800000C00000000380140B6
:10D75000120000001E0000000048004012000000FF
:10D760001E01000000480040120A0000FFFFFFFFFA
:10D770000000000000000000030000000044004022
:10D78000100800000A0000000038014010060000E8
:10D790001700000000380140100500001B000000C9
:10D7A0000048004010000000FFFFFFFF00000000E5
:10D7B00000000000020000000044004012080000C9
:10D7C00009000000003801401206000016000000A9
:10D7D00000380140120500001A0000000048004017
:10D7E00012000000FFFFFFFF00000000000000002B
:10D7F0000000000000000040128000000001000056
:10D8000000000040129000000100000000000040F5
:10D81000121201000101000000000040121001007E
:10D82000020000000000004012920100020100000E
:10D83000000000401291010002020000004001407F
:10D8400012A60000030000000000004012120200B7
:10D85000030100000000004012110200030200005A
:10D8600000400140122601000600000000040040B4
:10D8700012950000060100000044014012A70000BC
:10D8800007000000002C0140128D1000070100006D
:10D89000000400401215010007020000004801408A
:10D8A00012A9000008000000002C0140128E0000A8
:10D8B00008010000002C0140128D0000090000004A
:10D8C000002C0140120E010009010000002C014053
:10D8D000120D01000A000000002C0140128E010010
:10D8E0000A010000002C0140128D01000B00000015
:10D8F000002C0140120E02000B010000002C014020
:10D90000120D02000F000000000000401291000004
:10D910000F01000000000040128F00001000000006
:10D92000002C0140120D1100100100000004004005
:10D930001295010010020000000400401294010042
:10D9400011000000002C0140128D11001101000097
:10D950000004004012150200110200000004004003
:10D960001214020013000000000000401211010018
:10D970001301000000000040120F0100140000001D
:10D980000004004012940000150000000004004054
:10D990001214010016000000000800401297000059
:10D9A0001601000000440140128010001700000022
:10D9B0000008004012170100170100000048014054
:10D9C00012801000180000000008004012970100AB
:10D9D000180100000044014012A8000019000000D6
:10D9E0000008004012170200190100000048014021
:10D9F00012AA00001A00000000000040129001006E
:10DA00001A01000000000040128F01001B000000FE
:10DA100000000040121002001B0100000000004046
:10DA2000120F02001D000000002C0140128E100099
:10DA30001E000000002C0140120E11001E0100000B
:10DA40000040014012A500001F000000002C014012
:10DA5000128E11001F0100000040014012801000D2
:10DA60001F0200000040014012250100FFFFFFFFE0
:10DA700000000000000000000400000000740040EE
:10DA80000380000005000000007400400300010056
:10DA9000FFFFFFFF0000000000000000000000008A
:10DAA00000240140030000000100000000240140A8
:10DAB0000380000002000000002401400300010078
:10DAC0000300000000240140038001000400000066
:10DAD0000024014003000200050000000024014072
:10DAE0000380020006000000002401400300030040
:10DAF0000700000000240140038003001000000024
:10DB00000024014003000400110000000024014033
:10DB100003800400FFFFFFFF000000000000000082
:10DB200000000000010000000200000003000000EF
:10DB300004000000050000000600000007000000CF
:10DB400010000000110000000000000001000000B3
:10DB500002000000030000000400000005000000B7
:10DB60000600000007000000080000000900000097
:10DB70000A0000000B0000000C0000000D00000077
:10DB80000E0000000F000000100000001100000057
:10DB90001200000013000000140000001500000037
:10DBA0001600000017000000180000001900000017
:10DBB0001A0000001B0000001C0000001D000000F7
:10DBC0001E0000001F0000002D0000002E000000BD
:10DBD0002F000000300000003100000006000700A8
:10DBE000080000000000000000000000ADA70008D1
:10DBF0005DA8000891A70008BBAA000867A7000855
:10DC0000A1AC000877A70008A7AF0008C9AF0008BB
:10DC100000202020202020202020282828282820FC
:10DC200020202020202020202020202020202020F4
:10DC3000208810101010101010101010101010105C
:10DC4000100404040404040404040410101010104C
:10DC50001010414141414141010101010101010116
:10DC60000101010101010101010101011010101068
:10DC700010104242424242420202020202020202E8
:10DC8000020202020202020202020202101010103C
:10DC90002000000000000000000000000000000064
:10DCA0000000000000000000000000000000000074
:10DCB0000000000000000000000000000000000064
:10DCC0000000000000000000000000000000000054
:10DCD0000000000000000000000000000000000044
:10DCE0000000000000000000000000000000000034
:10DCF0000000000000000000000000000000000024
:10DD00000000000000000000000000000000000013
:10DD10000000000000000000000000000000000003
:08DD200000000000000000807B
:08DD2800A824FF7F01000000A8
:10DD3000B1B40008811200087D3B00086D5F000847
:08DD4000B9980008D1AC0008FD
:0CDD48005D1200083D3C000891990008A5
:10DD540002000300050007000B000D001100130072
:10DD640017001D001F00250029002B002F0035007F
:10DD74003B003D004300470049004F005300590059
:10DD84006100650067006B006D0071007F00830017
:10DD940089008B00950097009D00A300A700AD00AB
:10DDA400B300B500BF00C100C500C700D300DF0049
:10DDB400E300E500E900EF00F100FB0001010701C9
:10DDC4000D010F01150119011B0125013301370153
:10DDD40039013D014B0151015B015D017B017F0173
:10DDE4008501F502F90201030503000008D50008C6
:10DDF40040D50008F2D4000847D500084FD50008E4
:10DE0400F7D400084DD500083AD5000848D50008D5
:10DE140022D5000807D50008FCD4000818D500084E
:10DE24004ED5000817D5000801D5000806D500080E
:10DE3400F3D4000841D5000819D500080CD5000812
:10DE44002ED5000811D500080BD5000810D5000800
:10DE540046D5000815D500081BD5000821D50008B3
:10DE640027D500082DD5000833D5000839D500087A
:10DE74003FD5000845D500084BD5000819CD00084A
:10DE840051D50008B5620611020008012292B5625C
:10DE94000611020008002191B56206242400FFFF48
:10DEA400060300000000102700000500FA00FA0035
:10DEB40064002C0100000000102700000000000096
:10DEC40000004DDBB562068A090000010000210054
:10DED400112006F24F00000080250000FFFF000023
:10DEE4000100000001000000010000000000803F6C
:10DEF4004000000001000000010000000A000000D2
:10DF04000F000000FF000000050000007D0000007D
:10DF140064000000E093040001010000B603000067
:10DF24000100000000000C4200004040010000001D
:10DF3400E0930400010000000101000040771B0091
:10DF4400E20400000100000004000000FFFFFFFFE6
:10DF5400E80300000100000028000000CD4CD94374
:10DF6400020000000000004007000000102700002D
:10DF7400CD4CD94301000000010000002F4F015790
:10DF84004944453200415042433431000B00000003
:10DF94000040D843010100006400000000010000BB
:10DFA400CDCCDA43010000000500000001010000AF
:10DFB400FFFFFFFF010000000700000080250000B4
:10DFC400010100001000000000080140000C0140A5
:10DFD400001001400014014000180140FFFFFFFF42
:10DFE400003002400000000000127A00A814002053
:10DFF400E803000008000000080000000C00000016
:10E004000A000000B802002000000000681300208D
:10E01400D01300203814002000000000000000008D
:10E0240000000000000000000000000000000000EC
:10E0340000000000000000000000000000000000DC
:10E0440000000000000000000000000000000000CC
:04E0540000000000C8
:040000050800B5D169
:00000001FF
